:020000040800F2
:1080000090AC0020A1810008A9810008A9A800085F
:10801000AD810008AF810008B181000800000000B8
:10802000000000000000000000000000B381000814
:10803000B581000800000000B7810008B981000880
:10804000BB810008BB810008BB810008BB81000820
:10805000BB810008BB810008BB810008BB81000810
:10806000BB810008BB810008BB810008BB81000800
:10807000BB810008BB8100087B9600087F96000842
:10808000BB81000883960008BB810008BB81000803
:10809000BB810008BB810008BB810008BB810008D0
:1080A000BB810008BB810008BB810008BB810008C0
:1080B000A5680108BB810008BB810008BB810008DE
:1080C000BB810008BB810008BB810008BB810008A0
:1080D000BB8100084D7001085170010855700108FE
:1080E0004B9A0008BB810008BB810008BB810008D7
:1080F000BB810008BB810008BB810008879600088F
:10810000BB810008BB810008BB810008BB8100085F
:108110004570010849700108BB810008BB81000857
:10812000BB810008BB810008BB810008BB8100083F
:10813000BB810008BB810008BB810008BB8100082F
:10814000BB810008BB810008BB810008BB8100081F
:10815000BB8100088B9600088F96000859700108B3
:10816000BB810008BB810008BB810008BB810008FF
:10817000BB810008BB810008BB810008BB810008EF
:10818000BB810008BB810008DFF810D000F0C6FBFF
:10819000004800474D8D0108AFF3008090AC0020EF
:1081A0000648804706480047FEE7FEE7FEE7FEE791
:1081B000FEE7FEE7FEE7FEE7FEE7FEE749680108A7
:1081C000898100082DE9F05F0546002092469B4614
:1081D00088460646814640241BE0284641464746DD
:1081E000224600F020F853465A46C01A914110D357
:1081F00011461846224600F04EFA2D1A67EB010888
:108200004F4622460120002100F045FA17EB0009F5
:108210004E41201EA4F10104DFDC484631462A46C7
:108220004346BDE8F09F202A04DB203A21FA02F001
:108230000021704721FA02F3D040C2F120029140A0
:1082400008431946704740EA01039B0703D009E041
:1082500008C9121F08C0042AFAD203E011F8013B32
:1082600000F8013B521EF9D27047421E12F8013F3E
:10827000002BFBD111F8013B02F8013B002BF9D197
:108280007047421C10F8011B0029FBD1801A70476F
:1082900030B505460020034600E05B1C934205D242
:1082A000EC5CC85C201A01D1002CF6D130BD2DE960
:1082B000FE4F804681EA0300C00F0C46009021F07B
:1082C000004123F00045B8EB0200A94105D2404629
:1082D000214690461C460B46024623F000401043C0
:1082E00047D0270DC7F30A00C3F30A510290401A82
:1082F000019040286BDAC3F3130040F4801B009810
:10830000924620B10023D2EB030A63EB0B0B0198DA
:108310005946C0F14002504600F0BDF906460D46F0
:1083200050465946019A00F0C5F910EB080061412A
:10833000002487EA115284EAE7731A4340D0009A76
:1083400062B3019A012A4FEA075215DC001B61EB68
:1083500002014FF0004202EA0752CDE90042001C40
:1083600041F5801132462B4600F04AFA03B0BDE8D1
:10837000F08F40462146F9E7001B61EB0201001C2B
:1083800041F5801300185B412018A2F5001747EB58
:10839000030140EAD570B6196D4111E06D084FEA4E
:1083A000360645EAC0754FEA0752001B61EB020131
:1083B000001C41F5801149084FEA30000019514175
:1083C00032462B4603B0BDE8F04F00F00ABA0098E1
:1083D000012240000023D0EB020263EBE07300981F
:1083E00021464FEAE074B8EB000061EB0401E9E7D5
:1083F00083F000435BE781F0004158E72DE9FE4F31
:1084000081EA030404F0004421F0004100944FF09D
:10841000000B23F0004350EA01045ED052EA03044B
:108420005BD0C3F30A54C1F30A552C44A4F2F334CD
:108430000194A0FB0254C1F3130141F48011C3F372
:10844000130343F4801301FB024400FB034E840A30
:10845000970A44EA815447EA8357A4FB07680295C8
:108460008D0A05FB07854FEA932C04FB0C54270566
:10847000029D4FEA065847EA1637B5EB08056EEB42
:10848000070C870E920E47EA811742EA8312A7FB78
:108490000201B6EB0B0164EB00042B0D43EA0C3335
:1084A0005E1844EB1C50DA465146E7FB0201C5F367
:1084B00013044FEA0B3343EA14534FEA0432019C8E
:1084C00043EA0603A4F10C040294009CCDE900B435
:1084D00000F096F903B0BDE8F08F00200146F9E7FF
:1084E0002DE9F04D81EA030404F0004B21F0004532
:1084F00014464FF0000A23F0004150EA050220D054
:1085000054EA01021DD0C5F30A570246C5F313030E
:10851000C1F31300C1F30A5640F4801543F48013ED
:10852000A7EB0608101BD64608F2FD3873EB0500D2
:1085300002D308F1010801E092185B41B8F1000F85
:1085400003DA00200146BDE8F08D00204FF48011D1
:10855000064684460EE0171B73EB050705D3121B76
:1085600063EB050306434CEA010C49084FEA30006F
:1085700092185B4150EA0107EDD152EA030012D094
:1085800082EA040083EA0501084305D0101BAB41D1
:1085900006D20122002306E000224FF0004302E051
:1085A0006FF0010253101AEB06004CEB085110EB70
:1085B0000A0041EB0B01BDE8F04D00F012B90EB519
:1085C00040F2334102910021CDE900110A460B46E9
:1085D00000F016F903B000BD0EB540F2334202922E
:1085E0000022CDE90022134600F00AF903B000BDD5
:1085F00070B5C1F30A5201F000450024C1F3130124
:1086000040F2FF3341F480119A4201DA002070BD3C
:1086100040F233439A42A2F2334203DC5242FFF764
:1086200002FE00E090402C43F1D0404270BDC1F307
:108630000A52C1F3130140F2FF3341F480119A4210
:1086400002DA00200146704740F233439A42A2F218
:10865000334202DC5242FFF7E6BD00F01CB801F0E5
:10866000004330B421F0004150EA010206D00A0D67
:10867000A2F56072C1F31301002A02DC30BC0020B5
:108680007047440F44EAC104C100E01830BC00EB5D
:10869000C25000F06FB8202A04DB203A00FA02F141
:1086A000002070479140C2F1200320FA03F31943E0
:1086B00090407047202A06DBCB17203A41FA02F09F
:1086C00043EAE07306E041FA02F3D040C2F120022F
:1086D00091400843194670470FB4002300B589B094
:1086E0000CA900910B996FF00042CB601E4B0693D2
:1086F0001E4B07930423CDE901321D4A089202461E
:108700006B46002000F0B6F909B05DF814FB70B5B7
:1087100086B006464FF0FF300091CDE90101002000
:1087200015460C4604903246694604A8FFF7D4FF6C
:1087300002460498211825B108B1084600E02046F9
:108740002860049800280DD0002A02DD0098884295
:1087500008D0081B0094CDE901043246694604A8FC
:10876000FFF7BAFF06B070BDAD8C0008CB8C0008D7
:10877000418900080029A8BF7047401C490008BF74
:1087800020F00100704710B4B0FA80FC00FA0CF041
:1087900050EA010404BF10BC704749B1CCF1200479
:1087A00021FA04F411FA0CF118BF01212143084306
:1087B000A3EB0C01CB1D4FEA00614FEA102042BF32
:1087C000002010BC704700EBC35010440029A4BF28
:1087D00010BC7047401C490008BF20F0010010BCCD
:1087E000704710B5141E73F1000408DA401C41F103
:1087F000000192185B411A4301D120F0010010BD25
:108800002DE9F04D92469B4611B1B1FA81F202E09A
:10881000B0FA80F220329046FFF73DFF04460F4643
:1088200040EA0A0041EA0B0153465A46084313D076
:10883000114653EA010019D0C8F140025046FFF733
:10884000F2FC05460E46504659464246FFF723FFC6
:10885000084305D0012004E020463946BDE8F08DEC
:108860000020054346EAE0762C4337430A98630527
:10887000E40AA0EB08000022FD0A44EA47540A304B
:1088800002D500200146E9E7010510196941DDE93B
:10889000084500196941BDE8F04DA2E770B521F027
:1088A000004303430CD0C1F30A550024D5EB040563
:1088B00064EB0403D617AD1AB34102DB0020014676
:1088C00070BD201841EB025170BD0EB5C10F80EA9A
:1088D000E0700844CA07002140F233438DE80E00DF
:1088E0000A460B46FFF78CFF03B000BD30B5041EEF
:1088F00071F1000404DB4FF00044404264EB0101DD
:10890000141E73F1000405DB1C464FF00043524275
:1089100063EB0403994208BF904230BD064C074DFB
:1089200006E0E06840F0010394E80700984710343F
:10893000AC42F6D3FFF72CFCD8B50108F8B5010816
:10894000C0B24FF4F05100F03BBA00002DE9FF4FE8
:10895000087883B09946FF2805D0491C2D2804D0FB
:108960000024002008E000200BE00124F9E700EBE0
:10897000800003EB4000491C0B78FF2BF7D104B1BA
:10898000404200230293147819461D462D2C01D035
:108990002B2C04D1521C2D2C13D000240294AA4657
:1089A0001478FF2C0FD00A25A3FB057801FB058165
:1089B0004FF0000C03FB0C11521CE3194AEB0101B0
:1089C000EEE70124EAE7814453EA010002D019F5F9
:1089D000C87F06DA03980021C0E9001107B0BDE89E
:1089E000F08F0025AE4E2F46DFF8B8821846FFF70D
:1089F000F3FDCDE90001B9F1000002DAC9F100048C
:108A000000E004460023A74A1AEB030B42EB045A8A
:108A100012E0E00707D02A46334638464146FFF7C2
:108A2000EDFC074688462A46334610461946FFF7AE
:108A3000E5FC05460E466410002CEAD1DDE9000194
:108A4000B9F1000F5A46534606DAFFF749FD3A4698
:108A50004346FFF745FD05E0FFF7D0FC3A464346A5
:108A6000FFF7CCFC029A0AB181F00041039AC2E9F7
:108A70000001B3E72DE9FF4F1F468DB0D7E901464E
:108A80004FF0FF382E2045464FF000090B90B96992
:108A90006D1C0E988847396A824688470028F6D1AF
:108AA000BAF1FF3F0AD024F4D064002E11DDBAF1F0
:108AB0002B0F08D0BAF12D0F0BD102E0404611B0B8
:108AC0008DE744F48064B9696D1C0E98884782462E
:108AD000761E6946600501D52D2000E02B208DF81B
:108AE000000001F1010B0DF1200809E0B9696D1CCE
:108AF0000E98884782460F9844F40074761E0560ED
:108B0000002E02DDBAF1300FF0D00B998A453ED12C
:108B100044F0800406E00F99681CA9F1010944F4AF
:108B200000740860B9696D1C761E0E9888478246ED
:108B30003028F0D02BE00B998A4505D1200603D4CC
:108B400044F08004761E18E050460FF069FD08B32B
:108B50000DF11301761E44F400748B4508D2AAF17E
:108B600030000BF8010B200607D5A9F1010003E046
:108B7000200602D409F101008146A00502D50F9913
:108B8000681C0860B9696D1C0E9888478246002EE3
:108B9000D1DC53E0002E51DDBAF1650F02D0BAF1FD
:108BA000450F4BD1A00549D5B9696D1C24F440741B
:108BB000761E0E9888478246002E0CDD2B2804D0A6
:108BC000BAF12D0F07D144F48074B9696D1C0E9869
:108BD00088478246761EE00501D52D2100E02B2135
:108BE00008F8011BCDF82C8021E00DF12901761E3B
:108BF00044F4007488450CD2AAF1300010F0FF0054
:108C000088F8000002D10B99884509D908F10108BC
:108C100006E0E00501D5244801E042F20F708146EC
:108C2000B9696D1C0E98884782460F980560002E22
:108C300004DD50460FF0F4FC0028D6D1F9690E98F7
:108C40008847FF208BF8000088F80000002006907D
:108C500007904B466A4608A906A8FFF777FEA005CD
:108C600002D46FF001002AE714F0240F0AD0E007C5
:108C700014D1DDE906123868031D3B600068C0E9C5
:108C800000120BE0DDE90601FFF7E9FC0146E00711
:108C900004D13868021D3A600068016028460EE77A
:108CA000000014400000F03FF1D8FFFF426842B1DD
:108CB000016811F8013B23B1521EC0E900121846A9
:108CC00070470121C160881E704742685AB1C3686D
:108CD000016843B983688B4205D0491E521CC0E924
:108CE0000012002070474FF0FF3070472DE9F04D23
:108CF00000231A461B1A8A4103DB00200146BDE807
:108D0000F08DC1F30A52C1F3130141F480154FF005
:108D1000000BD10702D100186D41521E00270446F6
:108D200040F2FF11384601EB620A3E468046024699
:108D300000204FF48011FFF776FAC2197141BB1879
:108D400046EB0100B4EB030C75EB000C04D3E41A02
:108D500065EB000517460E46241908F101006D4128
:108D600080463428E3DDF91946EB0600091BA841CB
:108D700003D24FF0FF32134601E0002213461BEBF3
:108D8000070046EB0A51BDE8F04DFFF72ABD000091
:108D900030B5041E71F1000404DB4FF00044404282
:108DA00064EB0101141E73F1000405DB1C464FF057
:108DB0000043524263EB04038B4208BF824230BD42
:108DC0007F2801D9002208E0064A02EB5002C007C2
:108DD000127800D1120902F00F02012090400840E1
:108DE0007047000098B5010870B58C1810F8015B49
:108DF00015F0070301D110F8013B2A1106D110F834
:108E0000012B03E010F8016B01F8016B5B1EF9D137
:108E10002B0705D40023521E0DD401F8013BFAE7BD
:108E200010F8013BCB1A921C03E013F8015B01F828
:108E3000015B521EF9D5A142D8D3002070BD027843
:108E400003E010F8013B1A44D2B2491E89B2F8D2AD
:108E50001046704770B5ADF5287D00260D46ADF87B
:108E60009462ADF8986200EB40012D4800EBC1041C
:108E7000608AA84251D9ADF898624AE0A089228A56
:108E8000284481B2274800F0B1F8ADF894626A46F0
:108E9000208A0BE0BDF894326168C95CBDF8943259
:108EA000D154BDF89412491CADF89412BDF8941237
:108EB0008842EFD8401E81B21046FFF7C0FF1A4922
:108EC0008870228A0DF1FF31515C814219D1ADF8D1
:108ED00094620CE0BDF894126068BDF89422405C86
:108EE000A1688854BDF89402401CADF89402208A11
:108EF000BDF89412401E8842ECDC01200DF5287D5F
:108F000070BD64200FF0C4FDBDF89802401CADF8A0
:108F10009802BDF898020628B0D30020EEE70000C2
:108F2000A4940108FC6500201E100020F0B50D4639
:108F3000064600EB46011C48002200EBC104ADF5DB
:108F4000257D608AA8422BD9694606E0A06863683F
:108F5000805C98548854521C92B2208A401E9042E1
:108F6000F4DC208A401E81B26846FFF768FF228A3F
:108F70000DF1FF3100275054A089228A284481B284
:108F8000684600F02FF929463046FFF763FF0128B5
:108F900007D064200FF07CFD7F1CBFB2062FEBD3FF
:108FA00000200DF5257DF0BDA494010838B50025FD
:108FB000ADF800500CF0AAF80A4C207000F088F8C8
:108FC00020780949242807D0272808D0282802D14A
:108FD000022081F8650038BD81F8655038BD012058
:108FE000F7E700001E100020D41000202DE9F0410A
:108FF000064615460C46012080F31088254F0020B8
:10900000B8800CF063F8000609D401200FF040FD91
:10901000B888401C80B2B880C828F2D335E0B88840
:10902000C82832D21C4F1021384601F09EF9082181
:10903000384601F09CF9E82000F030F8C4F38710BE
:1090400000F02CF8A006000E00F028F8002000F038
:1090500025F80024002000F021F8641CA4B2042CA0
:10906000F8D3002405E0FF2000F018F83055641C08
:10907000A4B2AC42F7D31021384601F078F90020B1
:1090800080F310880120BDE8F081002080F3108873
:10909000F9E700001E1000200000024070B50B4CE4
:1090A0000546022120460CF02BF90028F9D029466C
:1090B00020460CF02EF9012120460CF021F9002861
:1090C000F9D020460CF023F9C0B270BD0030014049
:1090D00010B5012080F310881A4C0020A0800BF0FE
:1090E000F5FF000609D401200FF0D2FCA088401C37
:1090F00080B2A080C828F2D320E0A088C8281DD262
:10910000114C1021204601F030F90821204601F0D1
:109110002EF93D20FFF7C2FF2A20FFF7BFFF802076
:10912000FFF7BCFFA720FFF7B9FF1021204601F091
:109130001EF9002080F31088012010BD002080F36C
:10914000108810BD1E100020000002402DE9F041E3
:1091500006460D46012080F31088204C0020A08098
:109160000BF0B4FF000609D401200FF091FCA08899
:10917000401C82B2A280C82AF2D32AE0A088C82864
:1091800027D2174F1021384601F0EFF80821384652
:1091900001F0EDF88420FFF781FF0020FFF77EFF4C
:1091A0000020FFF77BFF0020FFF778FF002404E09A
:1091B000305DFFF773FF641CA4B2AC42F8D31021FA
:1091C000384601F0D4F8002080F310880120BDE873
:1091D000F081002080F31088F9E700001E100020C5
:1091E0000000024070B50D46012181F31088114640
:1091F000FFF7ACFF002832D01B4C0020A0800BF002
:1092000065FF000609D401200FF042FCA088401C35
:1092100080B2A080C828F2D322E0A088C8281FD23C
:10922000124C1021204601F0A0F80821204601F040
:109230009EF88320FFF732FFC5F38710FFF72EFF5C
:10924000A806000EFFF72AFF0020FFF727FF1021D6
:10925000204601F08CF8002080F31088012070BDBA
:10926000002080F3108870BD1E1000200000024016
:1092700010B500231A4604E010F8014B6340521C5D
:10928000D2B28A42F8D3184610BD000010B5044689
:1092900039200FF0EBFDE0B20FF008FEC4F3072019
:1092A0000FF004FEC4F307400FF000FE200E0FF095
:1092B000FDFD4FF48051034801F059F8BDE810401E
:1092C0000DF0BCBF000402402DE9F04105461446F4
:1092D0000E463A200FF0CAFDF0B20FF0E7FD300A5B
:1092E0000FF0E4FD104F4FF480563146384601F040
:1092F0003EF8B0463E460DF0A1FF1D2811D128468C
:1093000000F0A4F807463B200FF0B0FD4146304680
:1093100001F02DF83D44002CEDD020883844208009
:10932000E9E7BDE8F0810000000402402DE9F041CA
:10933000054614460E463C200FF098FDF0B20FF0A3
:10934000B5FD300A0FF0B2FD114F4FF48056314693
:10935000384601F00CF80CB100202080B0463E46A3
:109360000DF06CFF1E2811D1284600F017F90746B2
:109370003D200FF07BFD4146304600F0F8FF3D44B4
:10938000002CEDD0208838442080E9E7BDE8F0814A
:109390000004024010B50BF0E1FD08B100F028F820
:1093A000BDE81040302000F09FB80146362000F0A4
:1093B00089B810B508B100F0A5F8BDE81040342018
:1093C00000F092B810B5044600F09CF820785C28B4
:1093D00001D02F2803D10021642000F0FBF8BDE864
:1093E0001040322000F080B8682000F04BB8000038
:1093F00010B522200FF03AFD0FF02EFD04464FF479
:109400008051024800F0B3FF204610BD0004024026
:109410002DE9F0410FF020FD06460FF01DFD054639
:109420000FF01AFD04460FF017FD07464FF4805168
:10943000054800F09CFF46EA052040EA044040EA67
:109440000760BDE8F08100000004024070B50546E9
:1094500027200FF00BFD0FF0FFFC0446260007D07D
:109460000FF0FAFC641E05F8010B14F0FF04F7D1AD
:109470004FF48051024800F07AFF304670BD000082
:109480000004024010B504460C200FF0EFFC20460B
:109490000FF00CFDBDE81040FFF7BABF10B5044651
:1094A0000A200FF0E3FC20460FF000FD0FF0D4FC83
:1094B00004464FF48051024800F059FF204610BD89
:1094C0000004024010B50C460FF0D0FC20460FF00F
:1094D000EDFC4FF48051034800F049FFBDE8104017
:1094E0000DF0ACBE0004024010B50FF0BFFC4FF40D
:1094F0008051034800F03BFFBDE810400DF09EBED8
:109500000004024070B5054601200FF0AFFC0FF0DB
:10951000A3FC432828D22B20FFF7C0FF102823D21A
:109520002F200FF0A3FC00200FF0C0FC3220FFF72B
:10953000DBFF142818D1CF20FFF7B0FF040013D0B1
:109540004C20FFF79FFF00EB04214C2000F042F875
:109550005020FFF797FF00EB0421502000F03AF86D
:109560000021702000F036F82F200FF07FFC2C78BF
:1095700006E015F8014F5C2C01D02F2C00D10024FF
:1095800020460FF093FC002CF3D1BDE870404FF45F
:109590008051014800F0EBBE0004024070B5054662
:1095A0002D200FF063FC0FF057FC0446260007D077
:1095B00028780FF07BFC641E6D1C14F0FF04F7D1BB
:1095C0004FF48051024800F0D2FE304670BD0000DA
:1095D0000004024070B505460C460D200FF046FC15
:1095E00028460FF063FCE0B20FF060FCC4F30720E4
:1095F0000FF05CFCC4F307400FF058FC200E0FF096
:1096000055FCBDE870404FF48051014800F0AFBEFA
:109610000004024070B5094DFF22134605F580761F
:1096200005E010F8014B54402A5D5A40335D491E55
:1096300089B2F6D242EA032070BD000034920108DC
:1096400070B500221346154605E010F8014BA2182C
:109650006B41491E89B20029F7D1100C40EA034042
:1096600092B2801845EB13414FEA014242EA1041A1
:1096700008186FEA000080B270BD07F0AFBC07F0B9
:109680004DBC07F01BBC07F079BC00F0A3BF0AF08B
:109690005BBD0000074A904201D2074801E005483F
:1096A0001038064A8B0001EA020101D5C1607047FB
:1096B0008160704710640240006002407D0F7D0FA2
:1096C0000029016802D041F0010101E021F001010F
:1096D000016070472DE9F043016821F0010101604C
:1096E0000021016041608160C1600161212141610F
:1096F0003C493C4A3D251039904202D18D60BDE87D
:10970000F083384A4FF474661832904201D18E606B
:10971000F5E7344A4FF474173032904201D18F602C
:10972000EDE7304A4FF0746C4832904202D1C1F8F4
:1097300008C0E4E72B4B2C4A6033984201D1CA6041
:10974000DDE7284C294B7834A04201D1CB60D6E725
:10975000DFF89080264C08F19008404501D1CC609C
:10976000CDE7DFF880804FF03D5908F1A80840456B
:1097700002D1C1F80C90C2E71E49DFF878800839A1
:10978000404501D10D60BAE71A4D1835A84201D104
:109790000E60B4E7174D3035A84201D10F60AEE737
:1097A000144D4835A84202D1C1F800C0A7E7114DB9
:1097B00010496035091FA84201D10A609FE70D4A90
:1097C0007832904201D10B6099E70A4A9032904278
:1097D00001D10C6093E7074AA83290428FD1C1F8BB
:1097E00000908CE7106002403D000020400F0020F8
:1097F00000003D20106402400B0607D5436912B1FA
:1098000043F0800301E023F080034361802908D006
:10981000002A026801F01E0101D00A4300E08A43D9
:109820000260704730B50368124ACC6813400A687A
:109830002243D1E905452C432243CC6922430C6ADB
:1098400022434C6A22438C6A22434C6B22438C6B2A
:1098500022431A430260426922F00703D1E90B2434
:1098600022431A4342610A6942604A6882608968F9
:10987000C16030BD3F801CF02DE9FC41012120205A
:109880000BF074FB01268DF8046000258DF806505E
:1098900003208DF805001A4C302700978DF80750EB
:1098A0006946204600F00EFD3021204600F05FFDA5
:1098B000144C84F8F05484F8F25484F8F16484F879
:1098C000F3644FF4FA70C4F8F80400F01DF894F84B
:1098D0006802802812D16565232084F86D02052076
:1098E00084F86C0284F86B72142084F86A022020D9
:1098F00084F8690284F8685200F048F8BDE8FC81F9
:1099000000140240D41000207CB50FF083F9D02061
:109910000FF050F90FF0B2F900200FF04BF90FF0F3
:10992000ADF90FF077F9D1200FF044F90FF0A6F957
:1099300000246D4601E0062C01D2012000E0002049
:109940000FF008F92855641CE4B2072CF3D30FF08C
:109950007BF90D489DF8061080F86D129DF80510F2
:1099600080F86C129DF8041080F86B129DF80210BC
:1099700080F86A129DF8011080F869129DF80010B5
:1099800080F868127CBD0000D41000207CB51B4814
:10999000002490F868128DF8001090F869128DF884
:1099A000011090F86A128DF8021001218DF8031051
:1099B00090F86B128DF8041090F86C128DF8051069
:1099C00090F86D028DF806000FF024F9D0200FF00A
:1099D000F1F80FF053F900200FF0ECF80FF04EF90A
:1099E0006D46285D0FF0E6F80FF048F9641CE4B20C
:1099F000072CF6D30FF028F97CBD0000D41000200E
:109A000070B5094D0022134605F5807605E010F883
:109A1000014B54402A5D5A40335D491E89B2F6D24B
:109A200042EA032070BD000034920108072A00D9E1
:109A3000072240EA002021B1012901D1D040C0B263
:109A400070479040C0F3072070477047072A00D93D
:109A5000072240EA002029B1012902D19040C0F339
:109A600007207047D040C0B27047000070B5ADF518
:109A7000327D00260D46ADF8BC62ADF8C06200EB49
:109A80004001324800EBC104608AA8425CD9ADF8BD
:109A9000C06255E0012264212D4800F0A9F92C484C
:109AA00000788DF80000382842D1228AE06802FB55
:109AB0000501274800F09CF9ADF8BC626A46208A8F
:109AC0000BE0BDF8BC326168C95CBDF8BC32D15452
:109AD000BDF8BC12491CADF8BC12BDF8BC128842DE
:109AE000EFD8401E81B2104600F044FA228A0DF1F0
:109AF000FF31515C81421BD1ADF8BC620EE0BDF874
:109B0000BC226168895CA26800FB0520BDF8BC220C
:109B10001154BDF8BC02401CADF8BC02208ABDF84F
:109B2000BC12401E8842EADC01200DF5327D70BD7A
:109B300064200EF0ADFFBDF8C002401CADF8C002BD
:109B4000BDF8C0020628A5D30020EEE7B0900108BA
:109B500020410020F0B50E46074600EB470126489D
:109B6000ADF5317D002500EBC1048DF8BC52608A53
:109B7000B0423DD900210846FFF778FF012837D1D0
:109B8000694609E0A268401E00FB06206268285C66
:109B9000505548556D1CADB2208AA842F2D8002518
:109BA000208AE16800FB0611401E82B2134800F0D3
:109BB0009DF9208A401E81B2684600F0DBF98DF8DD
:109BC000BC02208AE168012201447043401E014426
:109BD000AFA800F08BF931463846FFF747FF012860
:109BE00007D064200EF054FF6D1CADB2062DD7D304
:109BF00000200DF5317DF0BDB0900108204100201E
:109C0000F0B5ADF5317D2C4D00208DF8BC022B4E0A
:109C1000288000243FE000206F4607E056F83220FD
:109C20004968125C0A543A54401C80B2298801EBFE
:109C3000410206EBC2010B8A5B1E8342EEDC2888E0
:109C400000EB400006EBC000008A401E81B238469F
:109C500000F090F98DF8BC02288800EB400006EB7C
:109C6000C000C168008A00FB0411401E82B2144883
:109C700000F03CF92888012200EB400006EBC00010
:109C8000C168008A01446043401E0144AFA800F04F
:109C90002DF9641CA4B2288800EB400006EBC0003C
:109CA000408AA042B7D82888401C80B22880072864
:109CB000AFD30DF5317DF0BD10000020B09001084C
:109CC000204100207CB5012108460BF04FF901200E
:109CD0008DF8040002258DF8055000248DF806400B
:109CE0008DF807001820154E00906946304600F0A8
:109CF000E9FA05221146304600F020FB0522062134
:109D0000304600F01BFB05220721304600F016FB11
:109D1000A02000908DF8045003208DF805008DF8E8
:109D200006408DF807406946304600F0CBFA4020E7
:109D300000906946304600F0C5FA7CBD0000024044
:109D4000F8B5002634460096FFF7BCFF00F0A0F8F7
:109D50002248641C8442FCD3214C0821204600F098
:109D600004FB1021204600F002FB062000F076F8EC
:109D70000821204600F0FBFA0821204600F0F5FA01
:109D80001021204600F0F3FA012000F067F80020CF
:109D900000F064F80821204600F0E9FA1148D0F8F4
:109DA0001C0208B9FFF72CFF0F4D2E800F4E002428
:109DB00005E0C0B22146FFF759FE641CA4B2288812
:109DC00000EB400106EBC101498AA142F1D880B203
:109DD000401C80B228800728E9D3F8BDFFFF0F00A0
:109DE000000002400000434210000020B090010833
:109DF0002DE9F0410546002416460F46012080F368
:109E00001088DFF854800821404600F0AEFA102197
:109E1000404600F0ACFA032000F020F8C7F30740FA
:109E200000F01CF8C7F3072000F018F8F8B200F0B3
:109E300015F806E0002000F011F8641C05F8010B8D
:109E4000A4B2B442F6D30821404600F090FA0020B4
:109E500080F31088BDE8F0810000024070B50B4C23
:109E60000546022120460BF04BFA0028F9D029467E
:109E700020460BF04EFA012120460BF041FA002853
:109E8000F9D020460BF043FAC0B270BD003001405B
:109E900010B5012186B008030BF0A4F8124C20463F
:109EA0000BF004FA0021ADF808106015ADF80A00B7
:109EB0003820ADF80C000720ADF80010ADF8100008
:109EC000ADF804104FF48270ADF80610ADF80E1026
:109ED000ADF80200694620460BF01DFA012120462C
:109EE0000BF0DAF906B010BD003001402DE9F04169
:109EF0000546002416460F46012080F31088DFF83F
:109F000070800821404600F030FA1021404600F0F1
:109F10002EFA0620FFF7A2FF0821404600F027FA9C
:109F20000821404600F021FA1021404600F01FFAB7
:109F30000220FFF793FFC7F30740FFF78FFFC7F338
:109F40000720FFF78BFFF8B2FFF788FF05E02878BE
:109F5000FFF784FF641CA4B26D1CB442F7D3082140
:109F6000404600F004FA002080F31088BDE8F0813C
:109F700000000240027803E010F8013B1A44D2B21C
:109F8000491E89B2F8D210467047000070B51E4ACB
:109F9000907A012825D1002595721C491C480F2470
:109FA0004E780123F6B14D70D0F82852D0F83462C3
:109FB00045EAC605D0F83062D0F82C02B60046EA71
:109FC00040000543AC43CC708878CC78A04208D1DF
:109FD00008710C78A04204D0D0710870002800D01D
:109FE000937170BD4B70D0F82852D0F8346245EAB6
:109FF000C605D0F83062D0F82C02B60046EA400020
:10A000000543AC438C70DFE7D4100020C91000205A
:10A01000000042422DE9F041ADF57C7D00273D4630
:10A02000ADF8E873FFF7B6F95F4C142807D084F851
:10A0300067520EF057FE0DF57C7DBDE8F0815B4860
:10A04000FFF7C0F9594E103E1428307006D0422850
:10A050007ED00120FFF7A9F93570ECE7FFF7C4F9CE
:10A06000C6E90205B046BDF8E803FFF70FF9FAAA02
:10A070004FF4FA716846FFF727F94DA168460EF0D4
:10A0800095FEB0806E46D0B1E11981F8BC557F1CB9
:10A09000BFB2282FF8D34746304447A10EF086FEC2
:10A0A00078800021001F08E0BA8863180A4432440F
:10A0B000D27883F8BC25491C89B28142F4DB3FA1E8
:10A0C00068460EF073FE4746A8F80400D0B10021A0
:10A0D000621882F8E455491C89B22829F8D3304423
:10A0E00035A10EF063FE78800021093808E0BA88B7
:10A0F00063180A443244127A83F8E425491C89B271
:10A100008142F4DB30A168460EF050FEB880D0B139
:10A110000021621882F80C56491C89B21429F8D320
:10A12000304425A10EF042FE788000210D3808E071
:10A13000BA8863180A443244127B83F80C26491CFF
:10A1400089B28142F4DB24A168460EF02FFE00E0C4
:10A1500025E0B880D0B10021621882F87655491CFC
:10A1600089B23229F8D3304413A10EF01FFE788053
:10A170000021C01F08E0BA8863180A44324492796B
:10A1800083F87625491C89B28142F4DB0021032043
:10A19000FFF7E0FC0120FFF708F901204BE7034837
:10A1A000FFF707F947E70000D4100020381000201F
:10A1B00041504E3D000000003B0000005749464919
:10A1C0004E414D453D0000005749464950415353CB
:10A1D000574F52443D0000005345525645523D00F2
:10A1E0002F4910B5884206D1012108460AF0CAFE5F
:10A1F000002101204FE02B49884206D10121022095
:10A200000AF0C0FE0021022045E02749884206D11D
:10A21000012104200AF0B6FE002104203BE023497E
:10A22000884206D1012108200AF0ACFE0021082056
:10A2300031E01F49884206D1012110200AF0A2FE18
:10A240000021102027E01B49884206D1012120204F
:10A250000AF098FE002120201DE01749884206D10F
:10A26000012140200AF08EFE0021402013E0134916
:10A27000884206D1012180200AF084FE002180203E
:10A2800009E00F4988420AD18415012120460AF0CD
:10A2900079FE00212046BDE810400AF073BE10BDD3
:10A2A000000002400004024000080240000C02408E
:10A2B000001002400014024000180240001C02403E
:10A2C00000200240F0B5002201274FF0030C0B687C
:10A2D00007FA02F52B40AB422CD1066853000CFA6A
:10A2E00003F4A64306600E79D0F800E09E4046EAEB
:10A2F0000E0606600E79012E01D0022E12D186685C
:10A30000A64386604E79D0F808E09E4046EA0E06E5
:10A3100086604668AE43466045688E799640B6B220
:10A3200035434560C568A543C560CC799C40C3688A
:10A330001C43C460521C102AC9D3F0BD4B07DB0E6E
:10A340009A40C90810B500EB8100016A0F249C40B7
:10A35000A1430162016A1143016210BD024600205F
:10A3600012690A4200D0012070474183704701837F
:10A37000704700002DE9F04F754800252DED028B48
:10A3800085B001782C4601294FD1002682460670FF
:10A3900000F1020898F80000DFF8B8918B46F52824
:10A3A00004D098F819004F2874D077E098F802008C
:10A3B00098F8011040EA012465482146801CFFF707
:10A3C00029F908EB0401497818F8042041EA022130
:10A3D00081422AD198F803105F4FF1292AD05F48B3
:10A3E000F2294BD0F32920D180F8486080F83CB0A6
:10A3F000F52038707E700520B870F320F870592071
:10A40000387105215448FFF705F9010A7971B871CF
:10A410005348076052490720083908605048012115
:10A420000C38FFF74DF98AF8016005B0BDEC028BDE
:10A43000BDE8F08F4946481980F8BC656D1CADB287
:10A44000282DF8D30020241F07E008EB0002127922
:10A450000B1883F8BC25401C80B2A042F5DB00211C
:10A460000320FFF777FB0028DFD009F0C9FFF520B4
:10A4700038707E700520B870F120BFE780F848B0D2
:10A4800080F83DB0F52038707E700520B870F2205D
:10A49000B4E7FFE798F81A004B281AD02C4831A1EE
:10A4A000801C0EF083FC050002D0022189F8021006
:10A4B00008EB0507B87B41280ED0B87B5628B4D1ED
:10A4C000C9F8396689F83D66C9F8396689F83D6684
:10A4D000ABE789F802B0A8E76E46291901EB08003E
:10A4E000007C3055641CA4B2092CF6D330460CF025
:10A4F000E3FE51EC100BFEF7B2F800EE100A9FEDF0
:10A500001A8A1A484146C0EE080AC0ED8D0AB87E84
:10A510004C4689F8380600202A180A44127F325423
:10A52000401C80B20928F7D368460CF0C5FE51ECF8
:10A53000100BFEF794F800EE100AC0EE080A10EEB9
:10A54000900AC4F8390697F8270084F83D066CE7AE
:10A5500012000020D4100020FC030020D440002072
:10A56000AC640240524D43000000C842D4140020A5
:10A5700070B5144C40F22446314620460CF0D1FD13
:10A5800000281ED0314620460CF068FD0E4D0021FB
:10A590002846FFF795F8314620460CF05FFD0B4941
:10A5A0002846FFF777F82088201D0088291D4FF4E2
:10A5B0007A70086001212846FFF782F804490120DB
:10A5C000087070BD0014014028640240008800102B
:10A5D0001200002010B5104C0E492046FFF75AF823
:10A5E00000212046FFF76CF80C4C402120460CF06F
:10A5F00091FD0028F9D0084C0949783C2046FFF726
:10A6000049F801212046FFF75BF806490120487010
:10A6100010BD000000802020A06402400014014012
:10A6200000880010120000202DE9F04301218FB0B6
:10A6300088050AF09BFCDFF88C904846FFF74AF843
:10A640004020050103900024CDE90545C60207948A
:10A650000894CDE909461C4F0B944FF02068CDE9D2
:10A6600000870C940D94694648460E94FFF7DAF87B
:10A67000012210214846FFF7BFF8DFF84890A9F102
:10A6800078094846FFF726F84FF47A70CDE9034081
:10A69000CDE9054507940894CDE909460B480B948C
:10A6A0000C940D94CDF800800E94CDE901706946AC
:10A6B0004846FFF7B7F801214846FFF701F80FB009
:10A6C000BDE8F083A064024004140140140000209F
:10A6D0007CB5012104200AF049FC164E082206210F
:10A6E0003046FFF72BFE082207213046FFF726FEF3
:10A6F00002218DF8051000258DF806500124C02098
:10A700008DF8074000908DF8041069463046FFF739
:10A71000D9FD600200908DF804408DF806500320AA
:10A720008DF805008DF8074069463046FFF7CAFDF1
:10A730007CBD0000000802402DE9F047FFF7C8FF8C
:10A740004FF4E13000F07AF8FFF76EFF00F058F8B0
:10A75000264D002685F8286685F82A66012085F8AA
:10A76000290685F82B0642F21070C5F83006214FF5
:10A770001F483860DFF87C800E21A8F10808C8F86F
:10A780000010A8F1040901214846FEF799FF1A4C70
:10A79000667060780028FCD04FF4FA700EF078F9FB
:10A7A0004FF4165000F04AF811490020134A1031B6
:10A7B00001EB000C135C401CC0B28CF808300A2876
:10A7C000F6D300202A1892F8B8250B18401CC0B206
:10A7D000DA740428F6D339601921C8F80010012171
:10A7E0004846FEF76DFF6670BDE8F087D410002084
:10A7F000E4070020AC64024012000020BC8E010877
:10A8000038B545208DF8000002208DF801000124A4
:10A810008DF802408DF80340684607F0FBF84720AA
:10A820008DF800008DF8014000208DF802008DF8B1
:10A830000340684607F0EEF838BD00001FB5044637
:10A84000012120200AF0CEFB0020ADF80400009486
:10A85000ADF80600ADF80800ADF80C000C200D4C6A
:10A86000ADF80A00694620460CF092FC0121204612
:10A870000CF0F7FB012240F2244120460CF070FC62
:10A88000102120460CF0EAFB0122C02120460CF0EA
:10A89000F2FB1FBD001401400249C8790022CA71B1
:10A8A00070470000D410002002480068C00700D0A4
:10A8B00000BEFEE7F0ED00E002494AF6AA2008607B
:10A8C000704700000030004010B50EF00BFABDE8F4
:10A8D000104064200EF0DCB82DE9F04F83466BA0E9
:10A8E000ADF57D7D002400689A460E462746FB9014
:10A8F000ADF8E843042A26D8DFF8949199F86C1251
:10A9000002EBC20505EB0215624A3023154403EB46
:10A910001111297199F86C1201F00F013031697130
:10A9200099F86B1203EB1111A97199F86B0200F001
:10A930000F003030E871FEF72DFD142807D089F89C
:10A9400067720EF0CFF90DF57D7DBDE8F08FDFF871
:10A950004481A8F1240898F8000014280ED0284655
:10A96000FEF730FD88F80000142807D042287DD07B
:10A970000120FEF71AFD88F80070E4E74FF47A70C2
:10A98000864200D90646FEF72FFD4546C5E9020777
:10A99000FEF77CFC99F86B224846302101EB12123D
:10A9A0008DF8002099F86B2202F00F0230328DF8FA
:10A9B000012099F86A2201EB12128DF8022099F811
:10A9C0006A2202F00F0230328DF8032099F86922D2
:10A9D00001EB12128DF8042090F8692202F00F02A8
:10A9E00030328DF8052090F8682201EB12118DF8B5
:10A9F000061090F8680200F00F0030308DF8070064
:10AA0000BAF1000F03D0BAF1010F02D004E05420D4
:10AA100000E052208DF808003A208DF809000A2342
:10AA2000EC4618E00BEB540210780009B0FBF3F190
:10AA3000C1EBC10108440CEB04013030887210787E
:10AA400000F00F00B0FBF3F2C2EBC2021044303052
:10AA5000A41CC872A4B2B4EB460FE3D303EB4600C8
:10AA600081B2FAAA6046FEF761FC00E009E0FAAAAA
:10AA70000221FBA8FEF75AFC0120FEF796FC2F707E
:10AA800061E72846FEF795FC5DE700000D0A00002F
:10AA9000D41000204C1000202DE9F04F00252DEDA2
:10AAA000028B99B08DF838508DF85C508DF8545069
:10AAB000CDE91255CDE900558DF808508DF80C50B0
:10AAC0008DF810508DF81450ADF818509FEDFD0A18
:10AAD000FD488DED0D0A00F5005725300124DFF803
:10AAE000ECA34FF0A30BD526DFF8E4830790A4E096
:10AAF000DFF8D49399F8720928B389F87259B7F836
:10AB0000F81FDAF88C205046C2F57A7291421AD1B9
:10AB1000D0F88C00C0F57A70A7F8F00FEB48002150
:10AB20008830FEF7CDFDE948EA498830FEF7B2FDEE
:10AB300088F800404FF47A70CAF88C00E34801218D
:10AB40008830FEF7BDFD99F87E0920B389F87E595B
:10AB5000B7F8FA1FDAF844205046C2F57A729142EB
:10AB600019D1406CC0F57A70A7F8F20FD7480021D0
:10AB70004030FEF7A5FDD548D7494030FEF78AFDA5
:10AB800088F801404FF47A70CAF84400CF48012198
:10AB90004030FEF795FD99F88A0920B389F88A5963
:10ABA000B7F8FC1FDAF814205046C2F57A729142C9
:10ABB00019D14069C0F57A70A7F8F40FC348002195
:10ABC0001030FEF77DFDC148C4491030FEF762FD2C
:10ABD00088F802404FF47A70CAF81400BB4801218B
:10ABE0001030FEF76DFD99F89619484629B380F8A4
:10ABF0009659B7F8FE1FDAF82C205046C2F57A7243
:10AC000091421AD1C06AD146C0F57A70A7F8F60F02
:10AC1000AE4800212830FEF753FDAC48B04928303B
:10AC2000FEF738FD88F803404FF47A70C9F82C001D
:10AC3000A64801212830FEF743FDA34890F8721979
:10AC400090F87E29114490F88A2990F896091044CA
:10AC5000C1427FF44DAF04F04DBF017819B10570CA
:10AC60008DF8085010E0417819B145708DF8084012
:10AC70000AE0817811B18570022003E0C17819B132
:10AC8000C57003208DF808009DF80800DFF83882B1
:10AC900000EB400101EB001008EB001090F8161AD1
:10ACA0009DF80800DFF83CA200EB4002C2EBC012A6
:10ACB0001AF83200C1280AD19DF8080000EB4002C2
:10ACC000C2EBC0120AEBC200807808280CD0082919
:10ACD00084F0DC86DFE811F0D6192800AC087A1081
:10ACE00004187D19B91CE21F7F4880F848409DF880
:10ACF000080030B1012807D002280FD0032808D15E
:10AD00000FE04FF4804101E04FF400517748FFF726
:10AD10002CFB7748C0F8885204F0B8BE4FF480513D
:10AD2000F4E74FF40061F1E79DF8080000EB400103
:10AD3000C1EBC0110AEBC1004078002105F0F2FF21
:10AD40008DF810008DF85450C14619E09DF80800A8
:10AD500000EB400101EB00109DF8541009EB0010CE
:10AD600000EB011090F8410A9DF8101088429DF800
:10AD7000540002D18DF8100010E0401C8DF85400F2
:10AD80009DF8080000EB400101EB001009EB0010FA
:10AD900090F8170A9DF854108842D7D89DF80800FB
:10ADA00000EB4001C1EBC0100AEBC00080780A2222
:10ADB000B2EB101F9DF8080000EB4002C2EBC01080
:10ADC0000AEBC000807801D100F00F008DF80C0074
:10ADD0009DF80C0010B910208DF80C009DF80800AB
:10ADE0009DF80C1000EB4002C2EBC01257460AEB74
:10ADF000C20008444078ADF818009DF8080000EB48
:10AE00004001C1EBC0110AEBC1009DF80C10491CB8
:10AE100006F06BFB8DF85C009DF8080000EB40012C
:10AE2000C1EBC01107EBC1009DF80C1008448078FD
:10AE30009DF85C10884244F029869DF8080000EBDC
:10AE40004001C1EBC01107EBC10138464978002928
:10AE500004F01C869DF8081001EB4102C2EBC11101
:10AE600000EBC1029DF80C101144CA789DF808103F
:10AE700001EBC10303EB012109EBC1039DF81010A5
:10AE800001EB411103EB810181F8142F9DF80810AB
:10AE900009EB01129DF81010114481F8D059BDF84A
:10AEA0001810CE292DD02DDCB9297DD022DC5A29CD
:10AEB000CED0B22904F06083B529F6D0B629BAD134
:10AEC000FEE3000000000000D410002000600240FB
:10AED0000F08002000880020008020102080001033
:10AEE000008800106C4E0020D44000200018024062
:10AEF00000004242C32904F00583C5297DD0CA2938
:10AF000099D1E4E3E129FCD003F3AB87D52908D03C
:10AF1000D7299DD0D9298ED17CE2E7298BD104F0A5
:10AF2000D1BD9DF8081001EB4102C2EBC11107EB46
:10AF3000C100C07889F862009DF8080000EB40016C
:10AF400001EB00109DF8101009EB001000EB011050
:10AF500099F86210A4EBD11290F8421A62F3000142
:10AF600080F8421A9DF8080000EB400101EB001048
:10AF70009DF8101009EB001000EB011099F8621019
:10AF80004A0990F8421A62F3410180F8421A9DF88A
:10AF9000080000EB400101EB00109DF8101009EBD8
:10AFA000001000EB011000E0E3E390F8420AC0F368
:10AFB00040019DF8080000EBC00202EB00209DF864
:10AFC000102009EBC00002EB421200EB820090F867
:10AFD000F00EC0F3400081424BD09DF8080000EB1A
:10AFE000C00101EB002009EBC0029DF810004946AA
:10AFF00000EB401002EB800000E0FDE39DF808202C
:10B0000002EB420303EB02129DF8103009EB02122F
:10B0100002EB031292F8422A530890F8F02E63F3E1
:10B02000410280F8F02E9DF8080000EB400202EB90
:10B0300000109DF8102001EB001000EB021090F8BA
:10B04000420A800716D59DF80800D92200EBC003FC
:10B0500003EB002009EBC0019DF8100000EB40104D
:10B0600001EB800080F8DC2E9DF808100220FEF72E
:10B0700071FD42E09DF8080000EBC00202EB0020E9
:10B0800001EBC0029DF8100000EB401002EB8000C5
:10B0900080F8E54E9DF80800D92200EBC00303EBD1
:10B0A000002001EBC0039DF8100000EB401003EB03
:10B0B000800080F8DC2E9DF8080000EB400202EBD7
:10B0C000001001EB00129DF8100002EB001292F844
:10B0D000420A20F0200382F8423A9DF8080000EB73
:10B0E000C00202EB002009EBC0019DF8100000EB4C
:10B0F000401001EB800080F8164F9DF8080000EB2F
:10B10000400101EB001009EB00119DF8100001EB6C
:10B11000001090F8420A00F001019DF8080000EBD1
:10B12000C00202EB002009EBC0029DF8100000EB0A
:10B13000401002EB800090F8F00E00F00100814218
:10B1400004F0E8809DF8080000EBC00101EB00204E
:10B1500009EBC0019DF8100000EB401001EB8000EE
:10B160009DF8081001EB410202EB01119DF810203F
:10B1700009EB011101EB021191F8421A90F8F02E3F
:10B1800061F3000280F8F02E9DF8080000EB40010A
:10B1900001EB001009EB00119DF8100001EB00100D
:10B1A00090F8420AC00739D09DF808004F4600EBDE
:10B1B000C00101EB002009EBC0019DF8100000EB7D
:10B1C000401001EB800090F8160F00289DF8080051
:10B1D00000EBC00101EB002009EBC0019DF810005D
:10B1E00000EB401001EB80003BD080F8155F9DF82C
:10B1F000080000EB400101EB001007EB00119DF887
:10B20000100001EB001191F8420A20F0010281F8D0
:10B21000422A97F8210638B304F07CB89DF808005C
:10B2200000EB400101EB00109DF8101009EB00103D
:10B2300000EB011090F8421A21F0200180F8421A28
:10B240009DF8080000EBC00101EB002009EBC001F4
:10B250009DF8100000EB401001EB800080F8155FB6
:10B26000DAE780F8154FD4E7387D0128D4D1786D1E
:10B27000F98A8842D0D29DF8080000EBC00101EBAA
:10B28000002007EBC0019DF8100000EB401001EB1F
:10B29000800090F8150F0128BED19DF8080000EB42
:10B2A000C00101EB002007EBC0019DF8100000EB8E
:10B2B000401001EB800090F8490F0028ACD19DF8B8
:10B2C000080000EB400101EB001007EB00119DF8B6
:10B2D000100001EB001090F8401A9DF8080000EBF8
:10B2E000C00202EB002007EBC00080F8D11E9DF8E1
:10B2F0000800C32100EBC00202EB002007EBC002F4
:10B300009DF8100000EB401002EB800080F8DC1E7E
:10B310009DF8080000EB400101EB001007EB001165
:10B320009DF8100001EB0010C0F8445A9DF8081079
:10B330000220FEF70FFC8DF8385017E09DF808004A
:10B3400000EBC00101EB002007EBC0019DF81000ED
:10B3500000EB401001EB80019DF83800084480F8B4
:10B36000175F9DF83810491C8DF838109DF838008B
:10B370001428E3D38DF8385017E09DF8080000EB4F
:10B38000C00101EB002007EBC0019DF8100000EBAD
:10B39000401001EB80009DF83810084480F8335FBE
:10B3A0009DF83800401C8DF838009DF838000A28B8
:10B3B000E3D331E79DF8080000EBC00101EB00206A
:10B3C00009EBC0019DF8100000EB401001EB80007C
:10B3D00090F8D80E012844F059839DF8080000EB3E
:10B3E000C00101EB002009EBC00080F8D35E9DF89E
:10B3F0000800022100EBC00202EB002009EBC002B2
:10B400009DF8100000EB401002EB800080F8D81E81
:10B41000B62140E29DF8081001EB410202EB011158
:10B4200009EB011191F81C1A00299DF80C1002D0AB
:10B430000A29D0D191E00829CDD18DF8385024E0E7
:10B440009DF8081001EB4102C2EBC1119DF83820B4
:10B4500000EBC1011144C97801F00F01092918D886
:10B460009DF8081001EB4102C2EBC1119DF8382094
:10B4700000EBC1011144C97801F0F001902908D80E
:10B480009DF83810491C8DF838109DF838100629A1
:10B49000D6D39DF838100629C4F0F8829DF808101C
:10B4A00001EB4102C2EBC11100EBC101C9780B04F1
:10B4B0009DF8081001EB4102C2EBC11100EBC10184
:10B4C00009799DF8082043EA012102EB4203C3EB0E
:10B4D000C21200EBC202527911439DF8082002EB20
:10B4E000C20303EB022209EBC2039DF8102002EB1A
:10B4F000421203EB8202C2F8F11E9DF8081001EB24
:10B500004102C2EBC11100EBC10189790B049DF826
:10B51000081001EB4102C2EBC11100EBC101C97976
:10B5200043EA01239DF8081001EB4102C2EBC1116F
:10B5300000EBC100007A03439DF8080000EBC00156
:10B5400001EB002009EBC0019DF8100000EB40105A
:10B5500001EB8000C0F8F53E95E08DF8385024E00E
:10B560009DF8081001EB4102C2EBC1119DF8382093
:10B5700000EBC1011144C97801F00F01092918D865
:10B580009DF8081001EB4102C2EBC1119DF8382073
:10B5900000EBC1011144C97801F0F001902908D8ED
:10B5A0009DF83810491C8DF838109DF8381008297E
:10B5B000D6D39DF838100829C4F068829DF8081089
:10B5C00001EB4102C2EBC11100EBC1018A799DF888
:10B5D000081001EB4103C3EBC11100EBC101C978B5
:10B5E00042EA01629DF8081001EB4103C3EBC1116F
:10B5F00000EBC10109790B049DF8081001EB41072C
:10B60000C7EBC11100EBC101497943EA01210A43AB
:10B610009DF8081001EBC10303EB012109EBC10305
:10B620009DF8101001EB411103EB8101C1F8F12EDF
:10B630009DF8081001EB4102C2EBC11100EBC10102
:10B640008A7A9DF8081001EB4103C3EBC11100EBAE
:10B65000C101C97942EA01629DF8081001EB41037A
:10B66000C3EBC11100EBC101097A0B049DF808106E
:10B6700001EB4107C7EBC11100EBC100407A43EA7F
:10B68000002003F0FDBE9DF8080000EBC00101EBB7
:10B69000002009EBC0019DF8100000EB401001EB09
:10B6A000800090F8D80E03289DF8080010D000EB19
:10B6B000400101EB001009EB00109DF8101000E0B4
:10B6C00063E000EB011090F8420A80072DD51AE0E4
:10B6D00000EBC00101EB002009EBC00080F8D35E55
:10B6E0009DF80800042100EBC00202EB002009EBEA
:10B6F000C0029DF8100000EB401002EB800080F8C3
:10B70000D81EC521C7E09DF8080000EBC00101EB81
:10B71000002009EBC0019DF8100000EB401001EB88
:10B72000800080F8DC6E04F0B1B99DF8080000EBF1
:10B73000C00101EB002009EBC0019DF8100000EBF7
:10B74000401001EB800090F8E60E0128EBD19DF847
:10B75000080000EBC00101EB002009EBC0019DF8DF
:10B76000100000EB401001EB800080F8E65EB6218F
:10B770005CE09DF8080000EBC00101EB002009EB44
:10B78000C00080F8D35EC32185E09DF8081001EB6E
:10B79000410202EB011109EB011191F81C1A002979
:10B7A0009DF8081001EB4102C2EBC11100EBC10191
:10B7B00003F0D486C9780A049DF8081001EB410310
:10B7C000C3EBC11100EBC101097942EA01229DF8E6
:10B7D000081001EB4103C3EBC11107EBC100407935
:10B7E00002439DF8080000EBC00101EB002009EBCB
:10B7F000C0039DF8100000E064E000EB401003EB94
:10B800008000C0F80C2F9DF8080000EBC00101EB90
:10B81000002009EBC0019DF8100000EB401001EB87
:10B82000800090F8D80E022819D0C5219DF8080094
:10B8300000EBC00202EB002009EBC0029DF81000F3
:10B8400000EB401002EB800080F8DC1E9DF8080041
:10B8500000EBC00101EB002009EBC0002CE09DF8DB
:10B86000080000EBC00101EB002009EBC00080F8EC
:10B87000D35E9DF80800032100EBC00202EB00201C
:10B8800009EBC0029DF8100000EB401002EB8000B5
:10B8900080F8D81ED9219DF8080000EBC00202EB09
:10B8A000002009EBC0029DF8100000EB401002EBF5
:10B8B000800080F8DC1E36E780F8D35E33E780F83E
:10B8C000422A30E79DF8081001EB410202EB01111A
:10B8D00009EB011191F81C1A00299DF80C1002D0F7
:10B8E0000E29E8D19BE00C29E5D18DF8385024E0F1
:10B8F0009DF808109DF8383001EB4102C2EBC111F0
:10B9000000EBC102D118C97801F00F01092918D83C
:10B910009DF8082002EB4203C3EBC21100EBC10209
:10B920009DF838101144C97801F0F001902908D829
:10B930009DF83810491C8DF838109DF838100A29E8
:10B94000D6D39DF838100A29B5D30022CDE90022BC
:10B95000134629468DF838501EE0009A1B0243EA30
:10B9600012631202CDE900239DF8082002EB420386
:10B97000C3EBC2129DF8383000EBC2021A44D278F1
:10B98000DDE900371A4341EA0703CDE900239DF8BA
:10B990003820521C8DF838209DF83820052ADCD339
:10B9A000DDE900379DF8082002EBC20C0CEB022207
:10B9B00009EBC20C9DF8102002EB42120CEB820244
:10B9C000C2F8F93EC2F8FD7E0023CDE900338DF8C0
:10B9D00038101FE0DDE900231B0243EA1263120264
:10B9E000CDE900239DF8082002EB4203C3EBC2120D
:10B9F0009DF8383000EBC2021A44127ADDE90037B4
:10BA00001A4341EA0703CDE900239DF83820521C70
:10BA10008DF838209DF83820052ADBD39AE08DF880
:10BA2000385024E09DF808109DF8383001EB4102B1
:10BA3000C2EBC11100EBC102D118C97801F00F01AE
:10BA4000092918D89DF8082002EB4203C3EBC21164
:10BA500000EBC1029DF838101144C97801F0F001E3
:10BA6000902908D89DF83810491C8DF838109DF899
:10BA700038100C29D6D39DF838100C29C4F0068054
:10BA80000022CDE9002229468DF83850BC461FE03F
:10BA9000DDE90002120242EA10620002CDE9000272
:10BAA0009DF8080000EB4002C2EBC0109DF8382062
:10BAB0000CEBC0001044C078DDE90023104341EADC
:10BAC0000302CDE900029DF83800401C8DF83800D3
:10BAD0009DF838000628DBD3DDE900239DF8080037
:10BAE00000EBC00707EB002009EBC0079DF8100032
:10BAF00000EB401007EB8000C0F8F92EC0F8FD3EC7
:10BB00000022CDE900228DF838101FE0DDE90002A7
:10BB1000120242EA10620002CDE900029DF808001C
:10BB200000EB4002C2EBC0109DF838200CEBC000C7
:10BB30001044407ADDE90023104341EA0302CDE9D5
:10BB400000029DF83800401C8DF838009DF8380040
:10BB50000628DBD3DDE900129DF8080000EBC003E6
:10BB600003EB002009EBC0039DF8100000EB401030
:10BB700003EB8000C0F8011FC0F8052F9DF80800F6
:10BB800000EBC00101EB002009EBC0019DF81000A3
:10BB900000EB401001EB800090F8D81E9DF80800E3
:10BBA00000EBC00202EB002009EBC00090F8D40EBD
:10BBB00081427CD199F821064F46B8B19DF8080022
:10BBC00000EB400101EB00109DF8101009EB001094
:10BBD00000EB011090F8421A41F0080280F8422A66
:10BBE0009DF808100220FDF7B5FF88E0C7F8355032
:10BBF0009DF8080000EBC00101EB002007EBC0013D
:10BC00009DF81000102200EB401001EB800101F6BE
:10BC1000F9610798FCF717FB9DF8080000EBC001DD
:10BC200001EB002007EBC0019DF8100000EB401075
:10BC300001EB8000D0F8F11EC7F81910D0F8F50E0E
:10BC4000C7F81D009DF8080000EB400101EB001053
:10BC500007EB00119DF8100001EB001090F8400A6E
:10BC60003876F548D0F86812C7F83910B0F86C0289
:10BC7000A7F83D009DF8080000EBC00101EB002093
:10BC800007EBC0019DF8100000EB401001EB8000B5
:10BC9000D0F80C0FC7F821009DF8080000EB400118
:10BCA00001EB001007EB00119DF8100000E014E01C
:10BCB00001EB0010D0F8440AC7F83F00786D81B25C
:10BCC0000220FDF733F900210620FDF743FF786DD0
:10BCD000401C78650021052085E79DF8080000EBF1
:10BCE000400101EB00109DF8101009EB001000EB73
:10BCF000011090F8421A41F0040180F8421A9DF8B0
:10BD0000080000EBC00101EB002009EBC0019DF829
:10BD1000100000EB401001EB800080F8165F9DF8EA
:10BD2000080000EBC00101EB002009EBC0019DF809
:10BD3000100000EB401001EB800080F8DC6E9DF8F5
:10BD4000080000EBC00101EB002009EBC0019DF8E9
:10BD5000100000EB401001EB800090F8D80E042892
:10BD600043F094869DF8080000EB400101EB0010C1
:10BD70009DF8101009EB001000EB011090F8421A2A
:10BD800041F0800280F8422A9DF8080000EBC001D3
:10BD900001EB002009EBC00080F8D34E9DF80800AD
:10BDA000052200EBC00101EB002009EBC0039DF868
:10BDB000100000EB401003EB800080F8D82EB2E4B6
:10BDC00009EBC0019DF8100000EB401001EB800072
:10BDD00090F8DA0EB228F2D19DF8080000EBC0010D
:10BDE00001EB002009EBC00080F8D35E9DF808004D
:10BDF000B22100EBC00202EB002009EBC0029DF86B
:10BE0000100000EB401002EB800080F8DC1E9DF873
:10BE1000080000EBC00101EB002009EBC0019DF818
:10BE2000100000EB401001EB800080F8DA5E7AE44D
:10BE30009DF8080000EB4001C1EBC01051461AF814
:10BE40003000042809D09DF8080000EB4002C2EB46
:10BE5000C01011F83000152801D1ADF818009DF878
:10BE60000800D14600EB4002C2EBC01001EBC0005D
:10BE700043789DF8080000EB4002C2EBC01011F8B7
:10BE8000300043EA0021A1F58050303822D09DF8DF
:10BE9000080000EB4001C1EBC01009EBC0004946AF
:10BEA00042789DF8080000EB4003C3EBC01019F87E
:10BEB000300042EA0020A0F58052313A0CD09DF8C3
:10BEC000080000EB4002C2EBC01011F8300002285D
:10BED00004D019E0A62015E0A72013E09DF8080083
:10BEE00000EB4002C2EBC01001EBC00002799DF8EC
:10BEF000080000EB4003C3EBC01009EBC000C078A2
:10BF000042EA0020ADF818009DF80800474600EB13
:10BF1000C00101EB002008EBC00090F8D21E8DF8A4
:10BF200010109DF8080008EB00119DF8100008445F
:10BF300080F8D059BDF8180043F23002811A9042BF
:10BF40007CD009DC04287AD0152879D0A6280DD019
:10BF5000A72843F09B85C8E0B1F5C06F71D0A1F56B
:10BF6000C06101396ED00429F3D1FDE39DF80800CA
:10BF700000EBC00101EB002007EBC00080F8D35EAE
:10BF80009DF8080000EBC00101EB002007EBC001A9
:10BF90009DF8100000EB401001EB800090F8D80EE7
:10BFA000032836D09DF8080000EBC00101EB00200B
:10BFB00007EBC0019DF8100000EB401001EB800082
:10BFC00090F8D80E08283ED09DF8080000EBC0017C
:10BFD00001EB002007EBC0019DF8100000EB4010C2
:10BFE00001EB800090F8D80E0D2836D09DF808009F
:10BFF00000EBC00101EB002007EBC0019DF8100031
:10C0000000EB401001EB800090F8DC0EA5282ED04C
:10C010003FE09DF80800042100EBC00202EB002085
:10C0200007EBC0029DF8100000EB401002EB80000F
:10C0300080F8D81EA821FCE3D4100020D1E0E3E072
:10C04000FDE11EE24DE29DF80800092100EBC0026F
:10C0500002EB002007EBC002ECE39DF808000E2184
:10C0600000EBC00202EB002007EBC002F6E39DF8F4
:10C07000080000EB400101EB00109DF8101007EBE9
:10C08000001000EB011090F8421A41F0040180F812
:10C09000421A9DF8080000EBC00101EB002007EBFD
:10C0A000C0019DF8100000EB401001EB800090F8FB
:10C0B000DA0EA12803F0EA849DF8080000EBC00125
:10C0C00001EB002007EBC0019DF8100000EB4010D1
:10C0D00001EB800090F8DA1E9DF8080000EBC0022A
:10C0E00002EB002007EBC002FDE39DF8080000EB27
:10C0F000C00101EB002007EBC00080F8D35E9DF883
:10C10000080000EBC00101EB002007EBC0019DF827
:10C11000100000EB401001EB800090F8D80E0528CD
:10C120009DF8080000EBC00101EB00200CD007EBEC
:10C13000C0019DF8100000EB401001EB800090F86A
:10C14000D80E092806D016E007EBC00080F8D35EB1
:10C15000062100E00A219DF8080000EBC00202EB76
:10C16000002007EBC0029DF8100000EB401002EB2E
:10C17000800080F8D81E9DF8080000EBC00101EB9C
:10C18000002007EBC0019DF8100000EB401001EB10
:10C19000800090F8DC0EA42821D19DF8080000EB67
:10C1A000400101EB00109DF8101007EB001000EBB0
:10C1B000011090F8421A41F0200180F8421A9DF8CF
:10C1C000080000EBC00101EB002007EBC0019DF867
:10C1D000100000EB401001EB800080F8155FA121FA
:10C1E00029E79DF8080000EBC00101EB002007EBF8
:10C1F000C00080F8D35E9DF8080000EBC00101EBA1
:10C20000002007EBC001FCE39DF8080000EBC00133
:10C2100001EB002007EBC0019DF8100000EB40107F
:10C2200001EB800090F8D80E01289DF8080000EB83
:10C23000C00101EB002054D007EBC0019DF81000B5
:10C2400000EB401001EB800090F8D80E07289DF815
:10C25000080000EBC00101EB002048D007EBC00153
:10C260009DF8100000EB401001EB800090F8D80E14
:10C270000B289DF8080000EBC00101EB00203CD02A
:10C2800007EBC0019DF8100000EB401001EB8000AF
:10C2900090F8D80E0C289DF8080000EBC00101EBC7
:10C2A000002040D007EBC0019DF8100000EB4010CB
:10C2B00001EB800090F8D80E0E284BD09DF80800B6
:10C2C00000EBC00101EB002007EBC0019DF810005E
:10C2D00000EB401001EB800090F8D80E0F2879D0C9
:10C2E0006DE507EBC00080F8D35E022120E007EB8C
:10C2F000C00080F8D35E08211AE007EBC00080F888
:10C30000D35E9DF808000C2100EBC00202EB002078
:10C3100007EBC0029DF8100000EB401002EB80001C
:10C3200080F8D81E5BE707EBC00080F8D35E0D21D4
:10C330009DF8080000EBC00202EB002007EBC002F2
:10C340009DF8100000EB401002EB800080F8D81E32
:10C35000594670E69DF808000F2100EBC00202EB81
:10C36000002007EBC0029DF8100000EB401002EB2C
:10C37000800080F8D81E9DF80800A12100EBC002C3
:10C3800002EB002007EBC0029DF8100000EB40100C
:10C3900002EB800080F8DC1E9DF8080000EBC00274
:10C3A00002EB002007EBC0029DF8100000EB4010EC
:10C3B00002EB800080F8DA1E9DF8080000EB4001D7
:10C3C00001EB001007EB00119DF8100001EB0010CD
:10C3D000FDE3FFE79DF8080000EBC00101EB002042
:10C3E00007EBC0019DF8100000EB401001EB80004E
:10C3F00090F8DA0EA12818D09DF8080000EBC002D2
:10C4000002EB002007EBC0029DF8100000EB40108B
:10C4100002EB800080F8DCBE9DF8080000EBC00154
:10C4200001EB002007EBC001F7E39DF80800A12114
:10C4300000EBC00202EB002007EBC002EEE39DF828
:10C440000800A12100EBC00202EB002007EBC002B4
:10C450009DF8100000EB401002EB800080F8DA1E1F
:10C460009DF8080000EBC00202EB002007EBC002C1
:10C470009DF8100000EB401002EB800080F8DC1EFD
:10C48000FEE39DF8080000EBC00101EB002007EB84
:10C49000C0019DF8100000EB401001EB800090F807
:10C4A000D80E062843F0F2829DF8080000EBC00188
:10C4B00001EB002007EBC00080F8D35E9DF8080078
:10C4C000072100EBC00202EB002007EBC0029DF841
:10C4D000100000EB401002EB800080F8D81EA7216E
:10C4E000A9E59DF8080000EBC00101EB002007EB77
:10C4F000C00080F8D35E9DF80800A72100EBC002C1
:10C5000002EB002007EBC0029DF8100000EB40108A
:10C5100002EB800080F8DC1E9DF808004B4600EB23
:10C520004001C1EBC01009EBC000407930289DF8F4
:10C53000080000EB400146D0C1EBC01003EBC00087
:10C54000407931289DF808007ED000EB4001C1EB16
:10C55000C01003EBC000407933289DF8080000EBC1
:10C56000400172D0C1EBC01003EBC0004079342809
:10C570009DF8080000EB400101EB00109DF8101041
:10C5800007EB001000EB011090F8421A73D021F075
:10C59000010180F8421A9DF8080000EB400101EB10
:10C5A000001007EB00119DF8100001EB001191F84D
:10C5B000420A20F0020281F8422A0020CDE9000060
:10C5C0008DF83850CCE101EB00109DF8101007EB0E
:10C5D000001000EB011090F8421A21F0010180F8E0
:10C5E000421A9DF8080000EB400101EB00109DF895
:10C5F000101007EB001000EB011090F8421A21F028
:10C60000020180F8421A9DF8080000EBC00101EB1E
:10C61000002007EBC0019DF8100000EB401001EB7B
:10C62000800090F8DB0E3128C7D19DF8080000EBA0
:10C63000400101EB00109DF8101007EB001000EB1B
:10C64000011090F8421A01E016E01BE121F02001F0
:10C6500080F8421A9DF8080000EBC00101EB0020B1
:10C6600007EBC0019DF8100000EB401001EB8000CB
:10C6700080F8155FA1E727E100EBC00101EB002086
:10C6800007EBC0019DF8100000EB401001EB8000AB
:10C6900090F8160F00289DF8080000EBC00101EB90
:10C6A000002007EBC0019DF8100000EB401001EBEB
:10C6B00080007DD080F8155F9DF8080000EB4001F8
:10C6C00001EB001007EB00119DF8100001EB0011C9
:10C6D00091F8420A20F0010281F8422A9DF80800F0
:10C6E00000EB400101EB00109DF8101007EB00106B
:10C6F00000EB011090F8421A21F0020180F8421A72
:10C7000097F821060028B5D1387D0128B2D1786D7F
:10C71000F98A8842AED29DF8080000EBC00101EB17
:10C7200000209DF8101007EBC00001EB411100EB59
:10C73000810090F8150F01289CD19DF8080000EBAE
:10C74000C00101EB002007EBC0019DF8100000EBD9
:10C75000401001EB800090F8490F00288AD14FF07B
:10C7600010419DF8080000E0BBE100EBC00202EBC5
:10C77000002007EBC0029DF8100000EB401002EB18
:10C780008000C0F8E01E9DF8080000EB400101EBBE
:10C79000001007EB00119DF8100001EB001090F85D
:10C7A000401A9DF8080000EBC00202EB002000E0F8
:10C7B00055E007EBC00080F8D11E9DF8080000EBA3
:10C7C000C00101EB002007EBC0019DF8100000EB59
:10C7D000401001EB800090F8D81E9DF8080000EB97
:10C7E000C00202EB002007EBC00090F8D40E81429B
:10C7F00089D19DF8080000EBC00101EB002007EB98
:10C80000C0019DF8100000EB401001EB800080F8A3
:10C81000DD5E9DF80800A42100EBC00202EB0020C1
:10C8200007EBC0029DF8100000EB401002EB800007
:10C8300001E0E9E3DFE380F8DA1E9DF8080000EB91
:10C84000C00202EB002007EBC0029DF8100000EBD5
:10C85000401002EB800080F8DCBEAEE6DEE380F83C
:10C86000154F9DF8080000EB400101EB001007EBAD
:10C8700000119DF8100001EB001191F8420A40F000
:10C88000010229E701EB00109DF8101007EB0010E2
:10C8900000EB011090F8421A41F0010180F8421AB1
:10C8A0009DF8080000EB400101EB00109DF810100E
:10C8B00007EB001000EB011090F8421A41F0020162
:10C8C00080F8421AA22118E021F0200180F8421AD3
:10C8D0009DF8080000EB400101EB001007EB001091
:10C8E0009DF8101000E0E0E300EB011090F8421A10
:10C8F00021F0020180F8421AA9219DF8080000EBFE
:10C90000C00202EB00209DF8102007EBC00002EBF4
:10C91000421200EB820080F8DA1E4EE6DDE90001EB
:10C92000090141EA10710001CDE900019DF80800FC
:10C9300000EB4001C1EBC0109DF8381003EBC000C4
:10C9400008448079DDE9002C3038C117104341EAF2
:10C950000C01CDE900019DF83800401C8DF838002D
:10C960009DF838000628D9D39DF80800009900EBFF
:10C97000C00202EB002007EBC0029DF8100000EBA4
:10C98000401002EB8000C0F8F11E0021CDE900113B
:10C990008DF8385021E0DDE90001090141EA10710C
:10C9A0000001CDE900019DF8080000EB4001C1EB5A
:10C9B000C0109DF8381003EBC0000844407BDDE94F
:10C9C000002C3038C117104341EA0C01CDE90001B9
:10C9D0009DF83800401C8DF838009DF83800042878
:10C9E000D9D39DF80800009900EBC00202EB0020AB
:10C9F00007EBC0029DF8100000EB401002EB800036
:10CA000000E09FE2C0F80C1F0021CDE900118DF875
:10CA1000385021E0DDE90001090141EA107100010F
:10CA2000CDE900019DF8080000EB4001C1EBC0100A
:10CA30009DF8381003EBC0000844407CDDE9002C71
:10CA40003038C117104341EA0C01CDE900019DF8CF
:10CA50003800401C8DF838009DF838000628D9D3DE
:10CA60009DF80800009900EBC00202EB002007EBE4
:10CA7000C0029DF8100000EB401002EB8000C0F8EF
:10CA8000F51E9DF8080000EB4001C1EBC01003EB60
:10CA9000C00041799DF8080000EBC00202EB0020C5
:10CAA00007EBC0029DF8100000EB401002EB800085
:10CAB00080F8DB1E9DF8080000EB400101EB001040
:10CAC00007EB00119DF8100001EB001090F8421ADE
:10CAD0009DF8080000EBC00202EB002007EBC0024B
:10CAE000FDE39DF8080000EBC00101EB002007EB1F
:10CAF000C00080F8D35E9DF8080000EBC00101EB98
:10CB0000002007EBC0019DF8100000EB401001EB86
:10CB1000800090F8D80E0A286DD09DF8080000EB30
:10CB2000C00101EB00209DF8101007EBC00001EBE5
:10CB3000411100EB810090F8D81E9DF8080000EB31
:10CB4000C00202EB002007EBC00090F8D40E814237
:10CB500014D197F82106D8B39DF8080000EB4001E6
:10CB600001EB00109DF8101007EB001000EB011016
:10CB700090F8421A41F0080280F8422A9DF8080015
:10CB8000A72100EBC00202EB002007EBC0029DF8DA
:10CB9000100000EB401002EB800080F8DC1E9DF8D6
:10CBA0000800A22100EBC00202EB002007EBC0024C
:10CBB0009DF8100000EB401002EB800080F8DA1EB8
:10CBC0009DF8080000EBC00101EB002001E05AE3F2
:10CBD00025E007EBC0019DF8100000EB401001EBD1
:10CBE000800080F8165F0022CDE9002211468DF802
:10CBF0003850CC469CE09DF808000B2100EBC002A9
:10CC000002EB002007EBC0029DF8100000EB401083
:10CC100002EB800080F8D81EB0E779E395E3C7F80F
:10CC200035509DF8080000EBC00101EB002007EB38
:10CC3000C0019DF81000102200EB401001EB8001B4
:10CC400001F6F9610798FBF7FEFA9DF8080000EB82
:10CC5000C00101EB002007EBC0019DF8100000EBC4
:10CC6000401001EB8000D0F8F11EC7F81910D0F881
:10CC7000F50EC7F81D009DF8080000EB400100E02C
:10CC800050E301EB001007EB00119DF8100001EBE1
:10CC9000001090F8400A38769DF8080000EBC001BB
:10CCA00001EB002007EBC0019DF8100000EB4010E5
:10CCB00001EB8000D0F80C0FC7F82100FE48D0F837
:10CCC0006812C7F83910B0F86C02A7F83D00786D0B
:10CCD00081B20220FCF72AF900210620FCF73AFF76
:10CCE000786D401C786500210520FCF733FF45E78F
:10CCF0000098090141EA10710001CDE900019DF899
:10CD0000080000EB4001C1EBC0109DF838100CEB9F
:10CD1000C0000844C07ADDE900233038C117104351
:10CD20001943CDE900019DF83800401C8DF838000A
:10CD30009DF838000A28DBD3DDE900129DF80800D1
:10CD400000EBC00303EB002007EBC0039DF81000CD
:10CD500000EB401003EB8000C0F8F91EC0F8FD2E78
:10CD60000021CDE900118DF8385020E0DDE9000107
:10CD7000090141EA10710001CDE900019DF80800A8
:10CD800000EB4001C1EBC0109DF838100CEBC00067
:10CD90000844407DDDE900233038C11710431943B2
:10CDA000CDE900019DF83800401C8DF838009DF851
:10CDB00038000A28DAD3DDE900129DF8080000EBFC
:10CDC000C00303EB002007EBC003FDE39DF8080060
:10CDD00000EB4001C1EBC01051461AF830000428A6
:10CDE00009D09DF8080000EB4002C2EBC01011F81A
:10CDF0003000152801D1ADF818009DF808005746FD
:10CE000000EB4002C2EBC01001EBC00042789DF87D
:10CE1000080000EB4003C3EBC01011F8300042EAF9
:10CE20000020A0F58051303922D09DF8080000EB99
:10CE30004001C1EBC01007EBC000394642789DF8B5
:10CE4000080000EB4003C3EBC01017F8300042EAC3
:10CE50000020A0F58052313A0CD09DF8080000EB7C
:10CE60004002C2EBC01011F83000022804D019E0D3
:10CE7000A62015E0A72013E09DF8080000EB400273
:10CE8000C2EBC01001EBC00002799DF8080000EB76
:10CE90004003C3EBC01007EBC000C07842EA00209B
:10CEA000ADF818009DF8080000EBC00101EB002070
:10CEB00008EBC00090F8D21E8DF810109DF8080005
:10CEC00008EB00119DF81000084480F8D059BDF817
:10CED0001800A7287DD007DC04287BD015287AD03D
:10CEE000A62842F0D38537E000F51D60B0F58040FC
:10CEF00004D0112870D01228F3D1FCE39DF808006B
:10CF000000EBC00101EB002008EBC0019DF8100010
:10CF100000EB401001EB800090F8D80E0028E0D123
:10CF20009DF8080000EBC00101EB002008EBC000F9
:10CF300080F8D35E9DF8080000EBC00101EB0020F3
:10CF400008EBC0019DF8100000EB401001EB8000E1
:10CF500080F8D84EFFF7C3BA9DF8080000EBC00177
:10CF600001EB002008EBC00080F8D35E9DF80800BC
:10CF700000EBC00101EB002008EBC0019DF81000A0
:10CF800000EB401001EB800090F8D80E022829D069
:10CF90009DF8080000EBC00101EB002008EBC00188
:10CFA0009DF8100000EB401001EB800090F8D80EC7
:10CFB00005282AD09DF8080000EBC00101EB0020F5
:10CFC00008EBC0019DF8100000EB401001EB800061
:10CFD00003E088E0C7E0CBE1ECE190F8DC0EA528A7
:10CFE00026D037E09DF80800032100EBC00202EBD9
:10CFF000002008EBC0029DF8100000EB401002EB8F
:10D00000800080F8D81EA921F4E39DF808000621CD
:10D0100000EBC00202EB002008EBC0029DF81000FC
:10D0200000EB401002EB800080F8D81EA221E1E363
:10D030009DF8080000EB400101EB001008EB001127
:10D040009DF8100001EB001090F8421A41F0040125
:10D0500080F8421A9DF8080000EBC00101EB0020A7
:10D0600008EBC0019DF8100000EB401001EB8000C0
:10D0700090F8DA0EA12802F009859DF8080000EB6F
:10D08000C00101EB002008EBC0019DF8100000EB8F
:10D09000401001EB800090F8DA1E9DF8080000EBCC
:10D0A000C00202EB002008EBC0029DF8100000EB6C
:10D0B000401002EB800001E0D410002080F8DC1E5C
:10D0C000A1219DF8080000EBC00202EB002008EB54
:10D0D000C0029DF8100000EB401002EB800080F8C9
:10D0E000DA1E02F0D3BC9DF8080000EBC00101EB92
:10D0F000002008EBC0019DF8100000EB401001EB90
:10D10000800090F8DC0EA42821D19DF8080000EBE7
:10D11000400101EB00109DF8101008EB001000EB2F
:10D12000011090F8421A41F0200180F8421A9DF84F
:10D13000080000EBC00101EB002008EBC0019DF8E6
:10D14000100000EB401001EB800080F8155F9DF8A7
:10D15000080000EBC00101EB002008EBC00080F8E4
:10D16000D35EFFF73CB89DF8080000EBC00101EB6F
:10D17000002008EBC0019DF8100000EB401001EB0F
:10D18000800090F8D80E01289DF8080000EBC0013F
:10D1900001EB002030D008EBC0019DF8100000EB3F
:10D1A000401001EB800090F8D80E04289DF808008C
:10D1B00000EBC00101EB002024D008EBC0019DF87A
:10D1C000100000EB401001EB800090F8D80E06280C
:10D1D0009DF8080000EBC00101EB002021D008EB16
:10D1E000C0019DF8100000EB401001EB800090F8AA
:10D1F000D80E072860D074E708EBC00080F8D35E33
:10D20000022104E008EBC00080F8D35E05219DF800
:10D21000080000EBC00202EB002008EBC002FFF7A1
:10D220008FB808EBC00080F8D35E9DF80800072295
:10D2300000EBC00101EB002008EBC0039DF81000DB
:10D2400000EB401003EB800080F8D82E9DF808001A
:10D25000A12200EBC00101EB002008EBC0039DF808
:10D26000100000EB401003EB800080F8DC2E9DF8EE
:10D27000080000EB400101EB00109DF8101008EBD6
:10D28000001000EB011090F8421A41F0800180F884
:10D29000421A9DF8080000EB400101EB00109DF8D8
:10D2A000101008EB001000EB011090F8421A41F04A
:10D2B000040180F8421A14E79DF8080000EBC00151
:10D2C00001EB002008EBC0019DF8100000EB4010BE
:10D2D00001EB800090F8DA0EA1282DD000E079E370
:10D2E0009DF8080000EBC00202EB002008EBC00232
:10D2F0009DF8100000EB401002EB800080F8DCBECF
:10D300009DF8080000EBC00101EB002008EBC00114
:10D310009DF8100000EB401001EB800090F8DA0E51
:10D32000A228C8D09DF8080000EBC00101EB002046
:10D3300008EBC000FEF7C0BA9DF80800A12100EB81
:10D34000C00202EB002008EBC0029DF8100000EBC9
:10D35000401002EB800080F8DC1E9DF8080000EB16
:10D36000C00101EB002008EBC00080F8D34EB8E606
:10D370009DF80800A12100EBC00202EB002008EBA1
:10D38000C0029DF8100000EB401002EB800080F816
:10D39000DC1E9DF8080000EBC00202EB002008EB49
:10D3A000C0029DF8100000EB401002EB800080F8F6
:10D3B000DA1EB7E79DF8080000EBC00101EB002082
:10D3C00008EBC00080F8D35E9DF80800A72100EBB1
:10D3D000C00202EB002008EBC0029DF8100000EB39
:10D3E000401002EB800080F8DC1E9DF808003B46F0
:10D3F00000EB4001C1EBC01007EBC00040793028C2
:10D400009DF8080000EB400151D0C1EBC01003EBC8
:10D41000C000407931289DF808007DD000EB400124
:10D42000C1EBC01003EBC000407933289DF8080021
:10D4300000EB400171D0C1EBC01003EBC00040799C
:10D4400034289DF8080000EB400167D0C1EBC01004
:10D4500003EBC0004079352872D09DF8080000EB3E
:10D46000400101EB00109DF8101008EB001000EBDC
:10D47000011090F8421A21F0010180F8421A9DF83B
:10D48000080000EB400101EB001008EB00119DF8D3
:10D49000100001EB001191F8420A20F0020281F81D
:10D4A000422A0020CDE900008DF83850D6E101EB8A
:10D4B00000109DF8101008EB001000EB011090F820
:10D4C000421A21F0010180F8421A9DF8080000EB91
:10D4D000400101EB00109DF8101008EB001000EB6C
:10D4E000011090F8421A21F0020180F8421A9DF8CA
:10D4F000080000EBC00101EB002008EBC0019DF823
:10D50000100000EB401001EB800090F8DB0E31289A
:10D51000C7D19DF8080002E013E019E13AE100EB01
:10D52000400101EB00109DF8101008EB001000EB1B
:10D53000011090F8421A21F0200180F8421AB0E759
:10D5400059E100EBC00101EB002008EBC0019DF8A0
:10D55000100000EB401001EB800090F8160F00283F
:10D560009DF8080000EBC00101EB002008EBC001B2
:10D570009DF8100000EB401001EB80007ED080F899
:10D58000155F9DF8080000EB400101EB001008EB6F
:10D5900000119DF8100001EB001191F8420A20F0F3
:10D5A000010281F8422A9DF8080000EB400101EBDE
:10D5B00000109DF8101008EB001000EB011090F81F
:10D5C000421A21F0020100E07FE380F8421A98F845
:10D5D00021060028B3D198F814000128AFD1D8F85B
:10D5E0005400B8F816108842A9D29DF8080000EB44
:10D5F000C00101EB00209DF8101008EBC00001EB0A
:10D60000411100EB810090F8150F012897D19DF88A
:10D61000080000EBC00101EB002008EBC0019DF801
:10D62000100000EB401001EB800090F8490F00283B
:10D6300085D19DF808004FF0104100EBC00202EBCD
:10D64000002008EBC0029DF8100000EB401002EB38
:10D650008000C0F8E01E9DF8080000EB400101EBDF
:10D66000001008EB00119DF8100001EB001090F87D
:10D67000401A9DF8080000EBC00200E055E002EB04
:10D68000002008EBC00080F8D11E9DF8080000EBD8
:10D69000C00101EB002008EBC0019DF8100000EB79
:10D6A000401001EB800090F8D81E9DF8080000EBB8
:10D6B000C00202EB002008EBC00090F8D40E8142BB
:10D6C00088D19DF8080000EBC00101EB002008EBB9
:10D6D000C0019DF8100000EB401001EB800080F8C5
:10D6E000DD5E9DF80800A42100EBC00202EB0020E3
:10D6F00008EBC00200E076E19DF8100000EB40105E
:10D7000002EB800080F8DA1E9DF8080000EBC002F2
:10D7100002EB002008EBC0029DF8100000EB401067
:10D7200002EB800080F8DCBEBBE680F8154F9DF868
:10D73000080000EB400101EB001008EB00119DF820
:10D74000100001EB001191F8420A40F0010228E7B5
:10D7500001EB00109DF8101008EB001000EB011019
:10D7600090F8421A41F0010180F8421A9DF8080031
:10D7700000EB400101EB00109DF8101008EB0010C9
:10D7800000EB011090F8421A41F0020180F8421AB1
:10D79000A22120E001EB00109DF8101008EB001012
:10D7A00000EB011090F8421A21F0200180F8421A93
:10D7B0009DF8080000EB400101EB00109DF81010EF
:10D7C00008EB001000EB011090F8421A21F0020162
:10D7D00080F8421AA9219DF8080000EBC00202EB74
:10D7E00000209DF8102008EBC00002EB421200EB75
:10D7F00082000FE0F7E29DF80800A12100EBC002D3
:10D8000002EB002008EBC0029DF8100000EB401076
:10D8100002EB800080F8DA1E43E6DDE9001000012B
:10D8200040EA11700901CDE900109DF8080000EBF5
:10D830004001C1EBC0109DF8381003EBC000084454
:10D840008079DDE900273038C11710433943CDE92D
:10D8500000019DF83800401C8DF838009DF8380014
:10D860000828DAD39DF80800009900EBC00202EB0B
:10D87000002008EBC0029DF8100000EB401002EB06
:10D880008000C0F8F11E0021CDE900118DF838505C
:10D8900020E0DDE90010000140EA11700901CDE946
:10D8A00000109DF8080000EB4001C1EBC0109DF88E
:10D8B000381003EBC0000844C07BDDE90027303896
:10D8C000C11710433943CDE900019DF83800401CD1
:10D8D0008DF838009DF838000628DAD39DF8080046
:10D8E000009900EBC00202EB002008EBC0029DF89B
:10D8F000100000EB401002EB8000C0F80C1F00216C
:10D90000CDE900118DF8385020E0DDE90001090172
:10D9100041EA10710001CDE900019DF8080000EB1B
:10D920004001C1EBC0109DF8381003EBC000084463
:10D93000407DDDE900273038C11710433943CDE978
:10D9400000019DF83800401C8DF838009DF8380023
:10D950000828DAD39DF80800009900EBC00202EB1A
:10D96000002008EBC0029DF8100000EB401002EB15
:10D970008000C0F8F51E9DF8080000EB4001C1EBE7
:10D98000C01003EBC00041799DF8080000EBC00215
:10D9900002EB002008EBC0029DF8100000EB4010E5
:10D9A00002EB800080F8DB1E9DF8080000EB4001D0
:10D9B00001EB001008EB00119DF8100001EB0010C6
:10D9C00090F8421A9DF8080000EBC00202EB00201C
:10D9D00008EBC0029DF8100000EB401002EB800045
:10D9E00080F8F01E07E49DF8080000EBC00101EB91
:10D9F000002008EBC00080F8D35E9DF8080000EB23
:10DA0000C00101EB002008EBC0019DF8100000EB05
:10DA1000401001EB800090F8D80E03286AD09DF8E2
:10DA2000080000EBC00101EB00209DF8101008EB8E
:10DA3000C00001EB411100EB810090F8D81E9DF869
:10DA4000080000EBC00202EB002008EBC00090F8D9
:10DA5000D40E814214D198F82106E0B39DF8080055
:10DA600000EB400101EB00109DF8101008EB0010D6
:10DA700000EB011090F8421A41F0080280F8422AA7
:10DA80009DF8080000EBC00101EB002008EBC0018D
:10DA90009DF8100000EB401001EB800080F8165F4D
:10DAA0009DF80800A72100EBC00202EB002008EB64
:10DAB000C0029DF8100000EB401002EB800080F8DF
:10DAC000DC1E9DF80800A22100EBC00202EB002042
:10DAD00008EBC00200E01FE09DF8100000EB4010D2
:10DAE00002EB800080F8DA1E0021CDE900118DF8EC
:10DAF00038509DE09DF80800042100EBC00202EBC5
:10DB0000002008EBC0029DF8100000EB401002EB73
:10DB1000800080F8D81EB3E7C8F835509DF808009B
:10DB200000EBC00101EB002008EBC0019DF81000E4
:10DB3000102200EB401001EB800101F6F96107981B
:10DB4000FAF781FB9DF8080000EBC00101EB002013
:10DB500008EBC0019DF8100000EB401001EB8000C5
:10DB6000D0F8F11EC8F81910D0F8F50EC8F81D004D
:10DB70009DF8080000EB400101EB001008EB0011DC
:10DB80009DF8100001EB001090F8400A88F818008A
:10DB90009DF8080000EBC00101EB002008EBC0017C
:10DBA0009DF8100000EB401001EB8000D0F80C0F46
:10DBB000C8F82100FE48D0F86812C8F83910B0F84B
:10DBC0006C02A8F83D00D8F8540081B20220FBF79F
:10DBD000ADF900210620FBF7BDFFD8F85400401C2A
:10DBE000C8F8540000210520FBF7B4FF48E7DDE941
:10DBF0000001090141EA10710001CDE900019DF821
:10DC0000080000EB4001C1EBC0109DF8381007EB95
:10DC1000C0000844C07ADDE900233038C117104342
:10DC20001943CDE900019DF83800401C8DF83800FB
:10DC30009DF838000C28DAD3DDE900129DF80800C1
:10DC400000EBC00303EB002008EBC0039DF81000BD
:10DC500000EB401003EB8000C0F8F91EC0F8FD2E69
:10DC60000021CDE900118DF8385020E0DDE90001F8
:10DC7000090141EA10710001CDE900019DF8080099
:10DC800000EB4001C1EBC0109DF8381007EBC0005D
:10DC90000844C07DDDE900233038C1171043194323
:10DCA000CDE900019DF83800401C8DF838009DF842
:10DCB00038000C28DAD3DDE900129DF8080000EBEB
:10DCC000C00303EB002008EBC0039DF8100000EB3D
:10DCD000401003EB8000C0F8011FC0F8052F81E65B
:10DCE0009DF8080043469DF8101008EB001008440A
:10DCF00080F8D0599DF80800D44600EB4001C1EBF4
:10DD0000C0100AEBC000407870280AD19DF80800C6
:10DD100000EB4001C1EBC0100CEBC0008078FA288A
:10DD200030D09DF8080000EB4001C1EBC0100CEBB7
:10DD3000C00040789DF8080000EB4001C1EBC01026
:10DD40001CF830009DF8080000EBC00101EB00203A
:10DD500003EBC00090F8D21E8DF810109DF808005B
:10DD600003EB00119DF81000084480F8D059BDF86D
:10DD70001800012841D065287ED0B128AFD0B62840
:10DD8000ADD103E0B120ADF81800DBE79DF8080045
:10DD900000EBC00101EB002003EBC0019DF8100077
:10DDA00000EB401001EB800090F8D80E012896D1CE
:10DDB0009DF8080000EBC00101EB002003EBC00060
:10DDC00080F8D35E9DF8080000EBC00101EB002055
:10DDD00003EBC0019DF8100000EB401001EB800048
:10DDE00080F8D84EB1219DF8080000EBC00202EB8C
:10DDF000002008EBC002FDF756BD9DF8080000EBBF
:10DE00004001C1EBC0100AEBC00000790128B5D079
:10DE10000228B3D00328B1D00528B1D19DF808005D
:10DE200000EBC00101EB002003EBC0019DF81000E6
:10DE300000EB401001EB800090F8D80E00289FD135
:10DE40009DF8080000EBC00101EB002003EBC000CF
:10DE500080F8D35E9DF8080000EBC00101EB0020C4
:10DE600003EBC0019DF8100000EB401001EB8000B7
:10DE700080F8D84EB62100E012E09DF8080000EBD3
:10DE8000C00202EB002003EBC0029DF8100000EB83
:10DE9000401002EB800080F8DC1EB221FFF711B9C0
:10DEA0009DF8080000EB4001C1EBC0100CEBC00076
:10DEB0000079B922ADF818209DF8080000EB400168
:10DEC000C1EBC0100CEBC000007900F00F018DF821
:10DED00014108DF838501DE09DF8080000EB40014B
:10DEE00001EB001003EB00119DF8380001EB00106E
:10DEF00090F8411A9DF8080000EB4007C7EBC010EE
:10DF00001CF830005038814212D09DF83800401C77
:10DF10008DF838009DF8080000EB400101EB00107F
:10DF200003EB001090F8170A9DF838108842D3D8F8
:10DF30009DF838009DF8141008448DF810009DF8E5
:10DF4000080000EBC00101EB002003EBC0079DF8C7
:10DF5000100000EB401007EB800090F8D80E01286D
:10DF600011D09DF8080000EBC00101EB002003EB8D
:10DF7000C0019DF8100000EB401001EB800090F80C
:10DF8000D80E01287ED19DF8080000EBC00101EBFE
:10DF9000002003EBC00080F8D35E9DF8080002214A
:10DFA00000EBC00707EB002003EBC00702E0000016
:10DFB000D41000209DF8100000EB401007EB80000B
:10DFC00080F8D81E9DF8080000EBC00101EB00208E
:10DFD000FAE39DF8080000EB400101EB001008EBAC
:10DFE000001090F81C0A20B101287DD00228C9D168
:10DFF00066E29DF8080008EB400000F50050B0F81C
:10E00000F00F801F81B29DF80800574600EB4002D8
:10E01000C2EBC0120AEBC200401CFBF711FBCDE9BA
:10E0200012059DF8080008EB400000F50050B0F81C
:10E03000F01F9DF80800394400EB4002C2EBC0100D
:10E040006FF0040202EBC0000844042107F06EFAEE
:10E05000DDE91223C117CDE90001504059400843C2
:10E0600090D19DF8080008EB001080F8D0599DF879
:10E070000800B94600EB4001C1EBC01107EBC1003D
:10E08000007900E0C5E2ADF81800BDF818003128AD
:10E09000ADD19DF8080008EB400000F50050B0F845
:10E0A000F00F4121183890FBF1F0C217CDE90002C2
:10E0B00088F804048DF838502F46BBE09DF808001E
:10E0C00000EB4001C1EBC0119DF8380009EBC10124
:10E0D00000EB80100844007D9DF83810414481F821
:10E0E00005049DF8080000E0AEE000EB4001C1EB44
:10E0F000C0119DF8380009EBC10100EB8010084405
:10E1000008211A3007F0DEF98DED0D0A10EE100A25
:10E110009DF8381008EB0111C1F815049DF80800AE
:10E1200000EB4001C1EBC0119DF8380009EBC101C3
:10E1300000EB801008440821323007F0C3F98DED60
:10E140000D0A10EE100A9DF8381008EB0111C1F805
:10E1500011049DF8080000EB4001C1EBC01109EB70
:10E16000C1009DF8381001EB8111084408213A30B4
:10E1700007F0A8F98DED0D0A10EE100A9DF8381081
:10E1800008EB0111C1F819049DF8080000EB4001EB
:10E19000C1EBC0119DF8380009EBC10100EB801004
:10E1A00008440821423007F08DF98DED0D0A10EE7C
:10E1B000100A9DF8381008EB0111C1F81D049DF8F4
:10E1C000080000EB400101EB00109DF8381008EB4F
:10E1D000001000EB011090F8421A41F0800180F825
:10E1E000421A9DF8080008EB400000F50050B0F816
:10E1F000F01F9DF80800494400EB4002C2EBC0103C
:10E200004FF0FF3202EBC000095C9DF8080000EB04
:10E21000C00202EB002008EBC0039DF8100000EBE9
:10E22000401003EB800080F8141F9DF83800401C5C
:10E230008DF838009DF83800DDE90012401A77EBC0
:10E240000200FFF43BAF4AE59DF80800574600EB9B
:10E250004001C1EBC0100AEBC000437D9DF80800EF
:10E2600000EB4002C2EBC0100AEBC000807D43EA25
:10E270000020C317CDE900039DF80800152100EB2D
:10E280004002C2EBC0100AEBC000FBF7C3F9CDE9B6
:10E290001205DDE90001129B694058400843D2D1C4
:10E2A0009DF8080000EB4001C1EBC011384617F89B
:10E2B0003120521E8DF810209DF8081008EB011235
:10E2C0009DF81010114481F8D0599DF81010414468
:10E2D00081F805549DF8101008EB0111C1F8155490
:10E2E0009DF8081001EB4102C2EBC11100EBC10126
:10E2F0008A799DF8081001EB4103C3EBC11100EBD3
:10E30000C101497942EA012100EE101AF8EE400AF3
:10E310009FEDFA0A9DF8081080EE801A01EB410289
:10E32000C2EBC11100EBC1010A799DF8081001EBA5
:10E330004103C3EBC11100EBC101C97842EA0121DD
:10E3400000EE901A9DF81010F8EE600A71EE200AA7
:10E3500010EE902A08EB0111C1F811249DF8081065
:10E3600001EB4102C2EBC11100EBC1018A7A9DF8B9
:10E37000081001EB4103C3EBC11100EBC101497A65
:10E3800042EA012100EE901A9DF80810B8EE601ADA
:10E39000C1EE000A01EB4102C2EBC11100EBC10169
:10E3A0000A7A9DF8081001EB4103C3EBC11100EBA1
:10E3B000C101C97942EA012100EE101A9DF810103E
:10E3C000B8EE400A30EE800A10EE102A08EB011178
:10E3D000C1F819249DF8081001EB4102C2EBC111EC
:10E3E00000EBC100C07A00069DF8080000EB400178
:10E3F000C1EBC01018D407EBC000027B9DF80800E9
:10E4000000EB4003C3EBC01007EBC000C07A42EA48
:10E41000002000EE100AB8EE400ADFEDB90A20EE47
:10E42000200A10EE100A19E007EBC000037B9DF8EC
:10E43000080000EB4001C1EBC01007EBC000C07A40
:10E4400043EA0020404280B2FAF7B9F89FEDAD1BD5
:10E4500053EC112BF9F7D2FFFAF701F99DF81010E0
:10E4600008EB0111C1F81D049DF8080000EB400104
:10E4700001EB00109DF8101008EB001000EB0110EC
:10E4800090F8421A41F0800180F8421A9DF8080085
:10E4900000EB4001C1EBC01107EBC100C17D9DF84D
:10E4A000080000EBC00202EB002008EBC0039DF85F
:10E4B000100000EB401003EB800080F8141FB7E061
:10E4C0009DF80800574600EB4001C1EBC0100AEB75
:10E4D000C000C3799DF8080000EB4002C2EBC010F9
:10E4E0000AEBC000007A43EA0020C317CDE900031D
:10E4F0009DF80800072100EB4002C2EBC0100AEBB8
:10E50000C000FBF787F8CDE91205DDE90001129B99
:10E510006940584008437CD19DF8080000EB400159
:10E52000C1EBC01117F83100401E8DF810009DF8A6
:10E53000080008EB001080F8D0599DF81000404406
:10E5400080F805549DF8080000EB4001C1EBC011B4
:10E5500007EBC1008079FAF732F841EC110B9FED1F
:10E560006B0B09F041F99DF80800B0EE408AF0EE1F
:10E57000608A00EB4001C1EBC01107EBC1000279DA
:10E580009DF8080000EB4001C1EBC01107EBC10092
:10E59000C07842EA0020FAF712F853EC182BF9F78A
:10E5A0009FFFFAF75CF89DF8101008EB0111C1F815
:10E5B00015049DF8100008EB0010C0F811549DF8E8
:10E5C000100008EB0010C0F819549DF8100008EB7B
:10E5D0000010C0F81D549DF8080000EB400101EB4D
:10E5E00000109DF8101008EB001000EB011090F8DF
:10E5F000421A41F0800280F8422A9DF8080000EBA0
:10E600004001C1EBC01107EBC100427A9DF8080040
:10E6100000E007E200EBC00101EB002008EBC003C3
:10E620009DF8100000EB401003EB800080F8142FE1
:10E630009DF8080000EB400101EB001008EB001012
:10E6400090F8170A88F80404ECE19DF8080000EB44
:10E650004001C1EBC0100AEBC0005146C3789DF8E1
:10E66000080000EB4002C2EBC0100AEBC00080784B
:10E6700043EA00208DF80C009DF8080000EB4002F2
:10E68000C2EBC0109DF80C200AEBC0001044437888
:10E690009DF8080000EB4002C2EBC0109DF80C2072
:10E6A00001EBC000805C43EA0020C317CDE9000302
:10E6B0009DF808009DF80C1000EB4002C2EBC01062
:10E6C0000AEBC000FAF7A6FFCDE91205DDE900016B
:10E6D000129B694058400843B6D19DF80800534644
:10E6E00000EB4001C1EBC0100AEBC00040788DF890
:10E6F00010008DF83850414626E0000000FF7F47AB
:10E700000000803D000000000000B0BF00000000DD
:10E71000000024409DF8080000EB400202EB0010CE
:10E720009DF8382001EB001000EB021090F8410A30
:10E730009DF8102090429DF8380002D18DF810000D
:10E7400010E0401C8DF838009DF8080000EB4002F6
:10E7500002EB001001EB001090F8170A9DF838202A
:10E760009042D7D89DF8080000EB400202EB001061
:10E770009DF8102001EB001000EB021090F8422AE7
:10E7800042F0800280F8422A9DF8080000EB400227
:10E79000C2EBC01003EBC0000079ADF818009DF883
:10E7A00008009DF8102001EB0010104480F8D059AB
:10E7B000BDF81800F32806D007DC052874D0F1282E
:10E7C00008D0F22888D189E18FE1F4286DD0F628AD
:10E7D000F8D18DE19DF8080000EBC00202EB0020AB
:10E7E00001EBC0029DF8100000EB401002EB80002E
:10E7F00090F8D80E00289DF8080021D000EB4002C8
:10E8000002EB00109DF8102001EB001000EB02104D
:10E8100090F8490AC00712D09DF80800C44600EBE2
:10E82000C00202EB002008EBC0029DF8100000EBD4
:10E83000401002EB800090F8580FC00720D0A8E0ED
:10E8400000EBC00202EB002001EBC0029DF81000BB
:10E8500000EB401002EB800080F8D84E9DF80800D5
:10E86000F42200EBC00707EB002001EBC0079DF886
:10E87000100000EB401007EB800080F8DC2E88E0F1
:10E880009DF8080000EBC00202EB00200CEBC00278
:10E890009DF8100000EB401002EB800090F84A0F4A
:10E8A00098B38DF8385028E092E133E19DF80800E4
:10E8B00000EBC00202EB00209DF810200CEBC00022
:10E8C00002EB421200EB82009DF83820104490F8D1
:10E8D0004B2F9DF8080000EB400707EB00109DF858
:10E8E00038700CEB0010384490F81E0A824208D1B0
:10E8F0009DF83800401C8DF838009DF83800042839
:10E90000D4D39DF83800042825D042E09DF80800B3
:10E9100000EBC00202EB00200CEBC0029DF81000DF
:10E9200000EB401002EB80009DF83820104490F876
:10E930004B0F9DF8082002EB420707EB02129DF8EF
:10E9400038700CEB02123A4492F81E2A904208D119
:10E950009DF83800401C8DF838009DF838000A28D2
:10E96000D4D39DF838000A2813D09DF8080000EB96
:10E97000C00202EB002008EBC0029DF8100000EB83
:10E98000401002EB800090F8582F42F0010280F80E
:10E99000582F9DF80C0011289DF8080000EB40024C
:10E9A00002EB00109DF8102001EB001000EB0210AC
:10E9B00090F8422A37D022F0080280F8422A9DF8C7
:10E9C000080000EBC00202EB002001EBC0029DF842
:10E9D000100000EB401002EB800090F8580FC007C9
:10E9E00020D09DF8080000EBC00202EB002001EBF4
:10E9F000C0029DF8100000EB401002EB8000A0F870
:10EA0000565F9DF80800052200EBC00303EB0020D1
:10EA100001EBC0019DF8100000EB401001EB8000FD
:10EA200080F8DC2E36E242F0080280F8422A8DF8A7
:10EA3000385023E09DF8080000EB4002C2EBC01004
:10EA400003EBC0029DF83800104442799DF808009D
:10EA500000EBC00707EB002001EBC0079DF810009A
:10EA600000EB401007EB80079DF83800384480F831
:10EA7000172F9DF83820521C8DF838209DF838004B
:10EA80000A28D7D38DF8385023E09DF8080000EB12
:10EA90004002C2EBC0109DF8382003EBC0001044C8
:10EAA000C27B9DF8080000EBC00707EB002001EBDC
:10EAB000C0079DF8100000EB401007EB80009DF8A8
:10EAC0003870384480F8302F9DF83800401C8DF89D
:10EAD00038009DF838000228D7D3DBE19DF8080004
:10EAE000F12200EBC00303EB002008EBC00191E72B
:10EAF0009DF80800032200EBC00303EB002001EBAC
:10EB0000C0039DF8100000EB401003EB800080F87C
:10EB1000D82EE3E79DF80820022002EBC20707EB9E
:10EB2000022201EBC2079DF8102002EB421207EB14
:10EB3000820282F8D80E9DF80800F62700EBC0028A
:10EB400002EB00209DF8102001EBC00002EB421206
:10EB500000EB820080F8DC7E9DF8080000EBC0022C
:10EB600002EB00209DF8102001EBC00002EB4212E6
:10EB700000EB820080F84A4F8DF8385023E09DF872
:10EB8000080000EB4002C2EBC0109DF8382003EBF8
:10EB9000C000104442799DF8080000EBC00707EB65
:10EBA000002001EBC0079DF8100000EB401007EBC0
:10EBB00080009DF83870384480F84B2F9DF838005D
:10EBC000401C8DF838009DF838000A28D7D361E141
:10EBD0009DF8080000EB4002C2EBC01003EBC00040
:10EBE00082799DF8080000EB4007C7EBC0100AEBE4
:10EBF000C000407942EA00229DF8080000EBC00303
:10EC000003EB002001EBC0039DF8100000EB401067
:10EC100003EB8000A0F8562F9DF8080000EBC0021F
:10EC200002EB002001EBC0029DF8100000EB401049
:10EC300002EB8000B0F8562F9DF8080000EB40036F
:10EC400003EB001001EB0010B0F82A0A8242BED399
:10EC50009DF80800F12200EBC00303EB002001EB5C
:10EC6000C0079DF8100000EB401007EB800080F813
:10EC7000DC2E9DF8080000EBC00202EB002008EB40
:10EC8000C0019DF8100000EB401001EB800090F8EF
:10EC9000581F21F0010180F8581FFBE09DF8080083
:10ECA000524600EB4001C1EBC0100AEBC0000079F6
:10ECB0008DF810008DF85450C14619E09DF80800F9
:10ECC00000EB400101EB00109DF8541009EB00101F
:10ECD00000EB011090F8410A9DF8101088429DF851
:10ECE000540002D18DF8100010E0401C8DF8540043
:10ECF0009DF8080000EB400101EB001009EB00104B
:10ED000090F8170A9DF854108842D7D89DF808004B
:10ED100000EB4001C1EBC01002EBC000C078ADF8C1
:10ED20001800BDF81800182812D2DFE800F0110C06
:10ED30000E118E8E868E881111118A8E8E8E8E8C7B
:10ED400011118E118E8E1A2000E00D208DF80C000E
:10ED50009DF80C00001FC1B29DF80800574600EB5B
:10ED60004003C3EBC0130AEBC300C01CFAF780FAE0
:10ED70008DF85C009DF8080000EB4001C1EBC0116C
:10ED800007EBC1009DF80C10084410F8010C9DF829
:10ED90005C1088427ED19DF8080000EB4001C1EB79
:10EDA000C01107EBC10138464978002972D09DF89F
:10EDB000081001EB4102C2EBC11100EBC1029DF84A
:10EDC0000C101144CA789DF8081001EBC10303EB45
:10EDD000012109EBC1039DF8101001EB411103EB78
:10EDE000810181F8142F9DF8081009EB01129DF89C
:10EDF0001010114481F8D059BDF81810CE293CF4F8
:10EE000082AC24DCB9293CF4B4AC7CF750A8C3290B
:10EE10007DD0C5297CF473A89DF8081001EB410250
:10EE200002EB011109EB011191F81C1A00299DF860
:10EE30000C106DD00E29ADD1FEE3072086E7082027
:10EE400084E70C2082E70A2080E706207EE7E1299C
:10EE5000D5D006DCD5293AD0D729A7D0D92999D140
:10EE60007CE2E5297CF459A889F860459DF8080002
:10EE700000EBC00101EB002009EBC0019DF8100080
:10EE800000EB401001EB800090F8D80E00289DF8B0
:10EE9000080000E0F0E200EBC00101EB00207CF490
:10EEA0008FAF09EBC00080F8D35E9DF8080000EB3F
:10EEB000C00101EB002009EBC0019DF8100000EB40
:10EEC000401001EB800080F8D84EFCF71CBC9DF888
:10EED000081001EB4102C2EBC11107EBC100C07881
:10EEE00089F862009DF8080000EB400101EB00107A
:10EEF0009DF8101009EB001000EB011099F862105A
:10EF0000A4EBD11290F8421A62F3000101E0F9E299
:10EF10005DE380F8421A9DF8080000EB400101EB28
:10EF200000109DF8101009EB001000EB011099F88B
:10EF300062104A0990F8421A62F3410180F8421ABD
:10EF40009DF8080000EB400101EB001009EB0011F7
:10EF50009DF8100001EB001090F8420AC0F3400148
:10EF60009DF8080000EBC00202EB002009EBC00294
:10EF70009DF8100000EB401002EB800090F8F00EBE
:10EF8000C0F34000814249D09DF808004A4600EB9A
:10EF9000C00101EB002009EBC0019DF8100000EB5F
:10EFA000401001EB80019DF8080000EB400303EBEB
:10EFB00000109DF8103009EB001000EB031090F8E2
:10EFC000420A430891F8F00E63F3410081F8F00E15
:10EFD0009DF8080000EB400101EB00109DF81010B7
:10EFE00002EB001000EB011090F8420A800716D5E2
:10EFF0009DF80800D92100EBC00303EB002009EBCA
:10F00000C0029DF8100000EB401002EB800080F879
:10F01000DC1E9DF808100220FAF79CFD42E09DF8E6
:10F02000080000EBC00101EB002002EBC0019DF8DD
:10F03000100000EB401001EB800080F8E54E9DF8D9
:10F040000800D92100EBC00303EB002002EBC00352
:10F050009DF8100000EB401003EB800080F8DC1EF0
:10F060009DF8080000EB400101EB001002EB0011DD
:10F070009DF8100001EB001191F8420A20F02003E6
:10F0800081F8423A9DF8080000EBC00101EB002036
:10F0900009EBC0019DF8100000EB401001EB80006F
:10F0A00080F8164F9DF8080000EB400101EB0010BE
:10F0B00009EB00119DF8100001EB001090F8420AD6
:10F0C00000F001019DF8080000EBC00202EB0020F7
:10F0D00009EBC0029DF8100000EB401002EB80002D
:10F0E00090F8F00E00F0010081426AD09DF808000F
:10F0F00000EBC00101EB00209DF8101009EBC000EF
:10F1000001EB411100EB81009DF8081001EB410279
:10F1100002EB01119DF8102009EB011101EB021126
:10F1200091F8421A90F8F02E61F3000280F8F02E68
:10F130009DF8080000EB400101EB00109DF8101055
:10F1400009EB001000EB011090F8420AC0073CF4F4
:10F1500065A89DF808004F4600EBC00101EB0020B8
:10F1600009EBC0019DF8100000EB401001EB80009E
:10F1700090F8160F00289DF8080000EBC00101EB85
:10F18000002009EBC0019DF8100000EB401001EBDE
:10F19000800017D080F8155F9DF8080000EB400153
:10F1A00001EB001007EB00119DF8100001EB0011BE
:10F1B00091F8420A20F0010281F8422A97F82106CC
:10F1C00018B1A7E080F8154FF8E7387D012865D120
:10F1D000786DF98A884261D29DF8080000EBC00181
:10F1E00001EB002007EBC0019DF8100000EB401080
:10F1F00001EB800090F8150F01284FD19DF8080011
:10F2000000EBC00101EB002007EBC0019DF81000EE
:10F2100000EB401001EB800090F8490FF0BB9DF827
:10F22000080000EB400101EB001007EB00119DF816
:10F23000100001EB001090F8401A9DF8080000EB58
:10F24000C00202EB002007EBC00080F8D11E9DF841
:10F250000800C32100EBC00202EB002007EBC00254
:10F260009DF8100000EB401002EB800080F8DC1EDF
:10F270009DF8080000EB400101EB001007EB0011C6
:10F280009DF8100001EB0010C0F8445A9DF80810DA
:10F290000220FAF75FFC8DF8385018E03AE09DF84C
:10F2A000080000EBC00101EB002007EBC0019DF856
:10F2B000100000EB401001EB80019DF8380008447D
:10F2C00080F8175F9DF83810491C8DF838109DF8AC
:10F2D00038001428E3D38DF8385017E09DF8080063
:10F2E00000EBC00101EB002007EBC0019DF810000E
:10F2F00000EB401001EB80009DF83810084480F8C6
:10F30000335F9DF83800401C8DF838009DF83800B8
:10F310000A28E3D39DF8080000EB400101EB001040
:10F320009DF8101009EB001000EB011090F8420A54
:10F3300080077CF53FA89DF80800D92100EBC002AA
:10F3400002EB002009EBC0029DF8100000EB40101A
:10F3500002EB800080F8DC1EFCF72CB89DF808104A
:10F3600001EB410202EB011109EB011191F81C1AAA
:10F3700000299DF80C1002D00A297DD193E00829BC
:10F380007AD18DF8385024E09DF8081001EB410245
:10F39000C2EBC1119DF8382000EBC1011144C978BE
:10F3A00001F00F01092918D89DF8081001EB41025E
:10F3B000C2EBC1119DF8382000EBC1011144C9789E
:10F3C00001F0F001902908D89DF83810491C8DF8FB
:10F3D00038109DF838100629D6D39DF83810062924
:10F3E0004AD39DF8081001EB4102C2EBC11100EBBA
:10F3F000C101C9780A049DF8081001EB4103C3EB71
:10F40000C11100EBC101097942EA01229DF80810FF
:10F4100001EB4103C3EBC11100EBC10149790A4380
:10F420009DF8081001EBC10303EB012109EBC103B7
:10F430009DF8101001EB411103EB8101C1F8F12E91
:10F440009DF8081001EB4102C2EBC11100EBC101B4
:10F4500089790A049DF8081001EB4103C3EBC1113F
:10F4600000EBC101C97942EA01229DF8081001EBC5
:10F470004103C3EBC11100E022E100EBC100007ABF
:10F4800002439DF8080000EBC00101EB002009EBEE
:10F49000C0039DF8100000EB401003EB8000C0F8A3
:10F4A000F52EFCF7F0B88DF8385025E09DF80810DF
:10F4B00001EB4102C2EBC1119DF8382000EBC10104
:10F4C0001144C97801F00F0109293CF672A89DF892
:10F4D000081001EB4102C2EBC1119DF8382000EB8E
:10F4E000C1011144C97801F0F0019029EDD89DF8CF
:10F4F0003810491C8DF838109DF838100829D5D3DC
:10F50000FCF757B89DF8080000EBC00101EB0020A4
:10F5100009EBC0029DF8100000EB401002EB8000E8
:10F5200080F8DC6E9DF8080000EBC00101EB0020C4
:10F5300009EBC00080F8D34E9DF8080000EB4001B5
:10F5400001EB00109DF8101009EB001000EB01100A
:10F5500090F8421A41F02002FCF7B1B90A799DF8FF
:10F56000081001EB4103C3EBC11107EBC100C078E8
:10F5700042EA0022FCF735B99DF8080000EBC00113
:10F5800001EB002009EBC00080F8D34E9DF8080085
:10F5900000EBC00101EB002009EBC0029DF8100058
:10F5A00000EB401002EB800080F8DC6E9DF8080054
:10F5B00000EB400101EB00109DF8101009EB00106A
:10F5C00000EB011090F8421A41F00402C4E70C2944
:10F5D00076D18DF8385024E09DF808109DF8383029
:10F5E00001EB4102C2EBC11100EBC102D118C97895
:10F5F00001F00F01092918D89DF8082002EB4203F9
:10F60000C3EBC21100EBC1029DF838101144C97858
:10F6100001F0F001902908D89DF83810491C8DF8A8
:10F6200038109DF838100A29D6D39DF838100A29C9
:10F6300046D30022134600E068E0CDE900222946C7
:10F640008DF838501EE0009A1B0243EA1263120242
:10F65000CDE900239DF8082002EB4203C3EBC21260
:10F660009DF8383000EBC2021A44D278DDE9003749
:10F670001A4341EA0703CDE900239DF83820521CC4
:10F680008DF838209DF83820052ADCD3DDE90037D5
:10F690009DF8082002EBC20C0CEB022209EBC20C15
:10F6A0009DF8102002EB42120CEB8202C2F8F93EE8
:10F6B000C2F8FD7E0023CDE900338DF8381020E03C
:10F6C000D1E0DDE900231B0243EA12631202CDE917
:10F6D00000239DF8082002EB4203C3EBC2129DF801
:10F6E000383000EBC2021A44127ADDE900371A43BF
:10F6F00041EA0703CDE900239DF83820521C8DF81C
:10F7000038209DF83820052ADBD399E08DF8385051
:10F7100024E09DF808109DF8383001EB4102C2EB5F
:10F72000C11100EBC102D118C97801F00F010929FC
:10F7300018D89DF8082002EB4203C3EBC21100EB7E
:10F74000C1029DF838101144C97801F0F0019029E8
:10F7500008D89DF83810491C8DF838109DF83810DD
:10F760000C29D6D39DF838100C297CD30022CDE982
:10F77000002229468DF83850BC461FE0DDE9000222
:10F78000120242EA10620002CDE900029DF8080070
:10F7900000EB4002C2EBC0109DF838200CEBC0001B
:10F7A0001044C078DDE90023104341EA0302CDE9AB
:10F7B00000029DF83800401C8DF838009DF8380094
:10F7C0000628DBD3DDE900239DF8080000EBC00725
:10F7D00007EB002009EBC0079DF8100000EB40107C
:10F7E00007EB8000C0F8F92EC0F8FD3E0022CDE9FD
:10F7F00000228DF838101FE0DDE90002120242EA13
:10F8000010620002CDE900029DF8080000EB400202
:10F81000C2EBC0109DF838200CEBC0001044407AB9
:10F82000DDE90023104341EA0302CDE900029DF81F
:10F830003800401C8DF838009DF838000628DBD3CE
:10F84000DDE900129DF8080000EBC00303EB002087
:10F8500009EBC0039DF8100000EB401003EB8000A3
:10F86000C0F8011F00E011E1C0F8052F9DF8080065
:10F8700000EBC00101EB002009EBC0019DF8100076
:10F8800000EB401001EB800090F8D81E9DF80800B6
:10F8900000EBC00202EB002009EBC00090F8D40E90
:10F8A00081427DD199F821064F46B8B19DF80800F4
:10F8B00000EB400101EB00109DF8101009EB001067
:10F8C00000EB011090F8421A41F0080280F8422A39
:10F8D0009DF808100220FAF73DF978E0C7F8355096
:10F8E0009DF8080000EBC00101EB002007EBC00110
:10F8F0009DF81000102200EB401001EB800101F692
:10F90000F9610798F8F79FFC9DF8080000EBC0012B
:10F9100001EB002007EBC0019DF8100000EB401048
:10F9200001EB8000D0F8F11EC7F81910D0F8F50EE1
:10F93000C7F81D009DF8080000EB400101EB001026
:10F9400007EB00119DF8100001EB001090F8400A41
:10F9500038769DF8080000EBC00101EB002007EBB2
:10F96000C0019DF8100000EB401001EB8000D0F8C2
:10F970000C0FC7F821006748D0F86812C7F8391093
:10F98000B0F86C02A7F83D00786D81B20220F9F75B
:10F99000CDFA00210620FAF7DDF8786D401C00E072
:10F9A00003E078650021052095E79DF8080000EB4D
:10F9B000400101EB00109DF8101009EB001000EB66
:10F9C000011090F8421A41F0040180F8421A9DF8A3
:10F9D000080000EBC00101EB002009EBC0019DF81D
:10F9E000100000EB401001EB800080F8165F9DF8DE
:10F9F000080000EBC00101EB002009EBC0019DF8FD
:10FA0000100000EB401001EB800080F8DC6E9DF8E8
:10FA1000080000EBC00101EB002009EBC0019DF8DC
:10FA2000100000EB401001EB800090F8D80E042885
:10FA30002CD19DF8080000EB400101EB00109DF86F
:10FA4000101009EB001000EB011090F8421A41F081
:10FA5000800180F8421A9DF8080000EBC00101EB1C
:10FA6000002009EBC00080F8D34E9DF80800052166
:10FA700000EBC00202EB002009EBC0029DF8100071
:10FA800000EB401002EB800080F8D81E98F8670267
:10FA9000A0B19DF8080008EB400000F50050B0F858
:10FAA000F01F9DF80800012300EB4002C2EBC012DA
:10FAB0000AEBC2009DF80820FAF70EFF8DF83850C7
:10FAC000514613E089F86055FBF71DBE9DF808000C
:10FAD00000EB4002C2EBC0109DF8382001EBC000E3
:10FAE00085549DF83800401C8DF838009DF838008A
:10FAF0001428EBD3084801784278114482781144E5
:10FB0000C278D1427BF4A9A819B0BDEC028BBDE844
:10FB1000F08F0000D41000200F0800202DE9F74FCF
:10FB20008EB04FF00008ADF80480ADF80080ADF85D
:10FB30000080ADF810808DF814808DF818808DF855
:10FB40001C80CDE90888CDE90888ADF83480FEA096
:10FB5000D0E90020CDE90220FDA0D0E90020CDE9C8
:10FB60000A20FD4880F804800E9800EB400202EB6A
:10FB70000010FA4A02EB0010814690F8160A8DF840
:10FB800014000E9802EB001000900844824690F892
:10FB9000D0290E9809EB011700EBC00303EB0020FE
:10FBA000EE4B042A03EBC00B01EB41130BEB830577
:10FBB0001ED105208AF8D00985F8D88E97F8420A18
:10FBC00020F0800087F8420A99F8162AA120072A17
:10FBD0000ED2DFE802F00D040B0B06080A00E52048
:10FBE00004E0B12002E0312000E0F12085F8DC0ED5
:10FBF0009DF814C00E9B10980222D94EC3EB03133C
:10FC0000A1384FF0410E03EB8304BCF1070F77D20C
:10FC1000DFE80CF07604F2F1F0EFEE0097F8410A1D
:10FC2000002101F031FD8DF8180095F8D81E9BF8E1
:10FC3000D40E814202D101218BF8D31E9AF8D0094B
:10FC4000401C8AF8D009109BA221A620CE2B7DD083
:10FC500012DC4FF0A502B92B79D006DCB22B77D09D
:10FC6000B52B35D0B62B4BD118E1C32B71D0C52B9A
:10FC700070D0CA2BF7D106E1E12B6CD006DCD52B76
:10FC800009D0D72B68D0D92BEDD10FE0E52B72D05E
:10FC9000E72BE8D132E2F52006F834009DF8180091
:10FCA00006EBC4056870A970D52009E0F52006F8B8
:10FCB00034009DF8180006EBC4056870A970D920BF
:10FCC000E8702846032101F010FC2871052009E2A4
:10FCD000F52106F834109DF8181006EBC40779706A
:10FCE00099F81C1A4FF0B50959B1D5F8E01EB1F1D9
:10FCF000104F39D34FF010410022CDE9081237E000
:10FD000086E2D5F8E00EB0F5100F05D34FF41000E1
:10FD10000021CDE9080103E0D5F8E00ECDE908089F
:10FD2000BA7040460FE0BDF80400C0F10200C20006
:10FD3000DDE90801F8F777FABDF804103944C87016
:10FD4000BDF80400401CADF8040006E040E12AE0E4
:10FD5000AFE08DE031E107E1DBE1BDF8040003280D
:10FD6000E1D387F80690E9E0D5F8E01ECDE9081860
:10FD7000B870404610E0B6E1BDF80400C0F10300E1
:10FD8000C200DDE90801F8F74EFABDF80410394465
:10FD9000C870BDF80400401CADF80400BDF80400B4
:10FDA0000428E9D362E0F52106F834109DF8181014
:10FDB00006EBC407797099F81C1A4FF0B90959B1CC
:10FDC000D5F8E01EB1F1104F34D0D5F8E01ECDE9E2
:10FDD0000818B870404643E0D5F8E00EB0F5100FB3
:10FDE0000BD0D5F8E00ECDE90808BA7040461AE00D
:10FDF000F7E3F7E3F7E3DCE296E14FF410000021CC
:10FE0000CDE90801F1E7BDF80400C0F10200C2002D
:10FE1000DDE90801F8F707FABDF804103944C870A5
:10FE2000BDF80400401CADF80400BDF80400032830
:10FE3000E9D396E74FF010410022CDE90812C8E758
:10FE4000BDF80400C0F10300C200DDE90801F8F7C5
:10FE5000EAF9BDF804103944C870BDF80400401C2C
:10FE6000ADF80400BDF804000428E9D348469CE03E
:10FE7000F52006F834009DF8180006EBC4056870FC
:10FE8000A970C3201CE7F52006F834009DF818007F
:10FE900006EBC4056870A970CA2011E7F52006F8C2
:10FEA00034009DF8180006EBC4056870A970B620F0
:10FEB00006E7F52006F834009DF8180006EBC407A5
:10FEC000787099F81C0AB22110B1BA7040462EE041
:10FED000A420B87040460EE0D5F80C0FBDF8042001
:10FEE000C2F10102D200D040BDF804203A44D070E3
:10FEF000BDF80400401CADF80400BDF80400022861
:10FF0000EAD379713846052101F0EFFAB8715FE163
:10FF1000D5F80C0FBDF80420C2F10202D200D04087
:10FF2000BDF804203A44D070BDF80400401CADF880
:10FF30000400BDF804000328EAD3B971384606214D
:10FF400001F0D3FAF8710DE0016932303130300040
:10FF500001693230453030000F080020D4100020F5
:10FF60000C4500200820BDE0F52106F834109DF86E
:10FF7000181006EBC4077970B87040460EE0D5F84B
:10FF8000100FBDF80410C1F10301C900C840BDF84D
:10FF900004103944C870BDF80400401CADF80400DA
:10FFA000BDF804000428EAD3E120F871384607219F
:10FFB00001F09BFA3872092094E0F52006F834002D
:10FFC0009DF8180006EBC4056870A970C52077E697
:10FFD000F52006F834009DF8180006EBC407787089
:10FFE00099F81C0A4FF0CE0918B1AE20B8704046FF
:10FFF00050E0AC20B870404611E0D5F8F90ED5F8C5
:020000040801F1
:10000000FD1EBDF80420C2F10402D200F8F70BF97E
:10001000BDF804103944C870BDF80400401CADF8A8
:100020000400BDF804000528E7D3404611E0D5F8E8
:10003000010FD5F8051FBDF80420C2F10402D2005B
:10004000F8F7F1F8BDF8041039440872BDF804005F
:10005000401CADF80400BDF804000528E7D387F87C
:100060000D9038460D2101F040FAB8730F2039E0A9
:10007000D5F8F90ED5F8FD1EBDF80420C2F1050231
:10008000D200F8F7D0F8BDF804103944C870BDF8B4
:100090000400401CADF80400BDF804000628E7D3B6
:1000A000404611E0D5F8010FD5F8051FBDF8042032
:1000B000C2F10502D200F8F7B6F8BDF804103944D1
:1000C0004872BDF80400401CADF80400BDF80400FF
:1000D0000628E7D387F80F9038460F2101F005FA7C
:1000E0003874112098E2F52006F834009DF81800C5
:1000F00006EBC4056870A970E520E1E5F52006F877
:1001000034009DF8180006EBC4056870A970E7205C
:10011000D6E5F52006F834009DF8180006EBC40576
:100120006870A970D720CBE597F8411A8DF81810A0
:1001300095F8D83E9BF8D41E8B4202D101238BF850
:10014000D33E9AF8D019491C8AF8D0199DF8181096
:1001500021B19DF81810491E8DF818100A2857D2A1
:10016000DFE800F02BEE4076D8EDEC05EB5706F813
:1001700034209DF8180006EBC4074030787087F8EB
:1001800002E03021F9703971352078713320B8716F
:100190003120F87139727972B9720320F872781CC3
:1001A0000B21F9F765F838730D20ADF8340095F898
:1001B000D80E04282CD1052028E0042206F834208B
:1001C0009DF8181006EBC4004031417051213AE10E
:1001D000072021E2287103206871681C0521F9F7C6
:1001E00047F8FCE3042206F834209DF8181006EBCB
:1001F000C4004031417080F802E00521C170ADF8C3
:10020000342095F8D80E0228D4D1032085F8D80ED2
:100210001EE106F834209DF8180006EBC4054030B6
:10022000687085F802E03120E870322028710320E0
:100230006871681C0521F9F71BF8A8710720ADF853
:10024000340097F8420A20F0200087F8420AFFE0C5
:1002500006F834209DF8180006EBC407403078708B
:1002600087F802E03121F97030203871D5F8E02E9E
:10027000B2F5100F00D23220787195F8DD0E01280A
:1002800003D095F8DD0E10B103E0B97101E0322022
:10029000B871ADF8048013E0D5F8E00EBDF8041095
:1002A000C1F105018900C840BDF8041000F00F003D
:1002B00039443030C871BDF80400401CADF804006A
:1002C000BDF804000628E7D332207873ADF8048027
:1002D00013E0D5F80C0FBDF80410C1F1030189003B
:1002E000C840BDF8041000F00F0039443030887366
:1002F000BDF80400401CADF80400BDF8040004285B
:10030000E7D30320B874781C1221F8F7B1FFF87412
:100310001420D0E306F834209DF8180006EBC4073B
:100320004030787087F802E03220F870312139715E
:100330007871B871ADF8048017E06CE04EE14EE1E1
:100340005BE0D5F80C0FBDF80410C1F10301890082
:10035000C840BDF8041000F00F0039443030C871B7
:10036000BDF80400401CADF80400BDF804000428EA
:10037000E7D3ADF80480302008E0BDF8041039441C
:10038000C872BDF80410491CADF80410BDF8041083
:100390001929F2D3032087F82400781C2421F8F7C8
:1003A00067FF87F82500262085E306EBC401487027
:1003B0004CE097F8411A8DF8181095F8D83E9BF844
:1003C000D41E8B4202D101238BF8D33E9AF8D01968
:1003D000491C8AF8D0199DF8181021B19DF8181001
:1003E000491E8DF818100A2832D2DFE800F0050601
:1003F000224EF9F8F7311432DFE606F834209DF882
:10040000180006EBC4054030687085F802E0312022
:10041000E8703520DEE606F834209DF8180006EB7B
:10042000C4054030687085F802E03220E870302062
:10043000D0E6042206F834209DF8181006EBC4001C
:1004400040314170714681700521C170ADF8342092
:1004500033E306F834209DF8180006EBC40540305D
:10046000687085F802E03120E8703220287103209E
:100470006871681C0521F8F7FBFEA87197F8420A1D
:1004800020F0200087F8420AA2E606F834209DF802
:10049000180006EBC4074030787087F802E031217D
:1004A000F97087F804E0D5F8E00EB0F1104F09D0EC
:1004B0003220787195F8DD0E012805D095F8DD0E13
:1004C00020B105E03020F4E7B97101E03220B871C5
:1004D000ADF8048013E0D5F8E00EBDF80410C1F1CA
:1004E00007018900C840BDF8041000F00F0039442E
:1004F0003030C871BDF80400401CADF80400BDF8F0
:1005000004000828E7D33220F873ADF8048013E024
:10051000D5F80C0FBDF80410C1F105018900C840E1
:10052000BDF8041000F00F00394430300874BDF8F5
:100530000400401CADF80400BDF804000628E7D311
:100540003020B875ADF8048008E0BDF804103944D7
:10055000C875BDF80410491CADF80410BDF80410AE
:100560000629F2D37877ADF8048008E0BDF80410CE
:1005700039448877BDF80410491CADF80410BDF863
:1005800004100629F2D387F82400ADF8048009E0AE
:10059000BDF80410394481F82500BDF80410491C49
:1005A000ADF80410BDF804100629F1D387F82B002C
:1005B000ADF8048009E0BDF80410394481F82C003E
:1005C000BDF80410491CADF80410BDF8041006294C
:1005D000F1D387F83200ADF804800FE06AE064E000
:1005E0001BE0B0E13BE16AE0BDF80410394481F85A
:1005F0003300BDF80410491CADF80410BDF8041018
:100600000629F1D3032087F83900781C3921F8F73F
:100610002FFE87F83A003B204DE206F834209DF883
:10062000180006EBC4074030787087F802E03220EB
:10063000F8703121397133217971B871ADF80480C6
:1006400013E0D5F80C0FBDF80410C1F105018900C5
:10065000C840BDF8041000F00F0039443030C871B4
:10066000BDF80400401CADF80400BDF804000628E5
:10067000E7D3ADF80480302108E0BDF80400384429
:100680004173BDF80400401CADF80400BDF804003F
:100690001928F2D3032087F82600781C2621F8F7C2
:1006A000E7FD87F82700282005E2102006F834002F
:1006B00030207AE6102006F83400312075E697F8ED
:1006C000410A8DF81800BDF8040000EB40100BEB58
:1006D000800090F8D82E9BF8D40E824202D10122DD
:1006E0008BF8D32E9AF8D009401C8AF8D009ADF8BF
:1006F00004800EE0BDF8042009EB021090F8410AD6
:100700009DF8182090420AD0BDF80400401CADF8B6
:10071000040099F8170ABDF804209042EAD8BDF801
:10072000042009EB021090F8400A081A401C8DF8CA
:100730001C009DF8180020B19DF81800401E8DF88F
:10074000180095F8D90E0F2805D295F8D90E401C3F
:1007500085F8D90E01E085F8D98E1099FA27652021
:10076000B13909297AD2DFE801F0050C44797964BE
:10077000791E30009DF81800503006F83400202112
:1007800066E09DF81800503006F8340095F8D90E50
:1007900006EBC40540F0300068700120A870E870D6
:1007A00085F8048036E09DF81810503106F83410B2
:1007B00095F8D91E06EBC40541F030016970A870A8
:1007C0000120E8709DF81C0023E09DF818105031BE
:1007D00006F8341095F8D91E06EBC40541F0300137
:1007E0006970A8700120E8709DF81C0040F01000AE
:1007F0000FE09DF81800503006F8340095F8D90E37
:1008000006EBC40540F0300068700120A870E87065
:100810000520287128460521F9F7F2F8CDE90808E6
:1008200068710898000AA8710320E8712F72FFF719
:10083000C2BB95F8DA0E85F8DC0E85F8DA8E9DF8E5
:100840001800503006F8340095F8D90E40F0C00179
:1008500006EBC4004170877003202CE189E0BDF8ED
:1008600004300098184490F8D0395B1C80F8D039D7
:1008700099F81C0A30B1491CC9B2012834D00228A9
:1008800077D143E01098312802D0452871D115E086
:10089000ADF8048002A90CE0BDF80400BDF80430F6
:1008A00006EBC402085CD054BDF80400401CADF84F
:1008B0000400BDF804000728EED389E4ADF80480F5
:1008C0000AA90CE0BDF80400BDF8043006EBC40230
:1008D000085CD054BDF80400401CADF80400BDF81D
:1008E00004000728EED373E48DF818109DF8180063
:1008F00006F8340006EBC4050320687085F8028012
:10090000EA7085F804800920687110E08DF81810ED
:100910009DF8180006F8340006EBC4050320687043
:1009200085F8028085F8038085F804806A7128467E
:100930000621F8F76FFECDE90808000AE87108986B
:10094000A871FFF700BBF34A9AF8D009401C8AF857
:10095000D00997F8410A8DF8180010980621F3285D
:1009600075D007DC052873D0F12808D0F22800D113
:1009700013E06FE0F4286CD0F6286BD1D3E0F520BB
:1009800006F834009DF8180006EBC405687085F879
:1009900002800520E870F120F6E0F52006F834002A
:1009A0009DF8180006EBC407787087F80280F220E3
:1009B000387195F8480F787195F8480F012812D0D2
:1009C00095F8480F20285AD0ADF83410BDF83400FF
:1009D000F8703846BDF83410F8F71CFE00E0DDE092
:1009E000CDE9080842E12520ADF834004146ADF8D4
:1009F00004800DE0BDF80400284490F8210FBDF8F4
:100A000004203A449071BDF80400401CADF8040085
:100A1000BDF804000F28EDD3ADF804100DE0BDF8CB
:100A20000400284490F8330FBDF804203A44507570
:100A3000BDF80400401CADF80400BDF804000A280D
:100A4000EDD395F8420FF877ADF8041012E03FE0CF
:100A5000A6E08CE031E0BDF80400284490F8430F94
:100A6000BDF80410394481F82000BDF80400401C92
:100A7000ADF80400BDF804000528ECD3A6E70A2071
:100A8000ADF8340040460BE0BDF80400284490F86F
:100A9000430FBDF8041039448871BDF80400401CB0
:100AA000ADF80400BDF804000428EDD38EE74870CB
:100AB000BDF83400801CADF834009748974D0E996E
:100AC00081B301297DD002297CD003297BD101E1AA
:100AD000F52006F834009DF8180006EBC40778707E
:100AE000404687F80280F321397195F8481F7971E3
:100AF0000C21ADF8341095F8421FB9710BE0BDF828
:100B00000400284490F8430FBDF804103944C8711C
:100B1000BDF80400401CADF80400BDF80400052831
:100B2000EDD353E7ABE0ADF83410F52006F8340010
:100B30009DF8180006EBC405687085F80280BDF8C2
:100B40003400E870F620287197F8480A6871284642
:100B5000BDF83410F8F75EFDCDE90808BDF8341093
:100B6000000A6854BDF83410089829449FE7F5201E
:100B700006F834009DF8180006EBC405687085F887
:100B800002800520E870F420287128460521F8F736
:100B900041FDCDE90808000A68710898A87173E45E
:100BA00040F21320ADF83400F52006F834009DF82B
:100BB000180006EBC4077870BDF83400000AB8705E
:100BC00002E06AE076E094E0BDF83400F8700520B9
:100BD000387140460CE0BDF8041009EB010090F8B4
:100BE0001E0ABDF8041039444871BDF80400401CC9
:100BF000ADF80400BDF804000A28ECD3B9F82A0ABD
:100C00009246000AF873B9F82A0A3874B5F8560FF4
:100C1000000A7874B5F8560FB874B5F8561F0E98D8
:100C200001EB802081B20320F8F714F94546ADF8B6
:100C3000048050464FF400720DE0BDF804100144EA
:100C400091F86610BDF804303B44D974BDF8041027
:100C5000491CADF80410BDF804109142EDD338469C
:100C6000BDF83410F8F7D6FCCDE90805BDF834100E
:100C7000000A7854BDF834100898394417E7BDF8D5
:100C80003410B1B38021F9F770FBBDF83400C5F81A
:100C9000A40022480121A03029E0BDF8341041B35E
:100CA0000821F9F762FBBDF8340068671B48012191
:100CB00070301CE0BDF83400D8B14FF48071184892
:100CC000F9F753FBBDF83400C5F8BC001348012107
:100CD000B8300CE0BDF8341059B14FF48061F9F729
:100CE00044FBBDF83400E8650C4801215830F8F7A2
:100CF000E7FC084890F86702002807D006EBC4001C
:100D00000023BDF834100E9AF9F7E6FD11B0BDE8E6
:100D1000F08F0000D4100020000C02400060024060
:100D2000000002402DE9F04700242DED048B8046A1
:100D300089469FED1E9B25462646E20040464946D1
:100D4000F7F771FAC7B22046F7F739FC41EC110BFF
:100D5000B0EE490AF0EE690A06F046FD380907F0E0
:100D60000F0100EB8000B0EE408AF0EE608A01EBEC
:100D70004000F7F724FC53EC182BF7F73FFB41EC4E
:100D8000180B28463146F7F727FC53EC182BF7F7DA
:100D90008EFAF7F74CFC641CE4B205460E46082CAC
:100DA000CBD3BDEC048BBDE8F08700000000000051
:100DB0000000594070B50F4D40F2244421462846AA
:100DC00006F0AFF9012813D1298828462A1D118879
:100DD000214606F043F90849012081F871090748C6
:100DE000D0F88C0001F50051C0F57A70A1F8F80F29
:100DF00070BD000000440040D4100020006002409C
:100E000010B50C4C40F22441204606F08AF9012826
:100E10000ED12088201D00880749012081F87D0916
:100E20000648406C01F50051C0F57A70A1F8FA0F40
:100E300010BD0000004C0040D410002000600240B3
:100E400010B50B4C40F22441204606F06AF9012807
:100E50000DD12088A0880749012081F8890906481A
:100E6000406901F50051C0F57A70A1F8FC0F10BD82
:100E700000500040D41000200060024010B50C4C1F
:100E800040F22441204606F04CF901280ED120887A
:100E9000201D00880749012081F895090648C06A8D
:100EA00001F50051C0F57A70A1F8FE0F10BD0000E9
:100EB00000480040D41000200060024010B5124CE1
:100EC00010492046F8F7E6FB00212046F8F7F8FB2A
:100ED0000E4C4021204606F01DF90028F9D0802153
:100EE0000B48F9F744FA084C0A49183C2046F8F731
:100EF000D1FB01212046F8F7E3FB074901200871E7
:100F000010BD000000802020A0600240004400408E
:100F1000000C0240008800200F08002010B5124C81
:100F200010492046F8F7B6FB00212046F8F7C8FB29
:100F30000E4C4021204606F0EDF80028F9D008219B
:100F40000B48F9F714FA084C0A49303C2046F8F7E8
:100F5000A1FB01212046F8F7B3FB074901200871E6
:100F600010BD00002080002070600240004C004056
:100F7000000C0240008020100F08002010B5124C19
:100F800010492046F8F786FB00212046F8F798FB29
:100F90000E4C4021204606F0BDF80028F9D04FF451
:100FA00080710B48F9F7E3F9074C0A49A83C204641
:100FB000F8F770FB01212046F8F782FB0649012073
:100FC000087110BD00800028B86002400050004049
:100FD00000000240208000100F08002010B5124CC5
:100FE00010492046F8F756FB00212046F8F768FB29
:100FF0000E4C4021204606F08DF80028F9D04FF421
:1010000080610B48F9F7B3F9074C0A49303C204698
:10101000F8F740FB01212046F8F752FB0649012072
:10102000087110BD00800018586002400048004060
:10103000000C0240008800100F0800202DE9F04746
:10104000012190B0480503F091FF8648F8F742FB74
:10105000402738010024CDE90540C50107940894D4
:10106000CDE9094546040C940D94DFF8FC917F48C6
:101070000B94CDE90207CDE9006969460E947948E1
:10108000F8F7D0FB012210217648F8F7B5FBDFF81E
:10109000D4A1AAF1180A5046F8F71CFB4FF47A784D
:1010A000CDE90348E811CDE9054007940894CDE95E
:1010B00009456F480B940C940D9400960E94CDE95D
:1010C000019069465046F8F7ADFB01215046F8F70C
:1010D000F7FADFF890A1AAF1300A5046F8F7FAFAC9
:1010E000E811CDE9054007940894CDE909450C9431
:1010F0000D94DFF8809160480B94CDE90207CDE9AB
:10110000006969460E945046F8F78CFB01221021C5
:101110005046F8F771FBDFF84CA1AAF1600A50467F
:10112000F8F7D8FACDE90348E811CDE9054007946E
:101130000894CDE9094551480B940C940D94009600
:101140000E94CDE9019069465046F8F76BFB0121FA
:101150005046F8F7B5FADFF80CA10AF1180A504624
:10116000F8F7B8FAE811CDE9054007940894CDE9FD
:1011700009450C940D94DFF8089142480B94CDE991
:101180000207CDE9006969460E945046F8F74AFB1C
:10119000012210215046F8F72FFBDFF8C8A0AAF172
:1011A000900A5046F8F796FACDE90348E811CDE9E0
:1011B000054007940894CDE9094533480B940C94F5
:1011C0000D9400960E94CDE9019069465046F8F7CB
:1011D00029FB01215046F8F773FADFF88890A9F14E
:1011E00048094846F8F776FA0397E811CDE9054033
:1011F00007940894CDE9094525480B940C940D9467
:10120000224F00960E94CDE9017069464846F8F7E2
:1012100009FB012210214846F8F7EEFADFF8449066
:10122000A9F178094846F8F755FACDE90348E811DD
:10123000CDE9054007940894CDE9094515480B947C
:101240000C940D9400960E94CDE9017069464846C1
:10125000F8F7E8FA01214846F8F732FA10B0BDE88D
:10126000F0870000A0600240044400400C450020CC
:101270006C4E0020044C0040644700205452002073
:1012800004500040BC4900203C5600200448004067
:10129000144C0020245A00202DE9FC41012108466D
:1012A00003F064FE0121042003F060FE0121082008
:1012B00003F05CFE0121402003F058FEDFF8FC80C3
:1012C000072205214046F9F739F807220621404652
:1012D000F9F734F8072208214046F9F72FF80722DA
:1012E00009214046F9F72AF8354F08220A213846E5
:1012F000F9F724F808220B213846F9F71FF80822DD
:1013000002214046F9F71AF808220C213846F9F76D
:1013100015F802268DF8056000244FF459708DF8F9
:101320000640012500908DF807508DF8046069464D
:101330004046F8F7C7FF8DF805604FF4E0508DF890
:10134000064000908DF807508DF8046069463846D5
:10135000F8F7B8FF4FF4916000908DF806408DF8D3
:10136000045069464046F8F7ADFF280200908DF81A
:1013700006408DF8045069461248F8F7A3FF8DF82F
:1013800006404FF4F040104C00908DF80450694630
:101390002046F8F797FFA9032046F8F7E6FF690310
:1013A0002046F8F7E2FFA1142046F8F7DEFFE1142B
:1013B0002046F8F7DAFFBDE8FC810000000C02408F
:1013C00000080240000002400018024070B50024EE
:1013D000FFF762FFFFF732FE00F022F80E4D00210A
:1013E00085F86C19012285F86C290C480170817010
:1013F0004170C2704FF47A718160042085F86C09E5
:1014000004E0204600F062F9641CE4B295F86C092F
:10141000A042F6D870BD0000D4100020104100207A
:10142000F8B511208DF8000002258DF80150012437
:101430008DF802408DF80340684600F0EBFA262054
:101440008DF800008DF8014000268DF802608DF8BF
:101450000340684600F0DEFA0E208DF800008DF89B
:1014600001508DF802408DF80340684600F0D2FA32
:1014700027208DF800008DF801408DF802608DF86E
:101480000340684600F0C6FA0F208DF800008DF882
:1014900001508DF802408DF80340684600F0BAFA1A
:1014A00034208DF800008DF801408DF802608DF831
:1014B0000340684600F0AEFA2F208DF800008DF84A
:1014C00001508DF802408DF80340684600F0A2FA02
:1014D00035208DF800008DF801408DF802608DF800
:1014E0000340684600F096FAF8BD01B9102110F8E3
:1014F000012B10F8013B491E5A400904090CF8D190
:1015000002F07F00704700002DE9FF5F14460F4690
:101510004FF480564FF480684FF4C0694FF00C0AC6
:1015200040F2244B002580B1012830D0022851D050
:10153000032871D10121880403F03CFD0097012CA0
:101540006DD0022C70D094B377E00121480403F0F1
:1015500031FD0097012C03D0022C06D054B10DE0D0
:10156000ADF80460ADF8088008E0ADF80460ADF8AF
:10157000089003E0ADF80450ADF80850ADF80650FF
:10158000ADF80C50ADF80AA069463B4C5DE0012176
:10159000C80403F00FFD0097012C03D0022C07D0E4
:1015A0005CB10EE0ADF80460ADF8088009E040E001
:1015B000ADF80460ADF8089003E0ADF80450ADF864
:1015C0000850ADF80650ADF80C50ADF80AA06946C9
:1015D0002A4C3AE00121080503F0ECFC0097012CAD
:1015E00003D0022C06D054B10DE0ADF80460ADF884
:1015F000088008E0ADF80460ADF8089003E0ADF8AD
:101600000450ADF80850ADF80650ADF80C50ADF8E8
:101610000AA069461A4C18E02CE000E004E0ADF89E
:101620000460ADF8088008E0ADF80460ADF80890FB
:1016300003E0ADF80450ADF80850124CADF8065078
:10164000ADF80C50ADF80AA06946204605F0A0FDA3
:101650000121204605F005FD01225946204605F0EE
:101660007FFD1021204605F0F9FC0122C021204613
:1016700005F001FDBDE8FF9F00440040004C004024
:1016800000500040004800402DE9FC410024CDE915
:1016900000446F4664220023F6F794FD0E4605468B
:1016A000104619460A220023F6F78CFD010102F0CC
:1016B0000F000818385504F10104E4B228463146F9
:1016C000082CE7D3DDE90001BDE8FC812DE9F05FDE
:1016D000644F4FF0040A0646002587F86CA900EB1A
:1016E000460000EB061007EB001494F81D0A0128D1
:1016F00003D10021304600F0B7F806EB4602B846A9
:1017000007EB82074FF0000B87F870B987F872B9C2
:1017100087F871B987F873B94FF00509C7F8789958
:1017200087F8A0B987F8A2B9012087F8A10987F83E
:10173000A309D4F8180A00EB80004000C7F8A809F4
:1017400094F8152AD4F8101A3046FFF7DDFE94F805
:10175000160A06EBC601434A01EB062102EBC1065D
:10176000072815D2DFE800F01404060A0C0E180052
:10177000484600E00F2086F8D40E09E00720FAE77B
:101780005046F8E7D4F8180A64214843C7F8A80976
:101790004FF0A10AC1465EE00320ECE705EB4510DF
:1017A00006EB800080F8E4BE012380F8E63E80F876
:1017B000E5BE80F8E7BE4FF47A73C0F8EC3E04EB68
:1017C000051383F842BA80F8D8BE94F8161A072990
:1017D0003FD2DFE801F03E0408080A0C0E00E521C4
:1017E00080F8DC1E35E05146FAE7B121F8E73121F7
:1017F000F6E7F12180F8DC1E002125E001EBC107AE
:1018000007EB012701EB410C02EBC7070CEB011CB6
:10181000002009EB0C1211E002EB001C9CF840CAFE
:1018200093F8488AC44507D193F840CA00EB4018A2
:1018300007EB880888F849CF401CC0B292F817CA55
:101840008445E9D8491CC9B299F86C094A468842CE
:10185000D4D86D1CEDB294F8170AA8429ED8BDE802
:10186000F09F0000D41000202DE9F04105466148AA
:101870004FF48042531006685F488414C71439B18E
:10188000C5B1012D18D0022D18D0032D1BD117E0A2
:1018900035B1012D06D0022D06D0032D13D105E060
:1018A000114604E0194602E0214600E03946F8F707
:1018B0005EFD08E0114604E0194602E0214600E022
:1018C0003946F8F752FD642007F0E2F800224FF4A1
:1018D00016512846FFF718FEDFF8208105EB45007A
:1018E00008EB8000002280F8A229C0F8A42905EBAB
:1018F000450000EB051008EB0011D1F8183A08F587
:1019000040504364012380F83D3091F8161A3C4C56
:10191000962305EB8500204406290AD2DFE801F072
:10192000090305050733762102E0837001E06E218B
:101930008170C5EB0511334B01EB8101C02403F825
:10194000314003EBC10462700821A170E27006F01F
:101950000F0105EB05121144217180786071202080
:10196000A071E171802020724C2060725420A0721E
:101970002548264F0B2645B1012D0FD0022D24D02E
:10198000032D14D12CE06621D2E78021F8F7EDFC7D
:10199000C7F8A4601D480121A03006E00821F8F72F
:1019A000E4FC7E67194801217030F7F789FE98F84A
:1019B000670228B1204600232A460B21F8F78CFF46
:1019C000BDE8F041642007F063B84FF4807110481F
:1019D000F8F7CBFCC7F8BC600C480121B830E4E74D
:1019E0004FF48061F8F7C1FCFE65084801215830CA
:1019F000DBE70000187AFF1F00180240D410002017
:101A00000C5E00200C450020000C024000600240EB
:101A10000000024030B50F23C27801780125FAB1E9
:101A2000144A126801F1E02102F4E062C2F5E062BA
:101A3000C2F30722C2F10404D3404278A240847862
:101A40001C401443220181F80024007800F01F019B
:101A50008D404009800000F1E020C0F8005130BD09
:101A600001F01F0085404809800000F1E020C0F827
:101A7000805130BD0CED00E0024A114001430248A4
:101A80000160704780FFFF1F08ED00E0BFF34F8F3C
:101A900004480168044A01F4E06111430160BFF3A6
:101AA0004F8FFEE70CED00E00400FA0510B50021B1
:101AB000074B0A46002003EBC004401CC0B262542E
:101AC0008028F8D3491CC9B20829F3D310BD0000FF
:101AD0000F6800202DE9FE4F0026171A8146701E60
:101AE0003546A3EB010A8846002F02DD4FF00101C5
:101AF00002E003D14FF00001019102E0C7F10007BD
:101B00000190BAF1000F02DD4FF0010002E003D1B5
:101B10004FF00000009002E0C7F1000A009050462C
:101B2000574501DD3C4600E00446601C4FF0000BC9
:101B3000029016E008F0FF0109F0FF000C9A00F097
:101B400015F83E445544A64202DD0199361B8944EE
:101B5000A54202DD00992D1B88440BF101001FFAFC
:101B600080FB02998B45E5DBBDE8FE8F30B5CC08E4
:101B700001F0070301259D40EBB2064D05EBC005C2
:101B8000C808285C0AB1184302E063EA0000C043B9
:101B9000285530BD0F6800202DE9FC4101210A20A5
:101BA00003F0E4F901248DF8044000264FF4C050FE
:101BB0008DF80660032700908DF805708DF80740BA
:101BC00069464648F8F77EFB8DF804408DF80660BC
:101BD0008DF80570A5028DF80740414C00956946C7
:101BE0002046F8F76FFBC82006F052FF2946204632
:101BF000F8F7BBFBC82006F04BFF29462046F8F754
:101C0000B6FBC82006F044FF0021FD2000F024FAB6
:101C10000021122000F020FA0021AE2000F01CFA72
:101C20000021D52000F018FA0021A02000F014FABD
:101C30000021A82000F010FA00213F2000F00CFA4B
:101C40000021D32000F008FA0021084600F004FA31
:101C50000021402000F000FA0021A02000F0FCF953
:101C60000021C02000F0F8F90021DA2000F0F4F99A
:101C70000021122000F0F0F90021812000F0ECF9A1
:101C800000217F2000F0E8F90021D92000F0E4F9DC
:101C90000021822000F0E0F90021DB2000F0DCF9D7
:101CA0000021342000F0D8F90021A42000F0D4F95C
:101CB0000021A62000F0D0F90021202000F0CCF96E
:101CC0000021084600F0C8F9FFF7F0FE0021AF2020
:101CD00000F0C2F900F054F8BDE8FC81000C0240AD
:101CE000000402400346012000E05843491EC9B2E7
:101CF000FBD270472DE9F84F82460A980D465043B3
:101D00006421B0FBF1F0984600F0FF0B4FF00109A1
:101D10000AEB02072B4600245046FAB21946CDF8CA
:101D20000090FFF7D7FE05EB0806F3B2FAB2F1B266
:101D30005046CDF80090FFF7CDFE5246F3B229464B
:101D40001046CDF80090FFF7C5FEF3B2FAB2F8B234
:101D50002946CDF80090FFF7BDFE4F460AEB0B0673
:101D600009E02819C3B2C1B2F2B250460097FFF79A
:101D7000B1FE641CE4B24445F3D3BDE8F88F000023
:101D800070B50025B020294600F066F9002108460C
:101D900000F062F90021102000F05EF9084E0024E6
:101DA00006EBC4000121405D00F056F9641CE4B26A
:101DB000802CF5D36D1CEDB2082DF0D370BD000062
:101DC0000F68002070B50B4C05460221204603F039
:101DD00097FA0028F9D02946204603F09AFA012103
:101DE000204603F08DFA0028F9D0204603F08FFA40
:101DF000C0B270BD003800402DE9FC4F1D4688463A
:101E000081468B460090082B0ED0680700D0012039
:101E100000EBD500690810FB01F0C0B2203A02F0D7
:101E2000FF0A0026019046E00620F7E7082D10D0B3
:101E30000C2D14D0102D16D0182D3FD121490AEBAE
:101E4000CA0001EB80000027845DE0070FD00B9AE9
:101E500010E01D490AEB4A0001EB4000F3E70AEBF2
:101E60004A001A49EDE71A4901EB0A10EBE70B9813
:101E700030B3002241464846FFF778FE7F1C6408D5
:101E800008F10100FFB200F0FF08082FDDD309F1CF
:101E9000010000F0FF09082D0AD00099A9EB01000C
:101EA000B0EB550F04D10BF10800894600F0FF0B91
:101EB000761CD846F6B201988642B7D3BDE8FC8FAF
:101EC0000122D7E710A3010884960108AC98010805
:101ED000209D01082DE9F84F1D00DDE90A799246A1
:101EE0008B4680464FF0000611D11046F6F767FB8F
:101EF00041EC100B05F0E0FB9FED1C1B51EC100BAF
:101F000053EC112BF6F7D3F9F6F772FBC5B2082F95
:101F100000D1022600241CE0281B401EC1B20A206A
:101F2000FFF7E0FEBAFBF0F00A21B0FBF1F201FB93
:101F30001200CDF8009088B13030C2B206EB5701E4
:101F400001FB0480C0B23B465946FFF755FF641CB5
:101F5000E4B2AC42E0D32846BDE8F88F06EB570167
:101F600001FB0480C0B23B463022EDE700000000D8
:101F70000000F03F2DE9FF4F81B0064600900F466C
:101F80004FF0000A8946580700D0012000EBD3002B
:101F90000490002032E0002029E00E98002410F880
:101FA0000A500AF101001FFA80FAE80701D00F9ADF
:101FB00002E00F9848B3002239463046FFF7D6FDBD
:101FC0007F1C641C6D08E4B2FFB2082CEDD3761CB4
:101FD0000098F6B2311A0398814204D109F1080041
:101FE000009E00F0FF0908F101004F46C0B20399BE
:101FF00080468842D1D30BF10100C0B204998346D8
:102000008842C8D305B0BDE8F08F0122D4E72DE99E
:10201000F8431D46DDE908781646894604460EE079
:102020003B4649462046CDF80080FFF7E5FE082FE5
:102030000ED004EB5700C4B26D1EEDB2761C002D1D
:1020400004D03278202A01D37E2AE9D9BDE8F8836A
:10205000A41DE4B2F0E700002DE9F041114C064662
:102060004FF4006500292946204602D0F8F77FF991
:1020700001E0F8F77AF94FF4805739462046F8F72F
:1020800074F939460848F8F772F93046FFF79AFEB6
:1020900039462046F8F76BF929462046BDE8F0415D
:1020A000F8F765B9000C0240000402402DE9F04F3A
:1020B00087B00027ADF80C70ADF80470ADF808706B
:1020C000ADF81470ADF81070ADF800704FF0F20B71
:1020D0004FF0A30AFD4EDFF8F883FDE391F82306E5
:1020E000022802D10720ADF80000BDF800003044FE
:1020F0008079BDF800203244D27840EA0260BDF811
:10210000002032441279BDF80030120433445B7968
:1021100042EA03221043EF4A5368984279D0506054
:10212000BDF8000030448078BDF800203244527879
:1021300040EA0225B1F8EA24BDF800002844801CDA
:10214000824266D30846B1F8EA14BDF80020491B64
:10215000891A891EA0F8EA14BDF800002946304407
:10216000F7F758FABDF80010294431444978BDF812
:1021700000202A44B25C41EA022181427AD1BDF8B2
:1021800000003044007900F001000490BDF8000028
:10219000304480790024C0F34209EB1F0FE0BDF802
:1021A000000020443044C0794A460499F7F73EFCC9
:1021B000BDF8001021443144C871641CA4B29C4293
:1021C000EDDB98F8670240B1A81C81B2BDF80000B1
:1021D000012330440422F8F77FFBBDF800003044AF
:1021E000C079012188F821164FF00009C8F8289518
:1021F00088F82695B84A82F83290C2F83490ADF843
:10220000149011287ED00DDCA0F10B00062815D209
:1022100000E0FCE3DFE810F007086D08A5089F0860
:102220009F0A1D00A2286FD004DC12286DD0A128BF
:1022300004D1F5E2A32869D0A42868D0002049463B
:10224000BDF800200244B154401C80B20528F7D3E9
:10225000F2E3ADF80C904446D2E1BDF80C0000EB7F
:10226000400101EB001004EB001090F8160A07285B
:102270007DD200E0F3E3DFE800F07A040404047A9E
:102280009B00484682E0BDF80000BDF814100844E9
:102290003044007AB8B3012802D002286ED112E08F
:1022A000BDF80C0000EB400101EB0010BDF804107C
:1022B00004EB001000EB011090F8421A21F0040129
:1022C00080F8421A5AE0BDF80C0000EB400101EB27
:1022D0000010BDF8041004EB001000EB011090F8A2
:1022E000421A21F0080180F8421ABDF80C0000EBF8
:1022F000400202EB0010BDF8042004EB001000EBDC
:10230000021005E0FDE339E0FCE3FCE3FCE3FCE361
:10231000C0F8449ABDF80C100220F7F71BFC00200F
:102320004A46BDF80C1001EBC10303EB012104EB9D
:10233000C103BDF8041001EB411103EB810101441D
:1023400081F8172F401C80B21428EAD30020BDF872
:102350000C1001EBC10303EB012104EBC103BDF839
:10236000041001EB411103EB8101014400E042E163
:1023700081F8332F401C80B20A28E8D3BDF814003E
:10238000401CADF81400BDF80400401CADF804007A
:10239000BDF80C0000EB400101EB001004EB001055
:1023A00090F8170ABDF8041088423FF66CAF22E19E
:1023B000CC46ADF804900FE1BDF80000BDF8141054
:1023C00008443044007A042805D005DC58B10128BF
:1023D00040D0022878D11BE1082876D010287DD083
:1023E000202871D1C1E1BDF80C0000EBC00101EB68
:1023F000002004EBC001BDF8040000EB401001EB2D
:10240000800090F8480F102820D1BDF80C0000EB98
:10241000C00101EB002004EBC001BDF8040000EB9B
:10242000401001EB800080F848CFBDF80C00F3218C
:1024300000EBC00202EB002004EBC002BDF8040078
:1024400000EB401002EB800080F8DC1EBDF81400A9
:10245000401CBAE0BDF80C0000EBC00202EB00200B
:1024600004EBC002BDF8040000EB401002EB80005A
:1024700080F8DCBEBDF80C0000EB400101EB001061
:10248000BDF8041004EB001000EB011090F8421AA4
:1024900021F0080180F8421ABDF80000BDF81410C0
:1024A00008443044017ABDF80C0000EBC00202EB96
:1024B000002004EBC002BDF8040000EB401002EB6A
:1024C000800080F8481F0AE081E0A1E0205E002043
:1024D000D410002014080020D4400020D2E00020B6
:1024E000BDF80010BDF814201144014431444A7A6B
:1024F000BDF80C1001EBC10303EB012104EBC10398
:10250000BDF8041001EB411103EB8101014481F896
:10251000212F401C80B20F28E2D30020BDF800100C
:10252000BDF814201144014431440A7EBDF80C105A
:1025300001EBC10303EB012104EBC103BDF804105F
:1025400001EB411103EB8101014481F8332F401C61
:1025500080B20A28E2D3BDF80000BDF81410084488
:10256000304490F82200BDF80C1001EBC10202EBE0
:10257000012104EBC102BDF8041001EB411102EB93
:10258000810181F8420F0020BDF80010BDF8142031
:1025900011440144314491F82320BDF80C1001EBA3
:1025A000C10303EB012104EBC103BDF8041001EBEF
:1025B000411103EB8101014481F8432F401C80B29B
:1025C0000528E1D3BDF814002030ADF81400BDF8A3
:1025D0000400401CADF80400BDF80C0000EB400105
:1025E00001EB001004EB001090F8170ABDF804107E
:1025F00088423FF6E1AEBDF80C00401CADF80C007F
:1026000094F86C09BDF80C1088423FF626AE1FE620
:10261000BDF80C0000EBC00202EB002004EBC0028E
:10262000BDF8040000EB401002EB800080F8DCBE37
:10263000BDF80C0000EB400101EB0010BDF80410E8
:1026400004EB001000EB011090F8421A21F0080191
:1026500080F8421ABDF80000BDF814100844304458
:10266000017ABDF80C0000EBC00202EB002004EB85
:10267000C002BDF8040000EB401002EB800080F8BF
:10268000481FE3E6BDF80C00F32100EBC00202EBAB
:10269000002004EBC002BDF8040000EB401002EB88
:1026A000800080F8DC1EBDF80C0000EB400101EB5F
:1026B0000010BDF8041004EB001000EB011090F8BE
:1026C000421A21F0080180F8421ABDF80000BDF856
:1026D000141008443044017ABDF80C0000EBC0022D
:1026E00002EB002004EBC002BDF8040000EB401038
:1026F00002EB800080F8481FBDF80000BDF8141000
:1027000008443044417ABDF80C0000EBC00202EBF3
:10271000002004EBC002BDF8040000EB401002EB07
:10272000800080F8421F0020BDF80010BDF8142082
:102730001144014431448A7ABDF80C1001EBC10305
:1027400003EB012104EBC103BDF8041001EB4111BF
:1027500003EB8101014481F8432F401C80B205281E
:10276000E2D3BDF81400C01D2FE7BDF80C0000EB4C
:10277000C00202EB002004EBC002BDF8040000EB35
:10278000401002EB800080F8DCBEBDF80C0000EBCE
:10279000400101EB0010BDF8041004EB001000EB49
:1027A000011090F8421A21F0080180F8421ABDF891
:1027B0000000BDF8141008443044017ABDF80C0044
:1027C00000EBC00202EB002004EBC002BDF80400E5
:1027D00000EB401002EB800080F8481F0020BDF89D
:1027E0000010BDF814201144014431444A7ABDF868
:1027F0000C1001EBC10303EB012104EBC103BDF895
:10280000041001EB411103EB8101014481F8432FD6
:10281000401C80B20428E2D3BDF81400401DD4E669
:10282000A81E0D2190FBF1F0C0B20490ADF80C9001
:102830004446ACE1484686E1BDF80C0000EB40019F
:1028400001EB0010BDF8041004EB001000EB0110C8
:1028500090F8420A80077DD407EB8700BDF800108E
:1028600000EBC70008443044007A0021FEF75AFA12
:10287000BDF80C2002EB420303EB0212BDF804305A
:1028800004EB021202EB031292F8402A89EA0103D8
:1028900042401A435ED1BDF80C0000EBC00101EBD1
:1028A000002004EBC001BDF8040000EB401001EB78
:1028B000800090F8150F01287DD1BDF8000030444C
:1028C000407BBDF800103144897A40EA0161BDF8CF
:1028D00000003044C07A00E0FEE3BDF800200004B0
:1028E0003244127B40EA02200143BDF80C0000EBA9
:1028F000C00202EB002004EBC002BDF8040000EBB4
:10290000401002EB8000C0F8E01EBDF8000030442B
:10291000007DBDF800103144497C40EA0160BDF8FB
:1029200000103144897CBDF8002009043244D27C77
:1029300041EA02210843BDF80C1001EB410202EB11
:102940000111BDF8042004EB011101EB0211C1F8E3
:10295000440A00E0F4E0BDF80C0000EB400101EB9C
:102960000010BDF8041004EB001000EB011090F80B
:10297000421A41F0200180F8421ABDF80C100220E2
:10298000F7F7E8F8BDF80C0000EB400101EB001090
:10299000BDF8041004EB001000EB011090F8401A91
:1029A000BDF80C0000EBC00202EB002004EBC000FD
:1029B00080F8D11E00E051E0BDF80C0000EB4001B2
:1029C00001EB001004EB001090F8160A012804D067
:1029D000022847D0032841D144E0BDF8000030442C
:1029E000407A10B1012839D13AE0BDF80C0000EB73
:1029F000400101EB001004EB001090F81C0A0028C5
:102A0000BDF80C0000EBC00101EB002000E0FDE38D
:102A100004EBC001BDF8040000EB401001EB8000A6
:102A2000D0F8E00E03D0B0F1104F03D105E0B0F5BF
:102A3000100F02D0B52101E0B0E0C321BDF80C00B9
:102A400000EBC00202EB002004EBC002BDF8040062
:102A500000EB401002EB800080F8DC1E6BE0FCE332
:102A6000B921EBE7BDF80C0000EBC00101EB002041
:102A700004EBC001BDF8040000EB401001EB800046
:102A800090F8D81EBDF80C0000EBC00202EB00204D
:102A900004EBC00090F8D40E81424CD1BDF8000088
:102AA0003044807BBDF8001000043144C97B40EA0B
:102AB0000121BDF800003044007C0143BDF80C004A
:102AC00000EBC00202EB002004EBC002BDF80400E2
:102AD00000EB401002EB8000C0F80C1FBDF80000B6
:102AE0003044417ABDF80C0000EBC00202EB00203C
:102AF00004EBC002BDF8040000EB401002EB8000C4
:102B000004E0F0E302E1EFE328E248E080F8DD1EB4
:102B1000BDF80C00A42100EBC00202EB002004EB86
:102B2000C002BDF8040000EB401002EB800080F80A
:102B3000DA1E514682E77F1C0498FFB2874213D207
:102B4000BDF80400401CADF80400BDF80C0000EB1B
:102B5000400101EB001004EB001090F8170ABDF8DB
:102B6000041088423FF668AEBDF80C0000EB40014F
:102B700001EB001004EB001090F8170ABDF80410E8
:102B800088420BD8BDF80C00401CADF80C0094F83E
:102B90006C09BDF80C1088423FF64CAE01E1ADF86F
:102BA0000C90444642E0ADF804901EE0BDF80000F1
:102BB0003044007A0021FEF7B5F8BDF80C2002EB96
:102BC000420303EB0212BDF8043004EB021202EBE5
:102BD000031292F8402A89EA010342401A432CD09A
:102BE000BDF80400401CADF80400BDF80C0000EB7B
:102BF000400101EB001004EB001090F8170ABDF83B
:102C000004108842D2D8BDF80C0000EB400101EB63
:102C1000001004EB001090F8170ABDF80410884269
:102C2000BCD8BDF80C00401CADF80C0094F86C0941
:102C3000BDF80C108842B6D8B3E0BDF80C0000EB2C
:102C4000400101EB0010BDF8041004EB001000EB94
:102C5000011090F8401ABDF80C0000EBC00202EB26
:102C6000002004EBC00080F8D11EBDF80C0000EB82
:102C7000400101EB001004EB001090F8160A012847
:102C800032D0022801D00328BDD1BDF80C0000EBE2
:102C9000C00101EB002004EBC001BDF8040000EB13
:102CA000401001EB800090F8D81EBDF80C0000EB3E
:102CB000C00202EB002004EBC00090F8D40E814269
:102CC000A1D1BDF80C00AA2100EBC00202EB00204C
:102CD00004EBC002BDF8040000EB401002EB8000E2
:102CE00080F8DA1E514600E0CA21BDF80C0000EB66
:102CF000C00202EB002004EBC002BDF8040000EBB0
:102D0000401002EB800080F8DC1E7CE7484640E083
:102D1000ADF804901EE0BDF800003044007A0021B8
:102D2000FEF700F8BDF80C2002EB420303EB0213A0
:102D300008EB0312BDF8043002EB031292F8402AAC
:102D400089EA010342401A432CD0BDF80400401C1C
:102D5000ADF80400BDF80C0000EB400101EB0011E0
:102D600008EB011090F8170ABDF804108842D2D879
:102D7000BDF80C0000EB400101EB001108EB011065
:102D800090F8170ABDF8041088420AD8BDF80C0064
:102D9000401CADF80C0098F86C09BDF80C2090426E
:102DA000B6D85FE1BDF80C00BDF8042000EB40018F
:102DB00001EB0010414608EB001000EB021090F808
:102DC000402ABDF80C0000EBC00303EB002008EB29
:102DD000C00080F8D12EBDF800003044407ABDF824
:102DE000002000043244927A40EA0222BDF800003A
:102DF0003044C07A0243BDF80C0000EBC00303EB83
:102E0000002001EBC003BDF8040000EB401003EB11
:102E10008000C0F80C2FBDF80C0000EB400202EB64
:102E2000001001EB001090F8160A012841D002288A
:102E300001D003289CD1BDF80C0000EBC00202EBCE
:102E4000002001EBC002BDF8040000EB401002EBD3
:102E5000800090F8D82EBDF80C0000EBC00303EB07
:102E6000002001EBC00090F8D40E824280D1BDF862
:102E70000C00A52200EBC00303EB002001EBC00314
:102E8000BDF8040000EB401003EB800080F8DA2E60
:102E9000BDF80C0000EBC00303EB002008EBC00101
:102EA000BDF8040000EB401001EB800080F8DCAEC0
:102EB0005EE7BDF80C0000EBC00202EB002001EB66
:102EC000C002BDF8040000EB401002EB800090F857
:102ED000D82EBDF80C0000EBC00303EB002001EB83
:102EE000C00090F8D40E8242E2D1BDF80C00B222AC
:102EF00000EBC00303EB002001EBC003BDF80400AE
:102F000000EB401003EB800080F8DA2EBDF80C00D7
:102F1000E52200EBC00303EB002001EBC003BDF88A
:102F2000040000EB401003EB800080F8DC2E002C46
:102F3000BED1BDF804000128BAD1BDF80C0000EBE9
:102F4000C00202EB002008EBC001BDF8040000EB5A
:102F5000401001EB8000D0F80C0F09E7BDF800002D
:102F60003044007A05287DD2BDF800003044007A54
:102F7000401EADF80C00BDF800003044407ABDF8AA
:102F8000001000043144897A40EA0120BDF80010A5
:102F90003144C97A0843C117FDF7C4FEBDF80C10CF
:102FA000444601EB410202EB011208EB0211C1F8A9
:102FB000100ABDF800003044007B0021FDF7B2FE8E
:102FC000BDF80C1001EB410202EB011204EB0211FF
:102FD00081F8140ABDF800003044407B0021FDF761
:102FE000A1FEBDF80C1001EB410202EB011204EB53
:102FF000021181F8150ABDF800003044807B0021E1
:10300000FDF790FEBDF80C1001EB410202EB01123E
:1030100004EB021181F8160ABDF800003044C07BB1
:103020000021FDF77FFEBDF80C1001EB410202EB21
:10303000011204EB021181F8170ABDF800003044B8
:10304000007C0021FDF76EFEBDF80C1001EB410283
:1030500002EB011204EB0211C1F8180ABDF80000DE
:10306000304400E035E2407C0021FDF75BFEBDF816
:103070000C1001EB410202EB011204EB021181F88A
:103080001C0ABDF80C0000EB400101EB001104EB41
:10309000011090F8160A0628484655D09CE0BDF865
:1030A0000000BDF8041008443044807C0021FDF786
:1030B00039FEBDF804204FF00309B2FBF9F2BDF868
:1030C0000C1001EB410303EB011304EB031101EBC3
:1030D000021181F8400A00E086E3BDF80000BDF867
:1030E000041008443044C07C0021FDF71BFEBDF8ED
:1030F0000420BDF80C10B2FBF9F201EB410303EB25
:10310000011304EB031101EB021181F8410ABDF830
:103110000000BDF8041008443044007D0021FDF794
:1031200001FEBDF80420BDF80C10B2FBF9F201EB72
:10313000410303EB011304EB031101EB021181F8CE
:10314000480ABDF80400C01CADF80400BDF80C002E
:1031500000EB400101EB001104EB011090F8170A9D
:10316000BDF8041000EB4000884298D845E0BDF857
:103170000000BDF8041008443044807C0021FDF7B5
:10318000D1FDBDF80C1001EB410202EB0111BDF8BD
:10319000042004EB0111520801EB021181F8400AEE
:1031A000BDF80000BDF8041008443044C07C002184
:1031B000FDF7B8FDBDF80C1001EB410202EB011167
:1031C000BDF8042004EB0111520801EB021181F853
:1031D000410ABDF80400801CADF80400BDF80C00E5
:1031E00000EB400101EB001004EB001090F8170A0F
:1031F000BDF80410B1EB400FB9D3BDF80C1002209C
:10320000F6F7A8FCBDF80C00C0B200E0D8E2FEF76B
:103210005DFABDF80C00012100EB400204EB8200D6
:1032200080F83115B7E2BDF800003044007A44461A
:1032300088F86D02BDF800003044407A88F86C02CE
:10324000BDF800003044807A88F86B02BDF80000B9
:103250003044C07A88F86A0200E0A2E2BDF80000BB
:103260003044007B84F86902BDF800003044407BA4
:1032700084F8680204F51A74F6F788FBF6F744FB45
:103280002078A4F51A74FF2829D1F6F7F5FABDF8CD
:1032900000003044007A84F86D02BDF8000030442C
:1032A000407A84F86C02BDF800003044807A84F8DB
:1032B0006B02BDF800003044C07A84F86A02BDF8A1
:1032C00000003044007B84F86902BDF800003044FF
:1032D000407B84F86802F6F759FBF6F715FB606D42
:1032E00018B10F2002E0F5E0FEE0102084F825067A
:1032F00051E21020444688F82506BDF8000030440D
:10330000007A88F86D02BDF800003044407A88F8F1
:103310006C02BDF800003044807A88F86B02BDF87A
:1033200000003044C07A84F86A02BDF800003044DE
:10333000007B84F86902BDF800003044407B84F8CB
:10334000680204F51A74F6F721FB01F0B9FEA060DB
:10335000A068A0681FE20E2188F8251688F8619001
:1033600019E24946ADF80C90444638E0ADF8041037
:1033700014E0BDF80C0000EB400202EB0010BDF8B9
:10338000042004EB001000EB021090F8420AC00782
:1033900012D1BDF80400401CADF80400BDF80C00CB
:1033A00000EB400202EB001004EB001090F8170A4B
:1033B000BDF804209042DCD8BDF80C0000EB4002C0
:1033C00002EB001004EB001090F8170ABDF804207F
:1033D000904208D8BDF80C00401CADF80C00BDF8B8
:1033E0000C000428C2D3BDF80C00042869D3FF4A9E
:1033F00089465170FE490120C1F88802C1F888024F
:1034000094F86500E8B30D2084F82506BDF80000A7
:103410003044407ABDF800103144097A40EA012076
:10342000ADF80800BDF800003044C07ABDF80010C7
:103430003144897A40EA0120508000204FF4007323
:10344000BDF8001001443144097B04EB000C8CF8FA
:103450006610401C80B29842F2D3E448408800F2E3
:10346000FF3081B20120F5F761FD50B184F8619021
:10347000DE48418864225143BDF80820B1FBF2F1D7
:1034800000E01CE084F860100121A1714188491C12
:1034900041804088BDF80810884210D914F85C0FAC
:1034A00040F001002070207820F00600801C207081
:1034B000BDF80800608000210120F6F74BFB48466C
:1034C00043E1102084F8250614F85C0F40F08000DA
:1034D000207060E1BDF800003044017A88F8611086
:1034E000112188F8251656E14946ADF80C9044465E
:1034F00038E0ADF8041014E0BDF80C0000EB400219
:1035000002EB0010BDF8042004EB001000EB0210E9
:1035100090F8420AC00712D1BDF80400401CADF873
:103520000400BDF80C0000EB400202EB001004EBBD
:10353000001090F8170ABDF804209042DCD8BDF8BE
:103540000C0000EB400202EB001004EB001090F8BE
:10355000170ABDF80420904208D8BDF80C00401CA2
:10356000ADF80C00BDF80C000428C2D3BDF80C0067
:1035700004287DD39D4B002058709D490120C1F83F
:103580008802C1F8880294F86500E8B3122084F834
:103590002506BDF800003044007A84F8610094F8F4
:1035A0006100401EADF80C000020BDF80010014481
:1035B00031444A7ABDF80C1001EB410C0CEB0111BF
:1035C00004EB0111014481F81E2A401C80B20A2834
:1035D000EBD3BDF800003044007DBDF8001031444D
:1035E000C97C40EA0120ADF80800BDF80000304475
:1035F000807DBDF800103144497D40EA01205880AB
:1036000000204FF4007100E056E0BDF800200244B5
:103610003244D27D04EB000C8CF86620401C80B252
:103620008842F0D358889946BDF80C1000EB8120F1
:10363000401E81B20320F5F779FCE8B3B9F8021017
:10364000484664225143BDF80820B1FBF2F184F8EA
:1036500060100121A171B9F80210491CA9F80210EB
:10366000B9F80210BDF80820914242D9002000E0CC
:1036700091E0BDF80C1001EB410202EB011104EBEB
:10368000011101EB001191F8492A42F0010281F881
:10369000492A401C80B21028E9D3BDF80C0000EB89
:1036A000400101EB001004EB001090F8281A41F0E3
:1036B000010180F8281A00E046E0BDF80C0000EB9C
:1036C000400101EB001004EB001090F8281A21F0E3
:1036D0000601891C80F8281ABDF80810BDF80C00F6
:1036E00000EB400202EB001004EB0010A0F82A1AD5
:1036F00025E04088012827D10020BDF80C1001EBFF
:10370000410202EB011104EB011101EB001191F8F0
:10371000492A22F0010281F8492A401C80B210286F
:10372000EBD3BDF80C0000EB400101EB001004EB03
:10373000001090F8281A21F0010180F8281ABDF82D
:103740000C100220F6F706FA00202949C1F8880279
:10375000C1F888021FE0D8F8540044460A21B0FBA3
:10376000F1F0BDF800103144097A884213D1BDF858
:1037700000003044007A18B1606D0A38606504E0DA
:10378000C4F85490102084F8250600210520F6F78F
:10379000E1F90120A071B8F8EA04424620B3002004
:1037A0001EE000200146BDF800200244B154401C38
:1037B00080B20528F7D3A8F8EA1407B0BDE8F08F67
:1037C0000020A1F8EA04F8E7BDF8001029440144FC
:1037D00031448978BDF800300344F154401C80B274
:1037E000B2F8EA148142EFD8414603E01408002001
:1037F00000004242B8F8EA0400287EF46FACDCE72F
:103800002DE9F74F002084B0FE4E0190054680461A
:10381000009096F826054FF0000B012876D196F817
:103820002106012872D108EB480101EB081000279E
:1038300006EB001A56E00AEB071494F8420A000659
:103840004ED594F8420A40F0040084F8420A94F8F5
:10385000420A000744D594F8420A20F0080084F890
:10386000420AC6F835B008EBC80101EB082006EBA8
:10387000C00007EB471100EB8109E24809F6F96146
:103880001022253004F52464F4F7DDFCD9F8F10E9C
:10389000C6F81900D9F8F50EC6F81D002078307664
:1038A000D9F80C0FC6F82100D648D0F86812C6F82F
:1038B0003910B0F86C02A6F83D006068C6F83F0009
:1038C000706D81B20220F5F731FB00210620F6F77A
:1038D00041F9706D401C706500210520F6F73AF93A
:1038E0007F1CBFB29AF8170AB842A4D841460220FA
:1038F000F6F730F908F101001FFA80F8B8F1040F6B
:1039000091D386F821B60B2086F82506BE4F0020FD
:10391000387000980DE001F0D3FBC6F87002D6F8BD
:103920007002C0F300400190D6F87002C0F342006C
:1039300000900028EFD096F82306B3493A310228C8
:1039400016D1B24890F832202AB1002180F8321006
:1039500001F08CF969E0072555200870FD204870BA
:10396000AA2088700020C870087161224A7188718D
:10397000F520485500208B46D6F87012C0F103029E
:10398000D200D1402B1803EB0B02D170401C80B247
:103990000428F1D396F8220630B39D48D0F80812D7
:1039A0003078B8B3002001433CD00020594632188B
:1039B00092F8A8252B180B44DA71401C80B2142809
:1039C000F5D30020321892F834262B180B44DA76FF
:1039D000401C80B20A28F5D30BEB0501069881F84C
:1039E000250005F1260405E00BEB05010698C871DA
:1039F00005F10804CCB18349069881F8E7040698DC
:103A00001021FF2311287DD013DCA0F10B00062824
:103A100022D200E004E0DFE800F01F1FFF11F420D5
:103A20000120C0E7012086F82605002007B0BDE888
:103A3000F08FA22810DA12280ED10FE2714880F818
:103A40002516744900205A4626180B5C9355401CD5
:103A500080B20A28F8D30A34F8E26A4890F85C1079
:103A6000C90704D0012080F31388FEF70FF84FF048
:103A7000000977E100EB400101EB091002EB0016B1
:103A800096F8160A032814D096F8160A012810D0C2
:103A900096F8160A02280CD096F8160A042808D0C0
:103AA00096F8160A05287DD096F8160A06287AD0C8
:103AB00054E101200BF80400E41CA0B202230290A0
:103AC0000BF80030401C80B21D230BF80030401C66
:103AD00084B20020A7E006EB081292F8400A59468B
:103AE0000BF80400641CA0B292F8424A0BF80040A4
:103AF000401C84B292F8420A400709D492F8420A64
:103B0000000700E059E103D492F8420A800777D514
:103B100000201F46D2F8443AC0F1030C4FEACC0C07
:103B200023FA0CF300EB040C01F80C30401C80B2BB
:103B30000428EFD3241DA3B209EBC90404EB092226
:103B400007EBC20408EB4812002004EB8207D7F809
:103B5000F12EC0F10304E400E240C4180A55401CF1
:103B600080B20428F3D31B1D9AB20020D7F8F53E8B
:103B7000C0F10304E400E34084180B55401C80B2FC
:103B80000428F3D3121D92B20020D7F80C3FC0F1E5
:103B90000204E400E34084180B55401C80B2032863
:103BA000F3D301E050E080E0D21C1FFA82FA002437
:103BB000D7F8F90ED7F8FD1EC4F10502D200F4F7CC
:103BC00032FB04EB0A020BF80200641CA4B2062CC0
:103BD000EED30AF106001FFA80FA0024D7F8010F8D
:103BE000D7F8051FC4F10502D200F4F71CFB04EB63
:103BF0000A020BF80200641CA4B2062CEED30CE0FF
:103C00000EE062E1D410002014080020D44000200F
:103C100000004042BC8E0108ACE00AF1060084B20C
:103C200008F1010080B2FF4B96F8171A8046414513
:103C30003FF651AF0298029A201A0BEB0201030AD9
:103C400001F8023D487089E002205E460BF804004E
:103C5000E41CA4B22346002090461AE0421C3255D0
:103C6000641CA1B23C1894F805447454491C8CB2ED
:103C7000002108EB0010471897F8117401EB040CB1
:103C800006F80C70491C89B21029F4D31034A4B280
:103C900090B298F8041447468142DFD80BEB03003A
:103CA000002100F8021DE11A57E003200BF8040080
:103CB000E41CA7B202200BF80700781C80B20E218A
:103CC0000BF80010401C84B200219646DA463AE018
:103CD00006EB011292F8400A0AF80400641CA0B234
:103CE00092F8424A0AF80040401C84B292F8420A14
:103CF000000726D509EBC90C0CEB09220EEBC2021A
:103D000001EB4113002002EB8302131893F8173FD5
:103D100000EB0408D4460AF80830401C80B20A2898
:103D2000F3D30A34A3B20020141894F8304F00EBF8
:103D300003080CF80840401C80B20228F4D39B1CF6
:103D40009CB2491C89B296F8170A8842C0D80AEB7F
:103D50000700002100F8021DE11B417009F101007C
:103D60001FFA80F9AF4A92F86C19484649453FF668
:103D700081AE6BE17878401C78707878052804D2A1
:103D8000A84890F85C20D20707D0A64880F82516EE
:103D900090F85C10C90704D005E00D2180F82516C5
:103DA00001E080F860307888010A0BF80410798807
:103DB0000BEB04004170A41C48E19A4F87F82516CC
:103DC00097F86100DC460BF804000022641C38E020
:103DD00097F8610002EB421600EBC00101EB0020F6
:103DE00007EBC00000EB860090F80207012826D1FF
:103DF00097F8610000EB400101EB001007EB0010A9
:103E000000EB021090F810090CF80400641CA3B237
:103E1000002097F8611001EBC10404EB012107EBCE
:103E2000C10101EB8601014491F803171C180CF83D
:103E30000410401C80B20A28EBD30A339CB2521CF7
:103E400092B297F8610000EB400101EB001007EB24
:103E5000001090F8E7089042BAD8F7E07878401C54
:103E60007870787805280CD26E4A92F8610000EBE1
:103E7000400606EB001002EB001090F8F808C007AF
:103E80000FD0684A82F8251692F8610000EB4001D5
:103E900001EB001002EB001090F8F808C00704D006
:103EA00005E0122082F8250601E082F860305D48C6
:103EB00090F861100BF8041079880BEB0400090AE4
:103EC000417079888170E41CC0E0564801218171FD
:103ED000416D0A22B1FBF2F259460BF80420426D03
:103EE000641C0A2A01D90A2300E0436D00220292D1
:103EF00099460B552222641C0A5500268046DA4654
:103F0000641C9CE0D8F8540038B1D8F85400801BE9
:103F1000401E81B20220F4F79DFF98F81800514628
:103F20000AF80400641CA2B20020D8F81930C0F1CD
:103F30000304E400E34084180B55401C80B20428BD
:103F4000F3D3121D92B20020D8F81D30C0F1030443
:103F5000E400E34084180B55401C80B20428F3D3DE
:103F6000121D92B20020D8F82130C0F10204E40002
:103F7000E34084180B55401C80B20328F3D3D21CB5
:103F800097B20024414651F8250F4968C4F1050253
:103F9000D200F4F748F9E2190AF80200641CA4B24E
:103FA000062CEFD3BF1DBFB20024414651F82D0FA0
:103FB0004968C4F10502D200F4F735F9E2190AF8AC
:103FC0000200641CA4B2062CEFD3BF1D98F83E304B
:103FD000B8B2414652460AF80030401C98F83D30CD
:103FE00080B20AF80030401C98F83C3080B20AF8E1
:103FF0000030401C98F83B3080B20AF80030401C7A
:1040000091F83A3080B21354401C91F8393080B2A4
:104010001354401C83B20020D1F83F40C0F1030785
:10402000FF0001E0D4100020FC40C718D455401C0C
:1040300080B20428F0D31B1D761C9CB2B6B2029A43
:104040000021B6EB09009141FFF45CAF661B0BEB5E
:104050000500310A5F46804641708670DFF878A01F
:104060009AF8670228B1B1B2404600230422F6F75D
:1040700033FC0023B9460AE0E91801EB0907F87997
:10408000DDE90021F5F7E2FCF8715B1C9BB29E4272
:10409000F2DCB1B24D464046F5F7BCFA010A2955AB
:1040A000641CA1B26854491C9AF823068CB20228F9
:1040B0000AD1601F010AE970287181B2681D01F000
:1040C00046F92855641CA4B2044804600121001F6D
:1040D000F5F7F6FA2046A9E4D4100020BC640240AB
:1040E00070B5164C40F224452946204603F019F8D5
:1040F000002821D02946204602F0B0FF104D0021B3
:104100002846F5F7DDFA61102846F5F7C3FA0D49A0
:10411000012081F824062088A088281D0268C2F5A5
:10412000FA62A1F8EA244FF4FA6101602846BDE87A
:1041300070400121F5F7C4BA70BD000000100140C5
:1041400088640240D410002010B5074C0549204671
:10415000F5F7A0FA00212046F5F7B2FA034901204D
:10416000087010BD00800028B864024014080020C8
:104170002DE9F04301218FB0880500F0F7FEDFF84C
:1041800094904846F5F7A6FA4020050103900024D4
:10419000CDE90545C60207940894CDE909464FF0DC
:1041A00000681E480B940C940D941B4FCDF80080B2
:1041B0000E94CDE9017069464846F5F733FB0122BC
:1041C00010214846F5F718FBDFF84890A9F13009AF
:1041D0004846F5F77FFA4FF4FA60CDE90340CDE9A0
:1041E000054507940894CDE909460D480B940C94B5
:1041F0000D94CDF800800E94CDE9017069464846D3
:10420000F5F710FB01214846F5F75AFA0FB0BDE863
:10421000F0830000B8640240041001404E08002002
:10422000205E00207CB50121032000F09FFE134D8D
:10423000072206212846F6F781F80722114628466C
:10424000F6F77CF8C020022100908DF805100024BC
:104250008DF8064001208DF807008DF8041069469E
:104260002846F6F72FF8072000908DF804408DF8C7
:10427000074069460248F6F725F87CBD0004024075
:104280000000024070B50024FFF7CCFFFFF770FF7D
:104290004FF4E13000F086F800F066F8012140208C
:1042A00000F07CFE012000F0FDFE2D490B2081F87E
:1042B0002506002581F8145581F8165581F8155505
:1042C00081F817554FF47A70C1F81C0581F8245510
:1042D000012381F8263581F8253581F82735C2007C
:1042E000C1F82C2581F8FC5481F8FE3481F8FD34A6
:1042F00081F8FF34C1F8040581F8085581F80A35C2
:1043000081F8093581F80B354210C1F81025154A9E
:10431000157095705370D37042F21076966042F625
:10432000F82604EB440201EB820282F8305582F851
:10433000325582F8313582F83355C2F83865641C3D
:10434000042CEED391F8202622B191F82026521E9B
:1043500081F8222604F09CFBBDE8704000F022B9F1
:10436000D41000200441002038B546208DF800000C
:1043700002208DF8010001248DF802408DF80340E1
:104380006846FDF747FB25208DF800008DF80140B9
:1043900000208DF802008DF803406846FDF73AFBD7
:1043A00038BD00001FB504460121102000F01AFEA0
:1043B0000020ADF804000094ADF80600ADF8080048
:1043C000ADF80C000C200D4CADF80A0069462046F3
:1043D00002F0DEFE0121204602F043FE012240F2FF
:1043E0002441204602F0BCFE1021204602F036FE99
:1043F0000122C021204602F03EFE1FBD00100140F8
:104400002DE9F04F8DB034225F496846F3F71BFF6A
:104410005E4D002695F8220600287CD0DFF870B1AA
:104420000121CBF888124FF0000985F82496594FE6
:10443000594C02E0B85DA055761C5648F3F721FFB1
:10444000B042F7D8DFF85481C8F800600121A8F124
:104450000400F5F735F94FF4FA7004F019FB85F80C
:104460002496DFF830A100260AF1750A03E01AF855
:104470000600A055761C47487530F3F702FFB0429E
:10448000F5D8C8F8006045480121001FF5F718F974
:104490004FF47A7004F0FCFA4E46A94685F824667B
:1044A000DFF8F0A000250AF1020A03E01AF805007F
:1044B00060556D1C3748801CF3F7E3FEA842F5D821
:1044C000C246C8F8005035480121001FF5F7F8F83A
:1044D0004FF47A7004F0DCFAB04689F824660026BE
:1044E00002E0B85DA055761C2A48F3F7CAFEB04238
:1044F000F7D85546CAF80060DFF8A0A00121AAF15C
:10450000040A5046F5F7DCF84FF47A7004F0C0FA6C
:104510002349684600E034E0F3F7A7FE1D496846EA
:10452000891DF3F7A2FE4F4689F824860026E94646
:1045300003E019F80600A055761C6846F3F7A1FEC3
:10454000B042F6D82E6001215046F5F7B9F84FF485
:104550007A7004F09DFA464687F824860D490020BB
:104560000A310A5C2254401C0728FAD3401E2860F6
:1045700001215046F5F7A4F8642004F089FACBF83D
:1045800088620DB0BDE8F08F34940108D41000208B
:1045900000004242589101084E080020BC640240CD
:1045A000901600202DE9F04FDFF8F48389B0002445
:1045B00098F8220600287DD0FA480125C0F88852D4
:1045C00098F8231608F27650F74E0090022904D08E
:1045D000A34688F824B6F54FEDE000203055641C62
:1045E000642CFBD3814688F82406F04900209631DC
:1045F0000A5C3254401C0828FAD3002708F2E4541D
:1046000006E008EB070090F8E405F11908727F1C3A
:104610002046F3F736FEB842F3D82C20F119087281
:10462000002408F20C6B093706E008EB040090F850
:104630000C0639197054641C5846F3F722FEA04248
:10464000F3D8DBA1D848F3F710FED748F3F719FEEB
:10465000DFF860B3CBF800000121ABF10400F5F7FF
:104660002FF84FF47A7A474605E0012004F010FA5B
:10467000641C54457ED897F824060028F5D0CE480F
:10468000D0F81802C949B331C8B100204A463254A3
:10469000401C6428FBD3B84687F824260024085D14
:1046A0003055641C0E2CFAD30098F3F7EAFD000491
:1046B000000C00E073E032D00024414629E0B84607
:1046C00087F82496002404E0B848B330005D3055E4
:1046D000641CB648B330F3F7D4FDA042F4D8CBF84D
:1046E0000040B4480121001FF4F7EAFF464605E008
:1046F000012004F0CDF9641C5445BBD896F824067B
:104700000028F5D015E00A1992F8762533199A7326
:10471000641C8442F7D3A6A1A348F3F7A6FDA248E0
:10472000F3F7AFFDCBF80000A2480121001FF4F71A
:10473000C7FF564697F8240690B3A048A0494C46B8
:10474000006808609D48001D006848609B4808306C
:104750000068886000203A1882F8A845401C142898
:10476000F9D3087A04AECD7A8B7A4A7A86E82D009E
:10477000CD7900E012E108798B794A798DE82D0036
:104780008B780A788FA19A4802F06AFD00210320F5
:10479000F5F7E0F9002802D08248C0F888424BE2E1
:1047A000FFE7012004F074F9641CB442C2D93BE273
:1047B000385D3055641C7D48F3F763FDA042F7D89F
:1047C0007C4804600121001FF4F77AFF4FF4FA706F
:1047D00004F05EF95846DA46C34688F82406DFF846
:1047E000CC81002408F1750803E018F80400305566
:1047F000641C6E487530F3F744FDA042F5D86D484F
:1048000004600121001FF4F75BFF4FF47A7004F09D
:104810003FF9D046D9468BF824A6DFF890A10024B2
:104820000AF1020A03E01AF804003055641C5F48DC
:10483000801CF3F726FDA042F5D8DFF878A1CAF86E
:1048400000400121AAF10400F4F73AFF4FF47A7016
:1048500004F01EF989F82486002402E0385D305502
:10486000641C5248F3F70DFDA042F7D85746CAF82A
:10487000004050480121001FF4F722FF4FF47A70E6
:1048800004F006F9C24689F82486DFF82081002466
:1048900008F16A0803E018F804003055641C434826
:1048A0006A30F3F7EEFCA042F5D8BB463C604148C5
:1048B0000121001FF4F704FF4FF4FA784F4605E09A
:1048C000012004F0E5F8641C444567D897F82406F5
:1048D0000028F5D0D14687F824A6DFF8D0A0002420
:1048E0000AF1390A03E01AF804003055641C2F4815
:1048F0003930F3F7C6FCA042F5D8DA46CBF80040D1
:104900002C480121001FF4F7DBFE05E0012004F034
:10491000BFF8641C4445D8D897F824060028F5D081
:1049200087F824962448D0F818022049113168B13C
:1049300000200A5C3254401C0D28FAD30098F3F78B
:10494000A0FC0104090C1BD0002013E000248B46BE
:1049500003E01BF804003055641C14481130F3F7D1
:1049600090FCA042F5D80FE03A1892F8762533185B
:104970005A73401C8842F7D30DA10B48F3F775FC1E
:104980000948F3F77EFC0446CAF8004009480121B3
:10499000001FF4F795FE4FF47A7B31E0BDE0000094
:1049A000D4100020000042424E0800205891010817
:1049B0000D0A0000BC64024000004342107AFF1F51
:1049C000F065002025303278253032782530327875
:1049D00025303278253032782530327825303278DB
:1049E00025303278253032782530327825000000A5
:1049F0007C1600200A2004F04BF8641C5C458AD821
:104A000097F824060028F5D087F824960024DFF8CC
:104A100038B203E01BF804003055641C8A48F3F7F1
:104A200030FCA042F6D8CAF8004001218748F4F7CC
:104A300047FE05E0012004F02BF8641C4445DED855
:104A400097F824060028F5D087F82496DFF8F8B107
:104A500000240BF1110B03E01BF804003055641C1B
:104A600079481130F3F70DFCA042F5D8D346CAF8C7
:104A7000004001217548F4F723FEC24605E00120FD
:104A800004F006F8641C544547D897F8240600281B
:104A9000F5D0C84687F824966B4800243730015D6E
:104AA0003155641C0C2CFAD3601ECBF80000012198
:104AB0006648F4F705FE05E0012003F0E9FF641CF9
:104AC00054452AD897F824060028F5D060A16248FA
:104AD00004F06CF9D8B1604A0021431813449146A0
:104AE0005B797C1884F86135491C1429F5D397F853
:104AF000BD0568B359495A48F3F7B7FB52495848BE
:104B00004239F3F7B2FB87F8248600240AE001203B
:104B100003F0BEFF641C5445D8D985E05048005DC1
:104B20003055641C4E48F3F7ACFBA042F6D8CBF8E6
:104B3000004001214548F4F7C3FD05E0012003F0E2
:104B4000A7FF641C54456FD897F824060028F5D0B9
:104B5000642003F09DFF002087F8240604463A48AD
:104B60004330B046025D3255641C0B2CF9D3601EF5
:104B7000CBF8000001213548F4F7A2FD05E0012043
:104B800003F086FF641C54454ED897F8240600288D
:104B9000F5D034A1304804F009F9061E37D064205E
:104BA00003F076FF00200446391881F8A845401C20
:104BB0001428F9D30020494632180A4452783B1889
:104BC00083F8AD25401C0F28F6D300210320F4F70D
:104BD000C1FF10B12448C0F88842642003F058FF98
:104BE00087F824461849002440463E390A5D02559C
:104BF000641C072CFAD3611ECBF800100121134866
:104C0000F4F75EFD642003F043FF564610E00120F8
:104C100003F03EFF641C5445BBD905E0012003F0BE
:104C200037FF641CB44203D985F31388FCF72EFFC9
:104C300097F824060028F1D00B490020C1F888021B
:104C400009B0BDE8F08F0000A0910108B8640240EF
:104C500049434349443A0000205E0020901600205A
:104C60001C080020493A0000000042422DE9F047AC
:104C70000020574E01463154401C6428FBD3554D4B
:104C8000884685F82416544900200A5C3254401C9A
:104C90000828FAD3002705F2E45405E0E81990F853
:104CA000E405F11908727F1C2046F3F7EAFAB842CE
:104CB000F4D82C20F1190872002405F20C69093788
:104CC00005E0281990F80C0639197054641C484600
:104CD000F3F7D7FAA042F4D840A13D48F3F7C5FA5C
:104CE0003B48F3F7CEFA3E4F3860A7F1040A0121A2
:104CF0005046F4F7E5FC05E0012003F0C9FE641C12
:104D0000642C03D895F824060028F5D03548D0F84F
:104D1000180231491D31B8B1002042463254401CBE
:104D20006428FBD3A84685F824260024085D305566
:104D3000641C0E2CFAD32C48F3F7A3FA0004000CE1
:104D400031D00024414628E04046A84685F8240694
:104D50000024894603E019F804003055641C1E48FD
:104D60001D30F3F78EFAA042F5D83C600121504681
:104D7000F4F7A6FC464605E0012003F089FE641C1A
:104D8000642C1FD896F824060028F5D01AE00A19DA
:104D900092F8762533199A73641C8442F7D30FA1D5
:104DA0000B48F3F762FA0A48F3F76BFA386001210F
:104DB0005046F4F785FC05E0012003F069FE641C11
:104DC000642C03D895F824060028F5D0BDE8F087B8
:104DD0004E080020D4100020EE9101080D0A0000BA
:104DE000BC640240000043424A1600202DE9FC5FEB
:104DF0000121592000F0BAF800248DF80440022067
:104E0000DFF894B04FF47C578DF80700009769469F
:104E10005846F5F757FAFC20DFF8809000908DF89F
:104E2000044001258DF8075069464846F5F74AFACF
:104E3000DFF86CA04FF440468DF8044000968DF8E2
:104E4000075069465046F5F73DFA0720DFF85480D1
:104E500000908DF804408DF8075069464046F5F7FC
:104E600031FA07214046F5F782FA31465046F5F708
:104E70007EFA39465846F5F77AFAFC214846F5F7A6
:104E800076FA0948D0F828120848012902D004709F
:104E9000BDE8FC9F0570FBE70010024000180240CF
:104EA000000C02400000024000004242D4100020EA
:104EB00010B5FFF79BFF642003F0EAFD1048D0F81F
:104EC0003C12104819B1002180F8221610BD0E497D
:104ED000D1F8182292B1012280F82226D1F80822B6
:104EE000D1F80C1242EA4101C94380F8231690F828
:104EF000231601F0030180F8231610BD0222EBE710
:104F000000804142D4100020000043427CB50121C2
:104F1000102000F02BF84CF20400012400908DF8D2
:104F2000044000208DF8060003208DF80500084D90
:104F30008DF8074069462846F5F7C4F9042128464C
:104F4000F5F713FA0348C0F8B842C0F8BC427CBD7C
:104F50000010024000004242FFF7D8BF4FF400614A
:104F60000148F5F7FBB9000000040240044A00299B
:104F7000116801D0014300E08143116070470000D7
:104F800030380240044A0029116801D0014300E092
:104F9000814311607047000010380240044A002924
:104FA000116801D0014300E08143116070470000A7
:104FB00034380240044A0029116801D0014300E05E
:104FC000814311607047000040380240044A0029C4
:104FD000116801D0014300E0814311607047000077
:104FE00020380240044A0029116801D0014300E042
:104FF000814311607047000044380240044A002990
:10500000116801D0014300E0814311607047000046
:105010002438024070B5204B1968204C11F00C0167
:1050200004D06610042903D0082903D004601BE0D3
:10503000066019E0184A121F1168C1F38055116803
:1050400001F03F0115B1B6FBF1F101E0B4FBF1F164
:1050500014681268C4F388146143C2F30142521CFD
:105060005200B1FBF2F1016019680F2202EA11113E
:105070000B4A545C0168E14041601C68072505EA61
:105080009424145D21FA04F484601B6805EA533308
:10509000D25CD140C16070BD083802400024F400E9
:1050A0000000002005490028086802D040F00400F4
:1050B00001E020F00400086070470000000806507E
:1050C00001480068704700000808065070B50120CC
:1050D00080F310880C4D10212846F5F746F9082179
:1050E0002846F5F744F9D720F3F7D8FFFF20F3F768
:1050F000D5FF044610212846F5F739F9002181F340
:105100001088204670BD00000000024070B50120EC
:1051100080F31088194C0020A080FFF7D7FF00060D
:1051200009D4012003F0B4FCA088401C80B2A08008
:10513000C828F2D31EE0A088C8281BD2104D102129
:105140002846F5F712F908212846F5F710F99F20AF
:10515000F3F7A4FFFF20F3F7A1FFFF20F3F79EFF73
:10516000607010212846F5F702F9002080F31088BE
:10517000607870BD002080F3108870BD1E10002084
:105180000000024070B5012188B08803FFF712FFCC
:1051900001210220FFF7EAFE00244FF400602F4EA9
:1051A0008DF8044000908DF8074069463046F5F7C9
:1051B00089F801218DF8041002258DF805500803A7
:1051C0008DF806408DF80710009069463046F5F7D7
:1051D00079F805220D213046F5F7B0F805220E21A9
:1051E0003046F5F7ABF805220F213046F5F7A6F863
:1051F0004FF4604000908DF8045003208DF80500B6
:105200008DF806408DF8074069463046F5F75AF8A4
:10521000134D284600F04AF8ADF810406815ADF877
:1052200012001820ADF814000720ADF81800ADF8F2
:1052300008404FF48270ADF80C40ADF80A00ADF8AC
:105240000E40ADF8164002A9284600F064F801218E
:10525000284600F021F808B070BD000000040240AC
:105260000038004070B50B4C05460221204600F086
:1052700047F80028F9D02946204600F04AF80121D5
:10528000204600F03DF80028F9D0204600F03FF815
:10529000C0B270BD003800400029018802D041F042
:1052A000400101E021F0400101807047114910B533
:1052B00088420AD1841401212046FFF79FFE204630
:1052C000BDE810400021FFF799BE0B49884202D18A
:1052D0000121041404E0094988420AD10121C413C0
:1052E0002046FFF773FE2046BDE810400021FFF77F
:1052F0006DBE10BD0030014000380040003C004051
:105300000246002012890A4200D00120704780899D
:1053100070478181704730B502884C8802F4415350
:105320000A88CD8822438C882C4322430C8922434F
:105330004C8922438C892243CC8922431A43028020
:10534000828B22F400628283098A018230BD024688
:10535000002003E012F8013B1844C0B2491E89B294
:10536000F8D2704770B501218D070024284601F05E
:1053700051FBE8B3F5F7A0FA0020264B3BE003EB26
:105380008401D1F840261278012AD1F8402603D0B2
:105390005278012A08D02AE01070D1F840265070C7
:1053A000D1F84026907030E0D1F840269278F2B9DA
:1053B000D1F840265668761C5660D1F840265268CF
:1053C000D1F84066B668B24211D3D1F840660122E6
:1053D000B270D1F84026D278012A16D0D1F84026F2
:1053E0005070D1F840265060D1F84016C87000E0E7
:1053F00005E0641CE4B293F83E16A142BFD82846EB
:10540000BDE87040012101F04FBAD1F84016486064
:10541000EDE70000D41000200CB5002225490092D1
:105420000192086840F4803008604FF4A063086877
:1054300000F4003001900098401C0090019810B9D1
:1054400000989842F3D10868800330D5012001907C
:1054500018484030026842F08052026016480268E4
:1054600042F4804202601348083002680260026819
:10547000026002680260031F104A1A600A6842F064
:1054800080720A600A689201FCD50D4A40F20561FB
:105490001160016821F003010160016841F002011F
:1054A00001600168C1F381010229FAD10CBD0192AA
:1054B0000CBD000000380240007000400854400756
:1054C000003C02407CB500229FED170A00928DED52
:1054D000010A6D4601AC16E0835CA3F13006102E84
:1054E00005D2009B1B010093865C303E07E0413BE8
:1054F000062B0CD2009B1B010093865C373E1E439B
:10550000521CD2B200968A42E6D3002006E0BFEEDB
:10551000000A7CBD2A5C2254401CC0B2B0EB510F83
:10552000F8D39DED010A7CBD0000000030B50546B2
:105530000022104611E0AB5CA3F13004102C02D223
:1055400044EA001007E0A3F14104062C08D204014C
:10555000A3F137002043521CD2B28A42EBD330BDB4
:105560004FF0FF3030BD00002DE9FC414E4D4FF0B3
:10557000380895F86A02002105F51A75FBF7D2FB89
:1055800001240826CDE90064024618200023414684
:10559000FCF7A0FC071D07EB47004006000E0823A0
:1055A0002D2241460094FCF727FC687800217F1CDF
:1055B000FBF7B8FB024607EB4700CDE90064400665
:1055C000000E00234146FCF785FC074407EB47002B
:1055D0004006000E08232D2241460094FCF70CFCE7
:1055E000287800217F1CFBF79DFB024607EB470054
:1055F000CDE900644006000E00234146FCF76AFC3A
:10560000074407EB47004006000E082320224146CE
:105610000094FCF7F1FB687900217F1CFBF782FB0B
:10562000024607EB4700CDE900644006000E002368
:105630004146FCF74FFC074407EB47004006000ECD
:1056400008232D2241460094FCF7D6FB287900213F
:105650007F1CFBF767FB024607EB4700CDE90064C0
:105660004006000E00234146FCF734FC074407EBDC
:1056700047004006000E08232D2241460094FCF707
:10568000BBFBE87800217F1CFBF74CFB024607EBD5
:105690004700CDE900644006000E00234146FCF7B8
:1056A00019FCBDE8FC810000D41000200249C8703C
:1056B0000120887170470000D41000202DE9FC5FA4
:1056C00000252C46F4F762FCF84FB87900287CD00E
:1056D000A94687F80690FCF7E9F9F878DFF8D0B327
:1056E00001264FF008084FF0100A0E286ED2DFE8AE
:1056F00010F00E008200EB007901BD01E4023704D6
:105700005C05A505F205850646078F07E307F5F753
:10571000C3F801280AD0022808D0042806D0082897
:1057200004D10220FFF7C2FF87F86090CDE900A600
:1057300000211523DFA20846FCF769FC97F86100F9
:1057400010B3CDE9008644460523DFA214210020D2
:10575000FCF75DFCCDE9004697F861200023142199
:105760001E20FCF7B7FBCDE9004697F861000A233D
:1057700000EB400101EB001007EB00121421282080
:1057800002F6EE02FCF743FC97F86000FF2825D0F4
:1057900017F8600FCDE900060A2364221E2118467F
:1057A000FCF7A8FACDE900863A7800232D213220B3
:1057B000FCF790FB00EB4000322101EB4000082396
:1057C0002522C0B22D21009601E0D2E30EE3FCF7C2
:1057D00013FB17F86009642807D007E3CDE90086BA
:1057E00015232D21BAA2142044E287F860900220EC
:1057F000FFF75CFFF1E7F5F74FF801280BD002281F
:1058000009D0042802D0082805D101E0082000E0D2
:105810000320FFF74BFF97F8210638B197F82206CF
:1058200038B1012808D0022811D108E01523ACA214
:1058300007E01523ADA204E01523B0A201E0152373
:10584000B1A2CDE9008600210846FCF7E0FBB8785C
:10585000012802D002280CD101E0AF4801E0AE4897
:105860001230CDE9000609231A460A210020FCF770
:1058700081FBA94818234838CDE900061A460021C3
:105880006820FCF777FBCDE9008644461523A3A2E8
:105890001A210020FCF7BBFBCDE900461523A5A289
:1058A00024210020FCF7B3FBCDE900467A6D0023EC
:1058B00024215420FCF70EFB786D10B90220FFF76D
:1058C000F5FEFFF751FE88E7F4F7E6FF012806D062
:1058D000022804D0042809D0082818D10EE097F82F
:1058E0005C0020F0800087F85C0010E097F85C0016
:1058F00020F0800087F85C00082006E097F85C0044
:1059000020F0800087F85C000320FFF7CFFE97F8B7
:10591000210638B197F8220668B101280ED0022876
:1059200014D118E0CDE900860021152385A2084690
:10593000FCF76DFB15E015236CA201E015236FA2A7
:10594000CDE9008600210846FCF761FB97F8E704E3
:105950000F2803D005E015236BA2F1E70120FFF724
:10596000A5FEB878012802D002280CD101E06A48CF
:1059700001E069481230CDE9000609231A460A21E0
:105980000020FCF7F7FA97F8600010B10020FFF74D
:105990008DFE614818234838CDE900061A460021DB
:1059A0006820FCF7E7FACDE900A65446102367A269
:1059B00014212820FCF72BFBCDE90086152365A2D6
:1059C00024211220FCF723FB97F85C0000067FF5EA
:1059D00078AFCDE90046102363A22E210020FCF70A
:1059E00016FB6EE7F4F758FF012806D0022809D00D
:1059F00004280ED008281ED121E03879D8B1387992
:105A0000401E04E03879032815D23879401C3871DB
:105A100011E0387930B1012806D0022806D00328D9
:105A200009D105E0042004E0052002E0062000E0A2
:105A30000720FFF73BFEF878032805D0CDE60220CB
:105A4000FFF734FE4846E2E73348042200212430C1
:105A500000F0C8FECDE900A938792F49243101EBC7
:105A6000001238790007010E1023F2E3F4F714FF57
:105A7000082802D10320FFF719FEF8780428DDD1A9
:105A8000254804220021643000F0ACFE97F822067D
:105A900020B1012875D0022872D198E01023CDE9F9
:105AA000008612A21946002083E06AE0D41000208C
:105AB000000042424669726D77617265446F776E8D
:105AC0006C6F616400000000506F72743A00000057
:105AD000446F776E6C6F6164204661696C210000D1
:105AE0004E6F205369676E616C00000054797065D9
:105AF0003A53746174696F6E0000000054797065E8
:105B00003A436C6F75640000547970653A436C6F6A
:105B100075642D5465737400BCB001084F66666CE3
:105B2000696E65205265636F72642055706C6F6199
:105B3000640000005265636F7264206E756D62656B
:105B4000723A00004F66666C696E6500424C5545BE
:105B5000534B5900454E4552475920544543484EF2
:105B60004F4C4F47590000005570677261646520C3
:105B700045525220436865636B2047756E000000F4
:105B800019E044461023AFF28C02CDE90086194695
:105B90000020FCF73CFACDE900461023F5A238219D
:105BA0000020FCF734FACDE900461123F34A3821EE
:105BB0001E20FCF72CFA97F8230600B397F823066B
:105BC00001281CD097F82306022854D005E6CDE919
:105BD000008610234446EAA219460020FCF717FA73
:105BE000CDE900461023E3A238210020FCF70FFA8C
:105BF000CDE9004611233821E54A1E20D9E778195E
:105C000090F8610518B96D1CADB2152DF7D3CDE92B
:105C1000008644461023DFA21A210020FCF7F7F982
:105C2000CDE900467A1910231A21202002F2615290
:105C3000FCF7EDF9CDE900461023D8A2242100207D
:105C4000FCF7E5F9CD4ACDE900462421102339328D
:105C50000846FCF7DCF9CDE900461023D1A22E213D
:105C60000020FCF7D4F9C54ACDE900460F232A32BB
:105C70002E2124202EE3CDE9008644461023CBA21A
:105C80001A210020FCF7C3F9BC4ACDE900461023D5
:105C900061321A211E20FCF7BAF9CDE90046102323
:105CA000C0A224210020FCF7B2F9B44ACDE9004695
:105CB000142325322E2100200CE3F4F7EDFD0128FA
:105CC00004D0022807D008280FD10BE0387960B142
:105CD0003879401E04E03879032806D23879401C10
:105CE000387102E00320FFF7E1FCF87805287DD148
:105CF00004220021AF4800F075FDCDE900A63A79F5
:105D0000BA46012300213E20521CFCF7E3F8CDE9FE
:105D1000008647461023A8A200214820FCF777F907
:105D2000DFF890820823A8F1F408CDE900861A462E
:105D300000217820FCF71EF9CDE900761023A1A2FE
:105D400008214820FCF763F908231A4619467820F1
:105D5000CDE90089FCF70EF9CDE9007610239CA26D
:105D600019460020FCF753F99AF8040000EB4001B3
:105D700001EB00110AEB011090F81D0A4FF010031F
:105D8000012840D094A2CDE9007610211E20FCF716
:105D90003EF9CDE90076B046102391A218210020EB
:105DA000FCF735F99AF8040000EB400101EB001014
:105DB0000AEB001090F8160ACDE9007805289AF849
:105DC000040000EB400101EB00100AEB00101CD0B6
:105DD00090F8160A7749403101EB00120C23182184
:105DE0003620FCF714F9C346B84600E025E2CDE9B9
:105DF000007B10237DA220210020FCF708F9092751
:105E00004FF0200A9EE07CA2BDE790F81C0A694989
:105E1000B031E1E707EB47014FF07A09B9EB410FE9
:105E200002D2641CA4B20027307900EB400101EBE0
:105E3000001006EB001000EB051090F8420AC009B4
:105E4000CDE90080307900EB400101EB001006EB5A
:105E5000001000EB051090F8402A0AEBC400C1B214
:105E600007EB47004006000E0023FCF733F83844E8
:105E700087B207EB4701B9EB410F02D2641CA4B211
:105E80000027307900EB400101EB001006EB001019
:105E900000EB051090F8420A0823C00900900AEBB5
:105EA000C400C1B207EB47004006000E2D22FBF7ED
:105EB000A3FF7F1CBFB207EB4701B9EB410F02D232
:105EC000641CA4B20027307900EB400101EB001004
:105ED00006EB001000EB051090F8420AC009CDE96E
:105EE0000080307900EB400101EB001006EB001060
:105EF00000EB051090F8412A0AEBC400C1B207EB91
:105F0000470040065646000E0023FBF7E3FF3844E7
:105F100087B207EB4701B9EB410F02D2641CA4B270
:105F2000002706EBC400C1B207EB47004006000E95
:105F300008233B22CDF800B0FBF75EFF7F1C6D1CF1
:105F4000BFB2ADB22E4E307900EB400101EB001034
:105F500006EB001090F8170AA8423FF65BAFD1E3BA
:105F6000F4F79AFC01284DD0022850D0082858D1C7
:105F700054E0CBE355524C3A000000005716002085
:105F8000547970653A436C6F75642D546173740075
:105F900076910108494343494400000041504E2096
:105FA0003A000000494D45493A0000005353494426
:105FB0003A00000060B101084F6E4C696E65203AEE
:105FC000200000004F66664C696E653A20000000B4
:105FD000547970653A00000052533438350000009F
:105FE00050726F746F636F6C3A00000047756E2DCE
:105FF000416464723A0000004C4F524100000000BE
:10600000D4100020387940B13879401E04E0387946
:10601000032806D23879401C387102E00320FFF7CC
:1060200045FBF87806289AD10126BE71042200218A
:10603000F84800F0D7FBCDE900A63A79012300210A
:106040004020521CFBF746FFCDE90086C3461023D3
:10605000F1A214210020FBF7DAFF092697E006EBF6
:1060600046014FF07A0ABAEB410F02D2641CA4B287
:1060700000264FF00108CDE900B8387900EB400167
:1060800001EB001007EB001000EB051090F8402A20
:106090004FF0140909EBC400C1B206EB46004006FC
:1060A000000E0023FBF716FF304486B206EB4601D4
:1060B000BAEB410F02D2641CA4B20026142000EBFC
:1060C000C400C1B206EB46004006000E08232D2294
:1060D000CDF80080FBF790FE761CB6B206EB4601C9
:1060E000D146BAEB410F02D2641CA4B20026CDE91E
:1060F00000B8387900EBC00101EB002007EBC000CD
:1061000005EB451100EB810090F8140F642110FBA2
:1061100001F0020A142707EBC400C1B206EB4600E7
:106120004006000E0023FBF7D5FE304486B206EB96
:106130004601B9EB410F02D2641CA4B2002607EB62
:10614000C400C1B206EB46004006000E082325221B
:10615000CDF80080FBF750FE761CB6B206EB460188
:10616000B9EB410F02D2641CA4B2002607EBC400B5
:10617000C1B206EB46004006000E08233B22CDF8D4
:106180000080FBF739FE761C6D1CB6B2ADB2A54F90
:10619000387900EB400101EB001007EB001090F89C
:1061A000170AA8423FF65BAFACE2F4F775FB08288C
:1061B00002D10320FFF77AFAF8783C460728F3D19A
:1061C000944804220021403000F00CFBCDE9008609
:1061D00047461023944A14210020FBF718FFA146DC
:1061E00005EB450000EB051109EB0110804690F826
:1061F000280AC0071DD005EB8501142000EB4104DF
:10620000CDE90076E1B2052388A20020FBF7FFFE6E
:10621000CDE90076E1B201236A1C1E20FBF75AFE8D
:10622000CDE9007608F61E22E1B20A232A20FBF708
:10623000EEFE6D1CADB2042DD2D363E2F4F72CFB5D
:10624000012807D002280CD0042812D0082828D111
:106250002BE03EE0387910B13879401E1CE0052073
:106260001AE03879042802D23879401C14E04846F4
:1062700012E03879052814D2DFE800F00305070999
:10628000100009200BE00A2009E00B2007E00C2099
:10629000FFF70CFA97F82006387102E00D20FFF79F
:1062A00005FAF878082804D02CE20220FFF7FEF95E
:1062B000DDE73879574C0422803404EB00100021CC
:1062C00000F090FACDE900A93879102304EB001210
:1062D00000210020EDE1F4F7DFFA012806D00228C2
:1062E00009D004280ED0082849D145E0387978B380
:1062F0003879401E04E03879032840D23879401CB0
:1063000038713CE0387900EB400101EB001007EBFD
:10631000001090F81D0A01280AD0387900EB4001DE
:1063200001EB001007EB001090F81D0A88B126E081
:1063300038794C4600EB400101EB001007EB0010F0
:1063400080F81D9A39790220F3F704FCCBF88842D3
:1063500015E0387900EB400101EB001007EB00106D
:1063600080F81D6A3879FBF7B1F9CBF88862397982
:106370000220F3F7EFFB02E00820FFF797F9F87827
:10638000092891D1042200212A4800F02BFACDE9F6
:1063900000864446152328A214212820FBF737FE47
:1063A000CDE900463A79012314214620521CFBF71F
:1063B00091FD387900EB400101EB001007EB001074
:1063C00090F81D0A01280AD0387900EB400101EB52
:1063D000001007EB001090F81D0A18B10AE0152311
:1063E00017A201E0152319A2CDE900461E210020C5
:1063F000FBF70DFE152318A2322105E1F4F74CFA44
:106400001A4C012834D002283DD0042848D008284E
:106410005AD14AE040B2010847756E2D5253534994
:106420003A000000D4100020BC8E0108506F727436
:106430002D00000050B30108504F52543A000000A4
:10644000545950453A4C4F52410000005459504560
:106450003A525334383500005061737320456E74DE
:106460006572204368616E6765000000D4400020BB
:10647000387948B394F8490010B13879FBF726F918
:106480003879401E0AE0387903281DD294F8490073
:1064900010B13879FBF71AF93879401C387113E0DC
:1064A00084F8496084F83D600EE00820FFF7FEF8AC
:1064B00084F83C6094F8490030B1CBF8889284F8B5
:1064C00049903879FBF702F9F8780A282FD104228D
:1064D00000218F4800F086F945461523AFF2A80247
:1064E000CDE9008612212820FBF791FDCDE9005669
:1064F0003A79012312214620521CFBF7EBFCCDE92F
:106500000056152383A21C210020FBF780FDCDE956
:106510000056152385A226210020FBF778FDCDE942
:106520000056152387A230210020FBF770FD94F858
:106530004900012854D1BE7194F83E0078B1CBF8DF
:10654000889284F83E9038790121FBF78DF9CDE9E6
:106550000086152380A238210020FBF758FD94F80F
:106560004800E8B384F84890CDE9008615237EA260
:1065700038210020FBF74BFDCBF88862C2E0F4F72E
:106580008BF9012813D0022811D0042802D0082842
:106590000DD109E0F2F7FEFE142802D087F86792C9
:1065A00005E087F8676202E00820FFF77FF8F878D7
:1065B0000B2815D1564804220021403000F012F972
:1065C000CDE90086444615236BA21A210020FBF773
:1065D0001EFDCDE90046152324216CA2002000E019
:1065E00069E0FBF714FDCDE9004615236BA22E21CF
:1065F0000020FBF70CFD97F867024FF0150308B178
:106600006CA200E071A23821CDE90046002050E0E4
:10661000F4F742F9012806D002280BD0042812D042
:10662000082821D11DE0387910B13879401E08E0E2
:10663000022006E03879032802D23879401C00E0B5
:106640004846387110E0387987F820060021032089
:10665000F3F780FA40B10220FFF728F8FDF712FEA9
:1066600002E00820FFF722F8F8780C284AD12848E1
:1066700004220021803000F0B5F8CDE900A697F89B
:1066800020065446224D1023C03505EB0012194652
:106690000020FBF7BCFC97F820063979884231D0FE
:1066A000CDE9004638790C2305EB001220210020AB
:1066B000121DFBF7ACFC25E0F4F7EEF8012819D029
:1066C000022817D0042802D0082813D10FE0F3F7CE
:1066D00097FA86F31388BFF34F8F3F4801683F4A0C
:1066E00001F4E06111430160BFF34F8FFEE7082022
:1066F000FEF7DCFFF8780D2804D104220021384889
:1067000000F070F8BDE8FC5FFBF73ABBBDE8FC9F0A
:1067100090B30108313A44697020737769746368F3
:106720002031616E6432204F4E000000323A496ED3
:106730007365727420736C617665206D6F64756C1F
:1067400065000000333A5061737320456E746572C2
:10675000205374617274000053746174653A536518
:106760006E64696E6700000053746174653A436F2C
:106770006D706C6574650000496E736572742055A8
:106780002D4469736B204669727374005468616E9E
:10679000205061737320456E74657200466F726D90
:1067A00061743A46415433323B4D41583A33324793
:1067B0000000000046696E6420552D4469736B2CFF
:1067C0004F7574707574696E67000000537461745E
:1067D000653A49646C6500000CED00E00400FA05C0
:1067E00090B401082DE9F84F00259246884681466D
:1067F000012715E000242E0109EB040101EB08102C
:1068000000EB051000970278E006F1B2000E1023AD
:10681000FBF7F2FA641CE4B2102CEDD36D1CEDB260
:106820005545E7D3BDE8F88F064800210172817213
:1068300001214172C1726422026181710220FEF75E
:1068400035BF0000D4100020124810B5016841F493
:10685000700101601048016841F0010101600E4AB9
:1068600000210832116002680C4B1A400260031DBF
:106870000B4A1A60026822F48022026006480C303B
:106880000160FEF7C9FD03494FF0006080390860E0
:1068900010BD000088ED00E000380240FFFFF6FE6A
:1068A00010300024FEF75EBDC94301827047002905
:1068B000018802D041F0010101E021F001010180D5
:1068C00070470000464910B5884206D101210846AC
:1068D000FEF794FB002101205BE0B0F1804F09D06E
:1068E000404988420DD101210220FEF76FFB0021B3
:1068F000022070E001210846FEF768FB002101201C
:1069000069E03949884206D101210420FEF75EFB87
:10691000002104205FE03549884206D1012108208A
:10692000FEF754FB0021082055E03149884206D18A
:1069300001211020FEF74AFB002110204BE02D49D9
:10694000884206D101212020FEF740FB00212020B3
:1069500041E02949884206D101210220FEF74EFB81
:106960000021022015E02549884202D101210C04B2
:106970000AE02349884202D101214C0404E0214964
:1069800088420AD101218C042046FEF737FB002102
:106990002046BDE81040FEF731BB1B49884206D1B6
:1069A00001214020FEF712FB0021402013E017498F
:1069B000884206D101218020FEF708FB00218020BB
:1069C00009E0134988420AD1841501212046FEF7C7
:1069D000FDFA00212046BDE81040FEF7F7BA10BDD1
:1069E000000001400004004000080040000C00408E
:1069F000001000400014004000040140004001402D
:106A0000004401400048014000180040001C0040C4
:106A10000020004002460020138A92890B4202EABD
:106A2000010202D0002A00D001207047002A82898A
:106A300001D00A4300E08A438281704730B5028862
:106A4000164C174DA0420DD0A8420BD0B0F1804F8C
:106A500008D0144B984205D0134B984202D0134BE8
:106A6000984203D122F070034A881A43104B98428F
:106A700006D0104B984203D022F440730A891A437F
:106A800002804A68C2620A880285A04201D0A842F8
:106A900001D1897A01860121818230BD0000014047
:106AA000000401400004004000080040000C0040C9
:106AB000001000400014004010B5FEF7F9F9FEF791
:106AC0004BFA00F0A9F9F3F73BF9154C14F85C0FF9
:106AD00020F001002070207840F006002070002097
:106AE000608001460120F3F735F8F3F725FEF2F751
:106AF0005DFAF2F7C1FEF3F7E7FEFBF74DF8FFF79B
:106B000093FEF3F787FAFAF761FCFDF7BBFB4FF44E
:106B1000FA6024F8460C012004F8480C10BD00006F
:106B2000D41000202DE9F0410024F3F723FCB94EE6
:106B300096F8F2040025012805D186F8F254F2F700
:106B4000E3FE0120B0713AE104EB440006EB800063
:106B500090F83215012901D180F8325590F831159D
:106B6000002979D190F8A2190129FAD104EB440146
:106B700001EB041106EB011292F8161A00296BD0F2
:106B800080F8A25992F8160A072864D2DFE800F0CC
:106B9000EC04376591E1E10004EBC40000EB042054
:106BA00006EBC00090F8D31E012909D090F8D21E40
:106BB00001EB411100EB810191F8D81E00294AD167
:106BC00090F8D21E491C80F8D21E90F8D01E29B130
:106BD00090F8D01E80F8D21E80F8D05E90F8D21EB9
:106BE00001EB411100EB810191F8D81E052932D04B
:106BF00090F8D21E01EB411100EB8100A6E004EBFE
:106C0000C40000EB042006EBC00090F8D31E01295D
:106C100009D090F8D21E01EB411100EB810191F8EF
:106C2000D81E002917D190F8D21E491C80F8D21E18
:106C300090F8D01E29B190F8D01E80F8D21E80F8AE
:106C4000D05E90F8D21E01EB411100EB810191F86A
:106C5000D81E0F29CCD187E0AFE004EBC40000EBD5
:106C6000042006EBC00090F8D31E012908D090F84C
:106C7000D21E01EB411100EB810191F8D81E71BBCE
:106C800090F8D21E491C80F8D21E90F8D01E29B16F
:106C900090F8D01E80F8D21E80F8D05E90F8D21EF8
:106CA00001EB411100EB810191F8D81E07299FD11A
:106CB0005AE004EBC40000EB042006EBC00191F89D
:106CC000D30E012808D091F8D20E00EB401001EB52
:106CD000800090F8D80E10B991F8D20E19E037E084
:106CE00091F8D23E02EB031393F8413A02EB0017FE
:106CF00097F8517ABB4205D091F8D20E401C81F82A
:106D0000D20E0AE091F8D23E5B1C81F8D23E401CC4
:106D1000C0B292F8173A8342E2D891F8D00E28B167
:106D200091F8D00E81F8D20E81F8D05E91F8D20E93
:106D300000EB401001EB800090F8D80E052813D02E
:106D400091F8D20E00EB401001EB800080F8D85E85
:106D50000AE004EBC40000EB042006EBC00090F84E
:106D6000D21E491C80F8D21E04EBC40000EB0420A4
:106D700006EBC00090F8D21E92F8172A914201D378
:106D800080F8D25E90F8D11E51B190F8D21E80F8F2
:106D9000D01E90F8D11E491E80F8D21E80F8D15E18
:106DA00090F8D21E01EB411100EB810191F8DC2E2D
:106DB00090F8D21E2046F8F7B1FE641CE4B296F8B3
:106DC0006C09A0423FF6C0AE96F8220620B196F8B4
:106DD000FE04012807D010E096F80A0501280CD11E
:106DE00086F80A5501E086F8FE5496F8252696F8AE
:106DF000211696F82206FCF703FDF3F74DFE96F8F0
:106E0000240618B186F82456FBF750F9BDE8F04186
:106E1000FEF754BCD4100020FEB501210024084622
:106E2000FEF7C8F8A720ADF80000002640F2E730D2
:106E300001904FF08045ADF80260ADF808606946FA
:106E40002846FFF7FBFD724981F83E6604EB4400DB
:106E500001EB800091F83E3600F5A66201EB83035A
:106E6000C3F8402691F83E26521C81F83E2691F840
:106E70003E3600F51A6201EB8303C3F8402691F811
:106E80003E26521C81F83E2691F83E3600F51762E8
:106E900001EB8303C3F8402691F83E26521C81F88B
:106EA0003E2691F83E2600F5405001EB8202C2F8E2
:106EB000400691F83E06401C81F83E0604EBC402F1
:106EC00002EB0422002001EBC20300EB401291F818
:106ED0003E6603EB820201EB860602F6E462C6F828
:106EE000402691F83E26521C81F83E26401CC0B236
:106EF0001028EAD3641CE4B2042CA7D3454891F8C7
:106F00003E2601EB8202C2F8400691F83E06401C84
:106F100081F83E063F4891F83E26283801EB820270
:106F2000C2F8400691F83E06401C81F83E063948FA
:106F300091F83E261C3801EB8202C2F8400691F817
:106F40003E06401C81F83E06324891F83E26103835
:106F500001EB8202C2F8400691F83E06401C81F81F
:106F60003E062D4891F83E2601EB8202C2F840060B
:106F700091F83E06401C81F83E06284891F83E26CE
:106F800001EB8202C2F8400691F83E06401C81F8EF
:106F90003E06204891F83E26343801EB8202C2F8C2
:106FA000400691F83E06401C81F83E061C4891F8C8
:106FB0003E2601EB8202C2F8400691F83E06401CD4
:106FC00081F83E06124891F83E26083001EB820215
:106FD000C2F8400691F83E06401C81F83E06104873
:106FE00091F83E260C3801EB8202C2F8400691F877
:106FF0003E06401C81F83E0601212846FFF757FC5B
:10700000012211462846FFF711FD00F00BF8FEBDE6
:10701000D4100020F8150020FC160020341A00209F
:107020001041002008B51C208DF8000001208DF8CB
:10703000010002218DF802108DF803006846FAF76E
:10704000E9FC08BDF9F7DCBEF9F7FABEFDF748B870
:10705000F9F7B0BEF9F712BFF3F78ABAC943018056
:1070600070470029818902D041F4005101E021F4E8
:10707000005181817047002A828A01D00A4300E0D2
:107080008A438282704700001C4910B5884206D1AD
:1070900001211020FDF7B2FF0021102028E018493F
:1070A000884202D101214C0410E01649884202D1E5
:1070B00001218C040AE01449884202D10121CC0448
:1070C00004E0124988420AD101210C052046FDF74F
:1070D0007DFF2046BDE810400021FDF777BF0C4939
:1070E000884209D101212020FDF788FF00212020BE
:1070F000BDE81040FDF782BF10BD00000010014048
:107100000044004000480040004C00400050004057
:10711000001401400246002012880A4200D00120DB
:10712000704770B501F01F0501260024C1F342131A
:1071300006FA05F2012B0FD0022B0FD0838A4FEAFB
:1071400011210088134206FA01F600EA060001D078
:1071500000B10124204670BD8389F0E7038AEEE781
:1071600010B5C1F3421301F01F040121A140012B0E
:1071700007D0022B07D01430002A026805D00A433A
:1071800004E00C30F8E71030F6E78A43026010BDE7
:107190007FB50446008A0D46C98820F4405001435B
:1071A0002182A08941F20C618843A9882A89114370
:1071B0006A8902431143A181A08A20F44071A88901
:1071C0000843A0826846FDF725FF1A48844202D092
:1071D0001948844201D1039800E00298A18909046A
:1071E00000EBC00101EB0010296801D5490000E067
:1071F0008900B0FBF1F06422B0FBF2F109010B0948
:107200006FF018056B4300EB8300A3891D044FF05A
:10721000320306D503EBC000B0FBF2F000F007002C
:1072200005E003EB0010B0FBF2F000F00F000843A4
:1072300020817FBD001001400014014070B5002482
:10724000064DFDF78BFE20B1641CAC42F9D3FA2049
:1072500070BDBDE87040F2F7CBB80000404B4C0069
:107260000FB4084B10B504A902AA039801F0E0F985
:10727000044602A9002001F006FC204610BC5DF87F
:1072800014FB0000878A010803B4019841000098AC
:1072900050EAC12018BF04204A0D18BF40F0010079
:1072A00040F2FF72B2EB515F08BF40F002000128CC
:1072B00008BF052002B0704730B583B0044601F026
:1072C00093F99FED090B05468DED000B0022214639
:1072D0006846F1F71CFA284601F09CF99DED000B79
:1072E00003B030BD000000000000000000000000FE
:1072F00070B5D94B00242DED020B2DED108BDDE97F
:107300001010984205DA20F000429A4201D809D1C3
:1073100041B19DED100BBDEC108B02B0BDE870408B
:1073200001F01EB9B0F5801F26DA11430BD00028FA
:1073300013DA012001F06EF9BDEC108B02B0BDE84C
:10734000704001F021B9022001F064F901F0F0F879
:1073500051EC100B81F000419EE06FF035049FED81
:10736000C00B53EC102B9DED100B51EC100BF1F7F3
:1073700045F8CDE91001084604EB2051C0F3130491
:10738000B948A1F2FF31204400F4801080F07F6200
:1073900082F04052224301EB20559FEDB50B119234
:1073A00053EC102B9DED100B51EC100BF1F720F866
:1073B00041EC180BA01CC0F313009FEDAFDB9FED59
:1073C000B0EBB14E7E4403286CD296ED000B51EC2D
:1073D000180B53EC102BF1F7DBFC1DD1002D01BF76
:1073E00096ED000BBDEC108B02B070BD2846F1F796
:1073F0006CFA41EC180B53EC1D2BF0F7FFFF41EC3E
:10740000190B53EC1E2B51EC180BF0F7F7FF53EC54
:10741000192BF0F74CFF3FE09FED9D0B51EC180B43
:1074200053EC102BF0F7EAFF9FED9B1B53EC112B55
:10743000F0F7E1FF41EC190B53EC182B51EC180B52
:10744000F0F7DCFF53EC192BF0F7D8FF41EC190BE8
:10745000002D04BF53EC192B51EC180B1AD0284601
:10746000F1F733FA41EC1A0B53EC1D2BF0F7C6FF82
:1074700053EC192BF0F7BFFF53EC182BF0F7B8FFC4
:1074800041EC180B53EC1E2B51EC1A0BF0F7B6FF26
:1074900053EC182BF0F7ACFFBDEC108B02B041ECB5
:1074A000100B70BD9FED7E0B51EC180B53EC102BA5
:1074B000F0F7FDFE41EC100B51EC180B53EC102BC8
:1074C000F1F70EF841EC190B2846F1F7FEF941EC03
:1074D0001B0B53EC192B51EC190BF0F78FFF41EC00
:1074E0001A0B714853EC1A2B261851EC1A0BF0F7B3
:1074F00085FF41EC1F0B6D48C4F1510404F5D724FE
:10750000B0EE4F0AF0EE6F0A0321784400F094FFCA
:1075100053EC1F2B51EC100BF0F770FF41EC1C0BE0
:107520006348B0EE4F0AF0EE6F0A0421784400F091
:1075300083FF53EC1A2B51EC100BF0F75FFF344331
:1075400053EC1C2BF0F7B3FE41EC1C0B002C4CDD74
:107550009FED510B51EC180B53EC102BF0F74EFF35
:1075600053EC182BF0F74AFF41EC1A0B55B353ECD0
:107570001D2B51EC1B0BF0F741FF41EC1D0B53ECA5
:107580001C2B51EC1A0BF0F792FE53EC192BF0F771
:1075900035FF53EC1D2BF0F78AFE53EC1A2BF0F756
:1075A0002AFF53EC182BF0F723FF41EC180B53EC98
:1075B0001E2B51EC1B0BF0F721FF53EC182BF0F7AF
:1075C00017FF69E753EC1C2B51EC1A0BF0F76FFE19
:1075D00053EC192BF0F712FF53EC1A2BF0F70BFFBB
:1075E00053EC182BF0F707FF56E735B353EC1D2B80
:1075F00051EC1B0BF0F702FF41EC1A0B53EC1C2B68
:1076000051EC180BF0F7F4FE53EC192BF0F7F6FEE3
:1076100053EC1A2BF0F7ECFE53EC182BF0F7E8FEC6
:1076200041EC180B53EC1E2B51EC1B0BF0F7E6FE54
:1076300053EC182BF0F7DCFE2EE753EC1C2B51EC2F
:10764000180BF0F7D5FE53EC192BF0F7D7FE53ECDF
:10765000182BF0F7D0FE1FE70000F07F00000000BD
:107660000000000000005043645F090000000000BB
:10767000000000000000F03F763C7935EF39EA3D2C
:107680000000E0FE422EE63FC8410000000000007E
:10769000555555555555D53F000000000000E03FB9
:1076A000000000000000004086EBF9FF4A400000A7
:1076B000404000000000000070B5414A00252DED5B
:1076C000020B2DED048BDDE90404944205DA24F06D
:1076D0000041914201D809D140B19DED040BBDECB0
:1076E000048B02B0BDE8704000F03ABFB4F5801FD3
:1076F00026DA08430BD0002C13DA012000F08AFFB1
:10770000BDEC048B02B0BDE8704000F03DBF02202C
:1077100000F080FF00F00CFF51EC100B81F00041F5
:1077200046E09FED290B6FF0350553EC102B9DEDD6
:10773000040B51EC100BF0F761FECDE904010C468F
:1077400005EB2450A0F2FF30C10F40F2FF32521A75
:1077500062F31F540844F1F7B8F805949DED040B4B
:1077600041EC180B51EC100B01F0B4FA9FED181B13
:1077700053EC112BF0F742FE9FED170B41EC190B68
:1077800053EC102B51EC180BF0F738FE53EC192B7F
:10779000F0F78DFD9FED120B41EC190B53EC102B04
:1077A00051EC180BF0F72AFE53EC192BF0F77FFD84
:1077B000BDEC048B02B041EC100B70BD000000006A
:1077C0000000F07F000000000000000000005043B7
:1077D0000EE526157BCBDB3F362BF111F3FE593D31
:1077E00000609F501344D33F2DE9F04D2DED040B65
:1077F0002DED0E8B96B0DDE92550279CDDF890A08D
:1078000025F0004624F00048BAF1000F14BF012112
:10781000002101EB4502FC4953184A1093422AD338
:10782000002814BF0123002303EB44030B44F74952
:107830008B4220D358EA00019FEDF59B76D0DFF80C
:10784000D8B35D4503D1BAF1000F05D188E0BAF194
:10785000000F08BF002100D0012101EB450111F507
:10786000001F08D8002814BF0121002101EB4401AA
:1078700011F5001F0BD99DED261B9DED240B16B0B5
:10788000BDEC0E8B04B0BDE8F04D00F073BE0027D8
:10789000002DBCBFE149884521DAE1498845A8BFF0
:1078A00002271CDAC3451ADCDE4901EB28511429F2
:1078B00008DDC1F1340220FA02F101FA02F282423B
:1078C0000DD108E058B9C1F1140228FA02F101FA09
:1078D00002F2424503D101F00101C1F1020756EA6B
:1078E0000A0124D1002C22DA002D18BF022F01D06A
:1078F000012F0AD0022000F08DFE16B0BDEC0E8BD9
:1079000004B0BDE8F04D00F013BE022000F082FE8E
:1079100000F00EFE51EC100B81F0004141EC100B19
:1079200016B0BDEC0E8B04B0BDE8F08D18E09FEDF5
:10793000BEAB9FEDBF8B002871D1B848804522D1E6
:1079400005F1804010F5801008BFBAF1000F07D094
:10795000B3450ADC002CA8BF9DED260BE0DA0DE054
:10796000B0EE490AF0EE690ADAE7002C06DA9DED7E
:10797000260B51EC100B81F000416FE0AE487844CB
:1079800090ED000BCCE7D8454DD1002C48DA2EB154
:1079900086423AD1BAF1000F42D126E0BAF1000F87
:1079A00013D0022000F036FE00F0FEFD8DED020B3C
:1079B0009DED240B8DED000B10EE900A039961F301
:1079C0001E0003909DED020BAAE78DED02AB9DED2D
:1079D000240B1AEE901A10EE900A8DED000B61F355
:1079E0001E0003909DED020B9AE78DED028B9DED3D
:1079F000240B18EE901A10EE900A8DED000B61F337
:107A00001E0003909DED020B8AE709DA9DED240B21
:107A100051EC190B53EC102BF0F762FD1EE020E047
:107A20009DED240B7CE786421BDAB4F1804F0DD02C
:107A3000A4F10050B0F1FF5013D1002D11DB9DEDEA
:107A4000240B51EC100B01F0D0F907E09DED240B55
:107A500053EC102B51EC100B00F0C2BC41EC100B9E
:107A60005EE79DED240B51EC100B01F026F8BAF106
:107A7000000FCDE90E0142D19FED710B46B3A6F187
:107A8000E040B0F17F600CD05E4538D1002D00DAC7
:107A9000A7B3022F0CBF01204FF0FF30F0F715FF06
:107AA000DCE7002D01DD002C0DDA002D01DD002CBE
:107AB0001FDB002D16DA002C14DB012F08BF9FED11
:107AC000620B3FF42DAFB0EE4A0AF0EE6A0A27E7E8
:107AD000022F18BF002D0CD0012F0AD1002DFFF668
:107AE0001FAF06E0002DB8BF002C08DA012F3FF4CD
:107AF00017AFB0EE480AF0EE680A11E71BE001206C
:107B000000EBE57050EA070115D0791EB0EE498A06
:107B1000F0EE698A084308BF9FED4D8B4E48002563
:107B2000804570DD4D494E48884514DDB0420DDB7F
:107B3000002C19DB2FE0012000F06CFD16B0BDEC2D
:107B40000E8B04B0BDE8F04D00F01EBDB34502DC65
:107B5000002C09DC1FE0864202DA002C1BDA03E06D
:107B60005E452BDD002C16DD022000F053FD00F0F9
:107B70001BFD8DED020B53EC1A2B51EC180BF0F79B
:107B80003DFCCDE900010399019861F31E000390CB
:107B90009DED020BC4E6022000F03CFD00F014FD58
:107BA00010EE901A18EE900A8DED020B8DED008B01
:107BB00061F31E0003909DED020BB1E69DED0E0BEF
:107BC00053EC192B51EC100BF0F712FC9FED260B28
:107BD000CDE9080153EC102B9DED080B51EC100B77
:107BE000F0F70CFC9FED221B53EC112BF0F703FC7C
:107BF0009DED081B53EC112BF0F700FC9FED1E1BB5
:107C000053EC112B3CE08CE0FFFF1F00FFFF0F0047
:107C1000000000000000F03F0000F03F0000F07F97
:107C20000000404301FCFFFF000000000000F07F67
:107C300000000000000000000E3C000000000000FA
:107C40000000000000000080000000000000F0FFC5
:107C5000000000000000F0BF0000E0410000F04321
:107C6000FFFFEF3F00000000000000000000D03FD9
:107C7000555555555555D53F000000000000E03FD3
:107C8000F0F7B9FB9DED080B41EC1A0B53EC102BF0
:107C900051EC100BF0F7B2FB53EC1A2BF0F7AEFBE4
:107CA00041EC1A0B9FEDFE0B53EC102B9DED080BD6
:107CB00051EC100BF0F7A2FB41EC1B0B9FEDFA0B04
:107CC00051EC1A0B53EC102BF0F798FB41EC1A0B0C
:107CD0009FEDF70B53EC102B9DED080B51EC100BA7
:107CE000F0F78CFB53EC1A2BF0F782FB41EC1A0BEC
:107CF00051EC1B0B53EC1A2BF0F7D9FA0690CDE997
:107D000006519DED060B53EC1B2B51EC100BF0F7BD
:107D10006FFB53EC1A2BF0F76EFB41EC100B00F0ED
:107D2000A1B90020B6F5801F0EDA9FEDE30B53ECEE
:107D3000102B9DED0E0B51EC100BF0F75FFBCDE916
:107D40000E016FF034000E4600EB2650A0F2FF3714
:107D5000C6F31300DA4940F07F6646F04056884289
:107D6000D8BF002408DDD7498142C8BF012403DC05
:107D70000024A6F580167F1CD348784400EBC4008D
:107D80000F9690ED00CB9DED0E0B53EC1C2B51ECA0
:107D9000100BF0F72DFB9DED0E0B41EC1B0B53EC84
:107DA0001C2B51EC100BF0F782FA41EC100B51EC4C
:107DB000190B53EC102BF0F793FB41EC1D0B51EC1E
:107DC0001B0B53EC1D2BF0F719FB41EC1A0BBF48B2
:107DD0008DED10AB7844109590ED000B4FF00050F6
:107DE00040EA660000EB84408DED080B00F50020B2
:107DF00009909DED080B53EC1C2B51EC100BF0F788
:107E0000F7FA9DED0E1B53EC112BF0F7F4FA41EC51
:107E1000100B53EC102B9DED100B51EC100BF0F7E9
:107E2000EDFA9DED080B41EC1C0B53EC102B9DED76
:107E3000100B51EC100BF0F7E1FA53EC1B2BF0F7A1
:107E4000DAFA53EC1C2BF0F7D3FA53EC1D2BF0F7B6
:107E5000D5FA41EC1C0B53EC1A2B51EC1A0BF0F732
:107E6000CDFA41EC1B0B9A480621B0EE4B0AF0EE1E
:107E70006B0A784400F0E0FAB0EE401AF0EE601AB7
:107E8000B0EE41DAF0EE61DA53EC1B2B51EC1B0B38
:107E9000F0F7B4FA53EC1D2BF0F7B0FA9DED100B90
:107EA00041EC1B0B53EC1A2B51EC100BF0F7FFF9C4
:107EB00053EC1C2BF0F7A2FA53EC1B2BF0F7F7F95D
:107EC0009DED100B41EC1B0B53EC102B51EC100BE8
:107ED000F0F794FA41EC1D0B9FED7FEB53EC1E2B5A
:107EE000F0F7E5F953EC1B2BF0F7E1F90890CDE939
:107EF00008519DED080B53EC1E2B51EC100BF0F7C5
:107F000077FA53EC1D2BF0F773FA53EC1B2BF0F7B9
:107F100072FA9DED080B41EC1D0B53EC102B9DEDFF
:107F2000100B51EC100BF0F769FA41EC1B0B53EC02
:107F30001A2B51EC1D0BF0F761FA9DED080B41EC8B
:107F40001A0B53EC102B51EC1C0BF0F757FA53ECB7
:107F50001A2BF0F7ACF941EC1A0B51EC1B0B53EC5C
:107F60001A2BF0F7A4F90C90CDE90C519DED0C0BF8
:107F700053EC1B2B51EC100BF0F73AFA53EC1A2B85
:107F8000F0F739FA41EC1B0B9FED550B53EC102B1E
:107F90009DED0C0B51EC100BF0F730FA41EC1A0B85
:107FA0009FED510B51EC1B0B53EC102BF0F726FA05
:107FB00041EC1B0B9FED4E0B53EC102B9DED0C0B6E
:107FC00051EC100BF0F71AFA53EC1B2BF0F76FF98A
:107FD00041EC100B4848784400EBC40090ED001BC6
:107FE00051EC100B53EC112BF0F761F941EC1B0B2A
:107FF0003846F0F76AFCCDE9080153EC1B2B51EC35
:108000001A0BF0F754F941EC100B3C48784400EBA4
:10801000C40090ED00CB51EC100B53EC1C2BF0F78F
:1080200046F99DED081B53EC112BF0F740F9069033
:10803000CDE906519DED080B53EC102B9DED060B81
:1080400051EC100BF0F7D4F953EC1C2BF0F7D0F9EE
:1080500053EC1A2BF0F7CCF953EC1B2BF0F7CBF9C0
:1080600041EC100B9DED261B53EC102B8DED001BEE
:1080700000959DED260B51EC100BF0F7BFF99DED2F
:10808000000B41EC1A0B53EC102B9DED260B51EC21
:10809000100BF0F7ADF99DED061B53EC112B2FE003
:1080A000000000604715F73FFE822B654715F73F3C
:1080B00044DF5DF80BAE543E00000000000040437A
:1080C0008E9803007AB60B0052370000B8370000D4
:1080D0008A36000000000000000000000000084098
:1080E000000000E009C7EE3FFD033ADC09C7EE3FA0
:1080F000F5015B14E02F3EBE16350000D0340000C1
:10810000F0F77CF953EC1A2BF0F7D1F89DED060B44
:1081100041EC1A0B53EC102B9DED000B51EC100BA6
:10812000F0F76CF9CDE90C019DED0C0B51EC1A0B3D
:1081300053EC102BF0F7BBF8CDE902010C46AA492D
:108140008C422FDB611A084318D19DED0C0B53ECC8
:10815000102B9DED020B51EC100BF0F749F941EC9F
:108160001B0B9FEDA30B51EC1A0B53EC102BF0F7EC
:108170009EF853EC1B2BF0F7B9FB2DD2022000F038
:1081800049FA00F011FA10EE901A18EE900A8DEDEF
:10819000020B8DED008B61F31E0003909DED020B31
:1081A000FFF7BEBB944A24F00041914214D3934997
:1081B000214408437FF4EFAC9DED0C0B53EC102BE6
:1081C0009DED020B51EC100BF0F712F953EC1A2B4A
:1081D000F0F78CFB7FF6DFAC24F000408849894A39
:1081E000002601EB205182422BDA481C4FF480110B
:1081F00021FA00F02044844AC0F30A517A44A1F2E3
:10820000FF3192ED000B814A8DED080BCA4020EA48
:108210000202C0F3130040F48010C1F1140120FAEF
:1082200001F60992002CB8BF76429DED080B53EC85
:10823000102B9DED0C0B51EC100BF0F7D9F8CDE99C
:108240000C019DED0C0B51EC1A0B53EC102BF0F7BD
:108250002EF89FED6F0B0890CDE9085153EC102BD1
:108260009DED080B51EC100BF0F7C8F841EC1B0B1F
:108270009FED690B53EC102B9DED080B51EC100B8F
:10828000F0F7BCF89DED0C0B41EC1C0B53EC102BE4
:108290009DED080B51EC100BF0F7AAF853EC1A2BDC
:1082A000F0F7A9F89FED5E1B53EC112BF0F7A6F841
:1082B00053EC1C2BEFF7FBFF41EC1A0B51EC1B0BA3
:1082C00053EC1A2BEFF7F3FFCDE902019DED020B02
:1082D00053EC1B2B51EC100BF0F78AF853EC1A2BD4
:1082E000F0F789F89DED020B41EC1A0B53EC102BC3
:1082F00051EC100BF0F782F8CDE908014A489DEDEA
:10830000080B0521784400F097F89DED081B51EC0F
:10831000100B53EC112BF0F771F89DED021B53EC91
:10832000112BF0F768F8CDE906019DED020B53EC37
:108330001A2B51EC100BF0F761F853EC1A2BEFF7F6
:10834000B6FF9FED3B0B41EC1A0B53EC102B9DED50
:10835000060B51EC100BF0F74BF89DED060B41ECC2
:108360001B0B53EC102B9DED020B51EC100BF0F797
:1083700045F853EC1B2BF0F7B3F853EC1A2BF0F73E
:1083800037F89DED021B53EC112BF0F731F853EC4D
:10839000192BF0F730F8CDE9020101EB0650011579
:1083A0000029C8BF039015DC9DED020B324651EC4D
:1083B000100BF0F773FAFEF767FF042808BF00F010
:1083C00003F932469DED020B51EC100BF0F766FA03
:1083D000CDE902019DED020B51EC180B53EC102B73
:1083E000F0F70CF8FFF73ABB0000904000000000E7
:1083F000FE822B654715973C00CC904000346F3FC0
:1084000001FCFFFF0000E03F90330000FFFF0F0082
:1084100000000000432EE63F396CA80C615C20BED2
:10842000EF39FAFE422EE63F28320000000000003D
:10843000000000000000004070B504462DED028BE6
:108440004D1E00EBC500B0EE408AF0EE608A90ED64
:10845000000B35F0060017D053EC182B51EC100B25
:10846000EFF7CCFF41EC100B6D1E04EBC50090ED57
:10847000001B51EC100B53EC112BEFF718FF41ECE4
:10848000100B35F00600E7D1022D36D0042D1CD09C
:10849000062D1CBFBDEC028B70BD53EC182B51ECAC
:1084A000100BEFF7ABFF94ED0A1B53EC112BEFF71A
:1084B000FEFE53EC182BEFF7A1FF94ED081B53ECD5
:1084C000112BEFF7F4FE41EC100B53EC182B51EC91
:1084D000100BEFF793FF94ED061B53EC112BEFF706
:1084E000E6FE53EC182BEFF789FF94ED040B53ECE9
:1084F000102BEFF7DCFE41EC100B53EC182B51EC7A
:10850000100BEFF77BFF94ED021B53EC112BEFF7F1
:10851000CEFE53EC182BEFF771FF94ED001B53ECDC
:10852000112BEFF7C4FEBDEC028B41EC100B70BDBC
:108530009FED070B10B553EC102B9FED070B51EC83
:10854000100BEFF7CDFF41EC100B10BD0000000049
:108550000000000000000000000000000000F03FEC
:1085600010B553EC102B51EC100BEFF7A0FE41ECC3
:10857000100B10BD10B553EC112B51EC100BEFF795
:1085800096FE41EC100B10BD9FED050B10B553ECA2
:10859000102B51EC100BEFF7A3FF41EC100B10BDAB
:1085A00000000000000000009FED050B10B553EC2B
:1085B000102B51EC100BEFF721FF41EC100B10BD0D
:1085C00000000000000000709FED050B10B553EC9B
:1085D000102B51EC100BEFF711FF41EC100B10BDFD
:1085E0000000000000000010014800687047000013
:1085F000D010002002E008C8121F08C1002AFAD1DA
:1086000070477047002001E001C1121F002AFBD112
:10861000704700000149086070470000D01000203A
:1086200030380A2801D2012070470020704700002E
:108630002DE9FF4F8DB00F460546002606E02528A0
:108640000BD0DDE90F1290476D1C761C28780028AE
:10865000F5D111B03046BDE8F08F0024A246A14606
:108660000122E94900E0044315F8013F203B02FAEA
:1086700003F00842F7D128782A2810D06FF02F0293
:108680002878A0F13001092914D80AEB8A0102EBFD
:10869000410144F0020400EB010A6D1CF0E701CF38
:1086A0005FEA000A03D544F40054CAF1000A44F01A
:1086B00002046D1C28782E2817D115F8010F44F0FC
:1086C00004042A280ED06FF02F022878A0F1300180
:1086D00009290AD809EB890102EB410100EB0109E4
:1086E0006D1CF2E757F8049B6D1C28786C280FD09E
:1086F00006DC4C2817D068280DD06A2814D104E075
:10870000742810D07A280FD10DE044F400140AE048
:1087100044F4801401E044F440146978814202D1A9
:1087200004F580146D1C6D1C28786E281ED00CDC9E
:10873000632830D004DC00288BD0582811D19FE06A
:10874000642867D069280CD164E073282DD004DC3C
:108750006F2872D0702804D194E075286ED07828E4
:108760006DD0DDE90F129047761C4BE1C4F3025047
:10877000022806D0032809D0042801CF09D00660BA
:1087800040E101CFF117C0E900613BE101CF068074
:1087900038E1067036E117F8040B8DF80000002070
:1087A0008DF80100EB46012003E057F804BB4FF0C1
:1087B000FF3061074FF0000102D40DE008F1010124
:1087C000884649450FDA8045F8DB1BF80810002978
:1087D000F4D108E008F1010188468142FADB1BF878
:1087E00008100029F6D1DDE90F23AAEB0800814625
:1087F000214600F031F9304400EB080604E0DDE9E1
:108800000F121BF8010B9047B8F10108F7D221466F
:108810004846F2E00A21C4F302524FF0000B0891DF
:10882000022A04D001CFC117032A09D00AE0FF1D94
:1088300027F00707F7E8020108E02CE01EE01FE040
:1088400000B2C117042A01D140B2C117021E71F152
:10885000000206DA0023D0EB030063EB01012D22B6
:1088600002E0220504D52B228DF82420012203E00A
:10887000E20701D02022F7E7904653E00A210BE0FF
:10888000102109E010214FF0000B44F004044FF0D8
:108890000809089103E008214FF0000B0891C4F388
:1088A0000252022A04D001CF0021032A06D006E09A
:1088B000FF1D27F00707F7E8020103E080B2042A52
:1088C00000D1C0B24FF0000822072BD52A78702AB9
:1088D00007D0DDF820C08CF0100C5CEA0B0C05D042
:1088E0000EE040228DF82420012208E050EA010326
:1088F00006D030238DF824308DF8252002229046B2
:10890000089B83F0080353EA0B030BD150EA0102E2
:1089100001D1620706D530228DF824204FF00108DE
:10892000A9F101092A78582A04D038A20B9208AA82
:108930000A920BE03AA2F9E75B46089AEFF742FC8D
:108940000B9B9B5C0A9A521E0A92137050EA01021A
:10895000F2D10A98ADEB000000F1200B600702D5C0
:1089600024F4803401E04FF00109D94502DDA9EB80
:108970000B0000E0002000EB0B0141440890AAEB43
:10898000010AE00306D4DDE90F232146504600F03A
:1089900063F806444FF0000908E009A911F809003E
:1089A000DDE90F12904709F10109761CC145F4DB9E
:1089B000E0030CD5DDE90F232146504600F04CF8CA
:1089C000064404E0DDE90F1230209047761C089938
:1089D000481E08900029F5DC08E00A980A990078FA
:1089E000491C0A91DDE90F129047761CBBF100018A
:1089F000ABF1010BF1DC21465046DDE90F2300F01D
:108A000019F806446D1C21E6092801003031323383
:108A100034353637383961626364656600000000BA
:108A200030313233343536373839414243444546A4
:108A3000000000002DE9F041044600251E461746BF
:108A4000880404D405E039462020B0476D1C641E1C
:108A5000F9D52846BDE8F0812DE9F041044600250E
:108A60001E469046C80301D5302700E02027880421
:108A700004D505E041463846B0476D1C641EF9D563
:108A80002846BDE8F0810A68531C0B6010707047DF
:108A9000002806D04DF6BC231946491EFDD2401EC3
:108AA000FAD17047002100EB800002E000BF491CB2
:108AB000C9B2B1EB400FF9D3704782B0CDE90001E4
:108AC00021F0004001909DED000B02B051EC100B25
:108AD0007047000010B50E4C10212046F1F745FC00
:108AE000206840F48060206020212046F1F73DFCA2
:108AF0000220FFF7D7FF10212046F1F738FC0220B3
:108B0000FFF7D0FF2046BDE810401021F1F72DBC43
:108B10000014024010B50E4C10212046F1F725FC40
:108B2000206840F48060206020212046F1F71FFC7F
:108B30000220FFF7B7FF10212046F1F718FC0220B2
:108B4000FFF7B0FF2046BDE810401021F1F70DBC43
:108B5000001402402DE9F041154E0746002430680C
:108B600020F440603060254610213046F1F7FDFBCF
:108B70000220FFF797FF10213046F1F7F8FB60065F
:108B8000040E20213046F1F7E9FB08B144F001045E
:108B90000120FFF787FF6D1CEDB2082DE4D317B15C
:108BA000FFF798FF01E0FFF7B5FF2046BDE8F08131
:108BB0000014024070B5164E05463046316841F447
:108BC000806131601021F1F7D0FB002428064FF0BE
:108BD0002001304602D5F1F7CAFB01E0F1F7C5FBF1
:108BE0006806050E0220FFF75DFF10213046F1F701
:108BF000BEFB0220FFF756FF10213046F1F7B5FB10
:108C00000220FFF74FFF641CE4B2082CDED370BDD6
:108C10000014024010B50B4C206840F480602060C6
:108C200020212046F1F7A3FB10212046F1F79FFBFE
:108C30000420FFF737FF2046BDE810402021F1F760
:108C400094BB00000014024010B50B4C206840F4A7
:108C50008060206020212046F1F787FB0420FFF789
:108C600021FF10212046F1F782FB2046BDE810408D
:108C70002021F1F77CBB00000014024070B5144DB8
:108C80000024286820F44060286020212846F1F75D
:108C90006EFB0120FFF706FF10212846F1F767FB66
:108CA0000120FFF7FFFE07E0641CE4B2FA2C03D9B1
:108CB000FFF7CAFF012070BD20212846F1F74EFBC7
:108CC0000028F1D110212846F1F74FFB002070BD9C
:108CD0000014024010B541EC100BFEF709FB51ECFB
:108CE000100B10BD70B5FCF74DFA062000F0BEF871
:108CF000552000F0DBF800F0AFF8124E04464FF4B8
:108D0000805529463046F1F730FB29460E48F1F7E9
:108D10002EFBAA2C11D1152000F0A8F8062000F097
:108D2000C5F81420FFF7BEFE00F096F80446294669
:108D30003046F1F71CFB512C01D0FA2070BD1420F5
:108D400070BD000000040240000C02404FF40041DE
:108D50000803F8F791FE4FF08040FDF7B3FD0F4890
:108D6000FEF792F90E48F0F7B5FC0D483030F0F7F9
:108D7000B1FC0C48F1F734FA0B48F1F731FAF1F78E
:108D80009BFD002080F310884FF47A70FFF780FE7F
:108D9000FDF792FEFDF7C6FEFCE700000010014063
:108DA0008864024000000240000402402DE9F041C6
:108DB00004460E4600250846EFF763FA07000ED179
:108DC0000120BDE8F0816D1C3178ADB2884205D13B
:108DD0003A4631462046EFF75BFA20B1641C207812
:108DE0000028F0D1EDE72846EBE700B52DED048B28
:108DF00083B041EC190BEFF779FF41EC180B18EE3B
:108E0000100A18EE901A8DED008B002818BF012073
:108E1000084320F00040C0F17F6000F1E040C00F47
:108E200014D019EE101A19EE900A8DED009B00294E
:108E300018BF0121084320F00040C0F17F6000F11D
:108E4000E040C00F04BF0120FFF7E4FB51EC180B1A
:108E500003B0BDEC048B00BD10B50120FFF722FE6E
:108E6000BDE81040FF20FCF7FDB9000070B50D4EC5
:108E700004464FF4805529463046F1F778FA03202E
:108E8000FFF710FE29463046F1F76FFA29460648EB
:108E9000F1F76DFA2046FCF7E5F9BDE870400320D4
:108EA000FFF700BE00040240000C024010B5FCF7C2
:108EB000D9F9BDE810400120FFF7F4BD5458485FD0
:108EC00056312E322E31003880250000010000007E
:108ED0000A00000000000000000000000000000088
:108EE0000000000000000000000000000000000082
:108EF0000000000000000000010100000000000070
:108F0000000000000000000002030000000000005C
:108F10000000000000000000030500000000000049
:108F20000000000000000000040700000000000036
:108F30000000000000000000050500000000000027
:108F40000000000000000000060600000000000015
:108F50000000000000000000070700000000000003
:108F600000000000000000000808000000000000F1
:108F700000000000000000000909000000000000DF
:108F800000000000000000000A0A000000000000CD
:108F900000000000000000000B0B000000000000BB
:108FA00000000000000000000C0C000000000000A9
:108FB00000000000000000000D0D00000000000097
:108FC00000000000000000000E0E00000000000085
:108FD00000000000000000000F0F00000000000073
:108FE0000000000000000000101000000000000061
:108FF00000000000000000006A6F796675656C2E45
:109000006A6F796675656C696E672E636F6D2C3754
:1090100030313100000000000000000000000000BE
:109020000000000000000000000000000000000040
:109030000000000000000000000000000000000030
:109040000000000000000000000000000000000020
:109050000000000000000000000000000000000010
:109060000000000000004B46422D322E3447000025
:1090700000000000000000000000000000000000F0
:1090800000000000000000000000000000004B464F
:109090004231323334353600000000000000000059
:1090A00000000000000000040000000000000000BC
:1090B000C78E010820410020371100206400000005
:1090C0000200010000000000A490010820410020DF
:1090D00030110020660000000500010001000000C2
:1090E000C88E010820410020E41A00206B00000017
:1090F0003101040002000000F88F01082041002027
:109100004A1600202F050000AC00010003000000FB
:10911000A390010820410020401A0020DB05000038
:109120000200010004000000A89001082041002076
:1091300028110020DD0500000500010005000000E9
:10914000AC900108204100202C110020E205000015
:10915000050001000600000061002B2B2B000D0A0A
:10916000000041542B530D0A0041542B534F434BE5
:10917000413D5443502C746573742E6A6F79667543
:10918000656C696E672E636F6D2C373031310D0A57
:109190000041542B574B4D4F443D4E45540D0A0052
:1091A00041542B55415254464C3D343039360D0A0A
:1091B0000041542B4845415254454E3D4F46460DC3
:1091C0000A0041542B453D4F46460D0A0041542BA1
:1091D000454E544D0D0A0041542B49434349443FE9
:1091E0000D0A0041542B494D45493F0D0A00415499
:1091F0002B574946493D4B46422D322E34472C4B86
:1092000046423132333435360D0A0041542B536F08
:10921000636B65743D302C302C746573742E6A6FEB
:10922000796675656C696E672E636F6D2C373031AA
:10923000310D0A0000C1814001C0804101C0804160
:1092400000C1814001C0804100C1814000C1814016
:1092500001C0804101C0804100C1814000C1814006
:1092600001C0804100C1814001C0804101C08041F6
:1092700000C1814001C0804100C1814000C18140E6
:1092800001C0804100C1814001C0804101C08041D6
:1092900000C1814000C1814001C0804101C08041C6
:1092A00000C1814001C0804100C1814000C18140B6
:1092B00001C0804101C0804100C1814000C18140A6
:1092C00001C0804100C1814001C0804101C0804196
:1092D00000C1814000C1814001C0804101C0804186
:1092E00000C1814001C0804100C1814000C1814076
:1092F00001C0804100C1814001C0804101C0804166
:1093000000C1814001C0804100C1814000C1814055
:1093100001C0804101C0804100C1814000C1814045
:1093200001C0804100C1814001C0804101C0804135
:1093300000C1814000C0C101C30302C2C60607C705
:1093400005C5C404CC0C0DCD0FCFCE0E0ACACB0B75
:10935000C90908C8D81819D91BDBDA1A1EDEDF1FA5
:10936000DD1D1CDC14D4D515D71716D6D21213D395
:1093700011D1D010F03031F133F3F23236F6F73745
:10938000F53534F43CFCFD3DFF3F3EFEFA3A3BFB35
:1093900039F9F83828E8E929EB2B2AEAEE2E2FEFE5
:1093A0002DEDEC2CE42425E527E7E62622E2E32355
:1093B000E12120E0A06061A163A3A26266A6A76785
:1093C000A56564A46CACAD6DAF6F6EAEAA6A6BABF5
:1093D00069A9A86878B8B979BB7B7ABABE7E7FBF25
:1093E0007DBDBC7CB47475B577B7B67672B2B37315
:1093F000B17170B0509091519353529296565797C5
:10940000559594549C5C5D9D5F9F9E5E5A9A9B5BB4
:1094100099595898884849894B8B8A4A4E8E8F4F64
:109420008D4D4C8C448485458747468682424383D4
:109430004181804041542B41504E3D0000000000CE
:10944000000000000000000000000000000000001C
:10945000000000000000000000000000000000000C
:1094600000000000000038000000000000000000C4
:1094700000000000000000000000000000000000EC
:1094800000000000000000000000000000000000DC
:1094900000000000000000000000000000000000CC
:1094A0000000000066940108FC65002038110020CF
:1094B00000000000020001000000000066940108A6
:1094C000FC6500203A1100200100000001020008A4
:1094D0000100000067940108FC650020EC100020EA
:1094E000010800003C00D00702000000669401085B
:1094F000FC6500203A110020D10F0000010200108D
:109500000300000000000000000000000000000058
:10951000000000000000000000000000000000004B
:10952000000000000000000000000000000000003B
:10953000000000000000000000000000000000002B
:10954000000000000000000000000000000000001B
:10955000000000000000000000000000000000000B
:1095600000000000000000000000000000000000FB
:1095700000000000000000000000000000000000EB
:1095800000000000000000000000000000000000DB
:1095900000000000000000000000000000000000CB
:1095A00000000000000000000000000000000000BB
:1095B00000000000000000000000000000000000AB
:1095C000000000000000000000000000000000009B
:1095D000000000000000000000000000000000008B
:1095E000000000000000000000000000000000007B
:1095F000000000000000000000000000000000006B
:10960000000000000000000000000000000000005A
:10961000000000000000000000000000000000004A
:10962000000000000000000000000000000000003A
:10963000000000000000000000000000000000002A
:10964000000000000000000000000000000000001A
:10965000000000000000000000000000000000000A
:1096600000000000000000000000000000000000FA
:1096700000000000000000000000000000000000EA
:10968000000000000000000000000000002F0000AB
:1096900000000700070000147F147F1400242A7FB5
:1096A0002A12006264081323003649552250000034
:1096B0000503000000001C224100000041221C00A4
:1096C0000014083E08140008083E0808000000A026
:1096D0006000000808080808000060600000002022
:1096E00010080402003E5149453E0000427F400000
:1096F000004261514946002141454B310018141286
:109700007F10002745454539003C4A494930000152
:109710007109050300364949493600064949291EA1
:109720000000363600000000563600000008142203
:109730004100001414141414000041221408000203
:109740000151090600324959513E007C1211127C28
:10975000007F49494936003E41414122007F414155
:10976000221C007F49494941007F09090901003E47
:109770004149497A007F0808087F0000417F410085
:10978000002040413F01007F08142241007F4040FB
:109790004040007F020C027F007F0408107F003EE3
:1097A0004141413E007F09090906003E4151215EC9
:1097B000007F091929460046494949310001017FC6
:1097C0000101003F4040403F001F2040201F003F5C
:1097D0004038403F0063140814630007087008070E
:1097E00000615149454300007F41410000552A5521
:1097F0002A55000041417F0000040201020400409C
:1098000040404040000001020400002054545478BD
:10981000007F4844443800384444442000384444DD
:10982000487F00385454541800087E09010200187B
:10983000A4A4A47C007F080404780000447D4000B8
:10984000004080847D00007F102844000000417F9C
:109850004000007C04180478007C08040478003878
:109860004444443800FC242424180018242418FC00
:10987000007C0804040800485454542000043F4469
:109880004020003C4040207C001C2040201C003C2C
:109890004030403C004428102844001CA0A0A07C7C
:1098A000004464544C4414141414141400000000B4
:1098B00000000000000000000000FC0000000000AC
:1098C00002000000000C020C02000000000000007A
:1098D00090D0BCD0BC900003000300001824FE44CC
:1098E0008C000302070201001824D8B04C8000034A
:1098F00000010201C038E438E00001020201020266
:10990000080600000000000000000000000000F851
:109910000402000000010204000204F80000000438
:10992000020100009060F86090000000010000005B
:109930002020FC20200000000100000000000000AA
:109940000000080600000000202020202000000069
:109950000000000000000000000000020000000005
:109960000080601C0200040300000000F8040404EE
:10997000F8000102020201000008FC0000000002E1
:1099800003020000188444241800030202020200AB
:1099900008042424D80001020202010040B088FC1F
:1099A00080000000000302003C242424C4000102C3
:1099B00002020100F824242CC0000102020201006E
:1099C0000C04E41C0400000003000000D82424243C
:1099D000D80001020202010038444444F8000003A8
:1099E0000202010000001000000000000200000060
:1099F0000000200000000000060000000020508849
:109A0000040200000000010290909090900000007D
:109A10000000000000020488502000020100000045
:109A20001804C4241800000002000000F804E494A4
:109A3000F80001020202020000E09CF08000020334
:109A40000000030204FC2424D800020302020100E7
:109A5000F80404040C0001020202010004FC0404E6
:109A6000F80002030202010004FC24740C0002034B
:109A70000202030004FC24740C0002030200000034
:109A8000F0080444CC4000010202010004FC202044
:109A9000FC040203000003020404FC0404000202AC
:109AA00003020200000404FC040406040403000092
:109AB00004FC24D00C0402030200030204FC040092
:109AC0000000020302020203FC3CC03CFC00030055
:109AD0000300030004FC30C4FC0402030200030082
:109AE000F8040404F80001020202010004FC24242A
:109AF0001800020302000000F8848404F800010248
:109B00000207050004FC246498000203020003021B
:109B1000182424448C000302020201000C04FC04FB
:109B20000C0000020302000004FC0000FC04000121
:109B300002020100047C80E01C040000030000001D
:109B40001CE03CE01C00000300030000049C609C3F
:109B50000400020300030200041CE01C04000002D5
:109B6000030200000C84641C0400020302020300D0
:109B70000000FE020200000007040400000E30C0D6
:109B80000000000000010200000202FE00000004CC
:109B900004070000000402040000000000000000B0
:109BA0000000000000000808080808080000020083
:109BB00000000000000000000040A0A0C000000164
:109BC0000202030204FC2020C00000030202010084
:109BD00000C02020600000010202020000C020241A
:109BE000FC0000010202030200C0A0A0C0000001AE
:109BF000020202000020F8242404000203020200F2
